:020000040000FA
:06000000F0EF0FF012000A
:060008005AEFB7F01200F0
:0600180068EFB7F01200D2
:06002A0025EC08F014684B
:10003000156AFD0EDBCF08F0FE0EDBCF09F014C011
:100040000DF015C00EF0A4ECBBF008C0DEFF09C037
:10005000DDFF9DEC07F009E0E66A8DECBBF0E552B0
:10006000DF06010EF6E2DB06F4D72DEC07F00D6893
:100070000E6A14C008F015C009F0A4ECBBF004C06F
:1000800014F005C015F004C0DEFF05C0DDFF9DECD7
:1000900007F005E0DFCFE6FF8DECBBF0E552020E86
:1000A000E15C02E2E16AE552E16E2AEF06F0010E40
:1000B000D16E1200D16A12000501505101E1040015
:1000C00012000501010E506F1200FAEC07F0A3ECCC
:1000D00006F0FB0EDBCFEEFFFC0EDBCFEDFFDF50BB
:1000E00001E09D80E5522AEF06F025EC06F0030EB4
:1000F00004EC08F0EDCFDBFFDF5001E09D80A4ECC5
:1001000007F014C0F3FF15C0F4FF030EE15C02E238
:10011000E16AE552E16E2AEF06F0FAEC07F0A3EC93
:1001200006F0F90EDBCFEEFFFA0EDBCFEEFFFB0E93
:10013000DBCFEEFFFC0EDBCFEEFFDF5001E09D805A
:10014000E5522AEF06F025EC06F0050E04EC08F067
:10015000EECFDBFF030EEECFDBFF040EEECFDBFFB7
:10016000DF5001E09D80A4EC07F0030EDBCF16F01A
:10017000040EDBCF17F014C006F066EC07F0050E96
:10018000E15C02E2E16AE552E16E2AEF06F0050168
:10019000806B80C57FF580C569F580C568F5120064
:1001A000FAEC07F005016829DF6E070EDF5C01E35A
:1001B000DF6A6951DF5C02E1010E2ED06851BEECAE
:1001C00006F0ABEC07F06851BEEC06F08FEC07F0E0
:1001D000DFCF68F52DEC07F0000E1416F00E1516A3
:1001E000145002E1200E15180FE0FD0EDBCF16F0C3
:1001F000FE0EDBCF17F0000E1616F00E1716165077
:100200000AE1100E171807E1FD0EDB50010B03E1A8
:100210000901010E056F000EE5522AEF06F025ECEC
:1002200006F005016951685D02E1010E10D06951C7
:10023000BEEC06F01EEC07F06951BEEC06F010ECC7
:1002400007F0692B070E695D01E3696B000E2AEF69
:1002500006F0FAEC07F005017F29DF6E070EDF5C80
:1002600001E3DF6A8051DF5C02E1010E0DD07F51B6
:10027000C8EC06F0ABEC07F07F51C8EC06F08FEC51
:1002800007F0DFCF7FF5000EE5522AEF06F025ECF0
:1002900006F0050180517F5D02E1010E10D0805112
:1002A000C8EC06F01EEC07F08051C8EC06F010EC2C
:1002B00007F0802B070E805D01E3806B000E2AEFB4
:1002C00006F025EC06F0050EE12615DB000970E1CD
:1002D00050EC07F0A4DFF2EC07F0000969E180ECD4
:1002E00007F006E247EC06F095DAF2EC07F060D092
:1002F000010EDB50C00B2BE0A9EC06F0DBCF64F362
:10030000040EDBCF65F3010EDB50800B0DE08BECB0
:1003100006F0F5CF63F30301676B686B04C966F3FE
:100320006A6B6B6B696B07D00301C80E636F010EBC
:10033000676F686B666B020EDBCF1AFDDBCF5DFD6E
:1003400080EC06F09D900D0136899D8031D079ECCE
:1003500007F015E1100E151812E1020EDBCFE6FFD3
:1003600003C9E6FF02C9E6FF0BEC08F0D890E936B6
:10037000EA36E806FBE1F6EC06F01AE117D079EC74
:1003800007F016E1200E151813E1020EDBCFE6FF91
:1003900001C9E6FF00C9E6FF0BEC08F0D890E9368A
:1003A000EA36E806FBE1F6EC06F002E10901056B2E
:1003B000050EE15C02E2E16AE552E16E2AEF06F029
:1003C00025EC06F0050EE126A0DA000932E150EC3A
:1003D00007F05DDFF2EC07F000092BE180EC07F09D
:1003E00006E247EC06F047DAF2EC07F022D0010E05
:1003F000DB50800B1EE0A9EC06F0DBCF65F2040EAB
:10040000DBCF66F28BEC06F0F5CF64F20201686B8D
:10041000696B04C967F26B6B6C6B6A6B020EDBCFA6
:100420001CFDDBCF5FFD80EC06F09D900D01368D4D
:100430009D80050EE15C02E2E16AE552E16E2AEF81
:1004400006F025EC06F0FE0EDB50200A01E17FD01D
:10045000290A01E17CD0530A70E00E0A64E0770AB1
:100460005AE0670A50E0070A4BE0010A46E0030A37
:1004700041E06B0A37E01A0A2DE0090A28E0010A78
:1004800023E00F0A1EE0010A19E0030A14E0010A42
:100490000FE0070A0AE0010A05E0030A60E1F7EC51
:1004A00007F022D0F7EC07F017D0F7EC07F035D0C3
:1004B000DDEC07F019D0DDEC07F00ED0DDEC07F035
:1004C0002CD0E2EC07F010D0E2EC07F005D0E2EC23
:1004D00007F023D0E7EC07F0A0EC06F0060EEE6E76
:1004E000230E43D0E7EC07F0A0EC06F0B10EEE6E61
:1004F0001F0E3BD0F7EC07F008D0DDEC07F005D07D
:10050000E2EC07F002D0E7EC07F0A0EC06F0CF0E2B
:10051000EE6E2A0E2AD0E7EC07F0A0EC06F0B80E3B
:10052000EE6E260E22D08ADB2D0EEE6E090EA0ECAA
:1005300006F0890EEE6E0B0E18D080DB950EEE6E77
:100540000C0EA0EC06F0410EEE6E100E0ED076DB17
:10055000EE6AED6A18EC08F0EE6AED6A07D0F7EC87
:1005600007F0EEDB450EEE6E120EED6E73D36DDB13
:100570002DEC07F0166A176AFD0E0B6EB50E0C6EA9
:10058000060E0D6E0E6A14C006F066EC07F018EC4D
:10059000BBF002C014F003C015F004C016F005C093
:1005A00017F0800E1526000E162217220B6A0C6A11
:1005B000010E0D6E0E6A02C006F066EC07F0B0EC9C
:1005C000B6F006C014F007C015F008C016F009C058
:1005D00017F006C0F3FF07C0F4FF3CD3FAEC07F0B6
:1005E000050EF36EFE0EDBCFF4FFF350F45C05E274
:1005F000050EF36EFE0EF3CFDBFFFE0EDB50166E24
:10060000176AFE0EDB5086EC07F014C008F015C028
:1006100009F016C00DF017C00EF0A4ECBBF00850A6
:10062000DF6EDFCF37FD0D013751E8240D01386F44
:10063000030E0D013703F3CF39FD040E3703F3CF5B
:100640003AFDDF5086EC07F014C009F0DFCF0EF062
:10065000D8ECBBF00950E552FDD2F7DAECEC07F02C
:10066000F3CF51F5F4CF52F5F5D2EFDA040EE126CF
:100670009D900D0136919D800D01320E4A6F060E40
:100680004B6F020E4ACDDBFF030E4BCDDBFFDF6A63
:10069000DF6ADF509BDBEF503BE0310EDF5C38E27E
:1006A000DF5094DBEF507F0BE76E010EE7CFDBFFEF
:1006B000DBCF14F05F0EE76E1418E8AE02D01434EE
:1006C00003D0E750D88014540AE2200E146E010EB5
:1006D000DBCFE7FF1450E75E010EE7CFDBFF7E0EB6
:1006E000146E4B0E156E010E166E010EDBCF17F059
:1006F000186A196A17AE02D018681968C7EC07F0B3
:10070000F550E66EB1DBE552E750EF6EDF2AC1D758
:10071000ABDBEF6A0D014C6B51C518FD52C519FDDD
:100720009D903F0E0D0111170D0136819D80040E25
:10073000E15C02E2E16AE552E16E8CD2FDEC07F089
:1007400089D2FDEC07F00D0136B1FDD783D29D9023
:100750000D0136910D01119D9D801200400E0D017D
:100760001115146E010E0D01361514101200FAEC5D
:1007700007F0DF6ABDEC07F00800F55010E0F90E55
:10078000DB50DF5C0CE26ADAD950FD0FCEDBEF22E2
:10079000D950FA0FCADBEE22EE22DF2AEBD75EDA5F
:1007A000E55258D252DAFE0EDB50040A32E0070A54
:1007B0001CE0010A0EE0030A2CE19D900D01369920
:1007C0000D011191EFDA630EE66E030E58DB98DA35
:1007D00020D09D900D01369B0D011195E3DA000E9E
:1007E000E66E030E4CDBF7DA14D09D900D01369DBA
:1007F0000D011199D7DA640EE66E020E40DB0D0191
:10080000640E516F020E526F0D01640E596F020E8D
:100810005A6F20D2EFDBDF6A4FD868DA5EDB09E07F
:1008200065DAF4DA010E14DBDBCF1AFDDBCF5DFDF8
:10083000DF88BCDB52DB18E0B9DB0900F5500900AA
:10084000F5CFE7FF0800F5CFF8FFE7CFF7FFF66E2B
:100850000800F55009E0AADBD9DA020EF9DADBCF9D
:100860001BFDDBCF5EFDDF8A9D90DF500D0136134F
:100870009D80E552EFD1E9D937D838DA2EDB0CE08C
:1008800035DAC4DA030EE4DADBCF1CFDDBCF5FFD23
:100890009D900D01368D9D80DDD1D7D90DD89CDB83
:1008A000F3CF12FDF4CF13FDFC0EDBCF1AFD9D90AC
:1008B0000D0111819D80CED19D90CF0E0D01361777
:1008C000FA0E0D0111179D801200BFD90DD884DBDF
:1008D000F3CF16FDF4CF17FDFC0EDBCF1CFD9D9072
:1008E0000D0111899D80B6D19D900D01369D0D01A0
:1008F00011999D801200300E0D01361505E1050E8F
:100900000D01111501E1000C010C400E0D01361511
:1009100005E1100E0D01111501E1000C010C6ADB5F
:10092000CBDF4DDA7AECADF0E552E552110EF35C17
:10093000000EF45803E3100E49DAEF6A0D01630E5E
:100940004D6F030E4E6F0D01000E4F6F030E506F73
:10095000FD0EDBCFE9FFDB2AFE0EDBCFEAFF01E372
:10096000DB2AEFCFDFFFDF5028E090DAFC0E67DBF9
:1009700092DAEE52E9CF14F0EACF15F0E9CFE6FFB4
:10098000EACFE6FF83DAEE52E9CF16F0EACF17F0AE
:10099000E9CFE6FFEACFE6FFDFCFE6FF52DD186ED4
:1009A000050EE15E185087DA71DAFB0E48DB3ADBA0
:1009B000EE52EE6AED6A7FDACBD768DAEF6A32DBA5
:1009C000EF6A69DAEE52EE6AED6A9AD904DAFA0E43
:1009D000DBCF1BFD1BCD1AFDDBCF5EFD5ECD5DFDCC
:1009E0009D90300E0D0136139D80E55233D12DD9E7
:1009F00063DF140EE66E0D0EE66E120EE66E0D0E41
:100A0000E66EFE0EDBCFE6FF1CDD146E050EE15E2A
:100A100014509D90050E0D0111139D801BD14CDFCC
:100A20000301640E636F0301006F0301950E646F91
:100A30000C0E656F0301410E016F100E026F030172
:100A4000640E666F0301036F0301676B686B03013C
:100A5000046B056B0301696B0301066B010E030157
:100A60006A6F6B6B0301076F086B4AD9B4D99D900D
:100A7000300E0D0136139D801200300E0D0136151B
:100A80001200400E0D013615120005016951685D16
:100A900001E1000C010C050180517F5D01E1000CBA
:100AA000010CA8DAFE0EDBCFE6FFE66AC3EC17F016
:100AB000E552E552F350F41004E0FE0EDB50D00F87
:100AC00004D0FE0EDB50BF0F0A0FDF6EDF50E55281
:100AD000C1D0BBDAFD0EDBCFDEFFDBCFDDFF04DAFA
:100AE000EF5005E0DF2A010EFAE3DB2AF8D7FCD944
:100AF000FC0EDBCFEFFFF8D9010EB0DAEF6AADD90B
:100B000014C0F3FF15C0F4FF020EE15C02E2E16ADB
:100B1000E552E16E9FD09D929F82D08EF90E941681
:100B20000F0EBD6EBA6E1C0ECA6ECB680D01116B36
:100B30000D017F0E1E6F0D011A6F0D011B6F0D0150
:100B40001C6F0D011D6F0D01370E126F1A0E136F02
:100B50000D01370E146F1A0E156F0D01370E166F3B
:100B60001A0E176F0D01370E186F1A0E196F12003B
:100B7000810ECD6E9F90140EE66E30DDE552E80ECC
:100B8000E66E030EE66E69DDE552E5520D017F0E5D
:100B9000606F60CD5FFD60CD5EFD60CD5DFD0D01E0
:100BA000366B0D013B6B1200870ED56EB16AF18E6C
:100BB000F26A9D6AA06AAFDFB8EF05F046D8AA6A6C
:100BC000FE0EDB50A96EA69EA69CA680A85042D021
:100BD0003CDAA198AA6AFE0EDB50A96EFD0EDB502E
:100BE000A86EA69EA69CA684F250800B01E0010E82
:100BF000DF6EF250400B01E0010EE76E010EE7CF11
:100C0000DBFFF29EF29C550EA76EAA0EA76EA6827F
:100C1000DF50E8B0F28EE8A0F29E010EDB50E8B0A3
:100C2000F28CE8A0F29CA1A8FED7A198A694020E8F
:100C3000E15C02E2E16AE552E16E0CD0FC0EDBCF32
:100C4000E9FFFD0EDBCFEAFF1200D9CFE6FFE1CFCF
:100C5000D9FF1200E552E7CFD9FF12008ED9080064
:100C6000F550E66E83D9E552E750EF6E86D909005C
:100C7000F5CF14F00900F5CF15F00800F5CF16F008
:100C800075D9EE5215C0EEFF16C0EDFF1200020E30
:100C9000DBCFE6FF950E176E4F0E186E010E196E24
:100CA000DECF1AF0DDCF1BF01C6A060E0C6E0D6A4B
:100CB0000E6A1AC007F01BC008F01CC009F0E4EC73
:100CC000B6F004C01AF005C01BF006C01CF01750A7
:100CD0000424146E18500520156E19500620166E47
:100CE00014C0E6FF15C0E6FFE66E1200FC0EDBCF77
:100CF000F6FFFD0EDBCFF7FFFE0EDBCFF8FF120095
:100D00000D01630E4D6F030E4E6F0D01630E556F97
:100D1000030E566F1200EB0E146E500E156E010E80
:100D2000166EDECF17F0DDCF18F01838186A0F0BEB
:100D3000176E070E1716000E1816196AC7EF07F080
:100D4000ED6E18EF08F09D50010BDF6E9D90B6EF31
:100D500007F07FD9FF0E14160F0E151614C0E6FF0C
:100D600015C0E6FFB7EC02F0E552E552030EF3CFF3
:100D7000DBFF040EF4CFDBFF030E1200030DF3CFF5
:100D8000E9FFF4CFEAFF530EE926050EEA2212002E
:100D9000030DF3CFE9FFF4CFEAFF6A0EE926050E53
:100DA000EA2212009D80210EE66EFB0EDBCFE6FFED
:100DB000FC0EDBCFE6FFFD0EDBCFE6FF1200FD0EE3
:100DC000DBCFE6FFFE0EDBCFE6FF1200E76ECED8EC
:100DD000E7502EEF08F00D01000E4F6F030E506F1D
:100DE0000D01000E576F030E586F1200060EE92614
:100DF000090EEA22EECFE6FFEFCFE6FF90DD146E9C
:100E0000050EE15E1450DF50010B12000900F5CF12
:100E1000E6FF0900F5CFE6FF0800F5CFE6FF120078
:100E2000020E1CD9EF50E66EFB0EDBCFE9FFFC0E85
:100E3000DBCFEAFFE552E750EF6E1200EECF14F081
:100E4000EECF15F093D814C0EEFF15C0EDFF1200E1
:100E5000E66EA8DCC7D8FB0E1200FD0EDBCF14F047
:100E6000FE0EDBCF15F01200DF50E76E020EDBCF77
:100E7000E9FF030EDBCFEAFFE7502EEF08F0E66E46
:100E800076DC146E060EE15E145012004DCDE9FFC3
:100E90004ECDEAFF12004FCDE9FF50CDEAFF120020
:100EA000D950020FE66E000EDA20E66ED9CFE6FFCB
:100EB000DACFE6FF12000D01030E4D27000E4E2380
:100EC0000D01030E4F27000E5023120015C007F02E
:100ED00016C008F017C009F012000900F55009000B
:100EE000F5100800F5101200DECFE9FFDDCFEAFFB4
:100EF0001200AFD8000E1416F00E15161450120082
:100F0000A8D8390E145C000E15581200156AE83086
:100F10007F0B146EF00E1426000E15221200020E26
:100F20009DD8FC0EDBCFEFFF1200E96EFF0EDA203A
:100F3000EA6E030EEE26000E1200D9CFE9FFDACFDB
:100F4000EAFFEE50ED101200010EDBCF14F0020E9E
:100F5000DBCF15F01200FD0EDBCFEEFFFE0EDBCF78
:100F6000EDFF1200450EEE6E120E1200FD0EDBCFED
:100F7000E9FFFE0EDBCFEAFF1200FA0EDBCFF6FF31
:100F8000FB0EDBCFF7FFFC0EDBCFF8FF1200145097
:100F90001724F36E15501820F46E16501920F86EB1
:100FA000F4CFF7FFF3CFF6FF080012009FDE030E29
:100FB000F626000EF722F822120040DE2F0EEE6E0B
:100FC000140E12003BDE560EEE6E160E120036DECA
:100FD000AB0EEE6E180E1200F2DEB7EC02F0E55228
:100FE000E5521200E552E552E552E552120026DEC6
:100FF000B2EF07F02ADEE652120027DEE0DE35EC23
:1010000003F0E552E5521200E1269DDE010EEECF1F
:10101000DBFF020E120068DF010EE916000EEA1671
:10102000010E120033DFEE52EE6AED6A4BEF07F06D
:10103000FA0EDBCFE9FFFB0EDBCFEAFF1200DBCFBE
:10104000EFFF29DFDBCFEFFF1200FFDD020EE1260D
:101050001200DECF14F0DDCF15F01200E926000EED
:04106000EA2212006E
:0C1064006EEC0DF0FB0EDBCFF3FFDB06A3
:10107000F35000090AE0BCEC0DF0FA0E27EC0EF07C
:10108000F3E1151CF1E1010E01D0000E9DEF0DF012
:101090006EEC0DF03B0EE12402E3E168E652E16EF6
:1010A000010EDB6A020EDB6AF90EDBCFF6FFFA0EE9
:1010B000DBCFF7FFFB0EDBCFF8FF0800F550DF6E4C
:1010C000DF5002E1C1EF0CF0250EDF5C02E0B4EF6F
:1010D0000CF0030EDB6A040EDB6A050EDB6A060EFB
:1010E000DB6A070EDB6AD6EC0CF02D0EDF5C0CE041
:1010F0002B0EDF5C09E0200EDF5C06E0230EDF5CD8
:1011000003E0300EDF5C1AE1DF50300A14E0130A0E
:101110000FE0030A0AE00B0A05E0060AE4E1030E09
:10112000DB80E1D7030EDB82DED7030EDB84DBD767
:10113000030EDB86D8D7030EDB88D5D72A0EDF5CFB
:101140001BE1D2EC0CF020EC0DF010E0030EDB8084
:1011500008680968130EDBCF0DF0140EDBCF0EF01C
:101160002DECB7F0040E06C0DBFF03D0130E09EC24
:101170000DF0D6EC0CF00BD0090EDB6A77EC0DF01D
:1011800003E0EBEC0DF0FAD7090E09EC0DF0030EBD
:10119000DBB0DB982E0EDF5C1BE1D6EC0CF02A0EE8
:1011A000DF5C0BE1D2EC0CF020EC0DF003E1130E50
:1011B0005BEC0DF0D6EC0CF00BD0090EDB6A77EC93
:1011C0000DF003E0EBEC0DF0FAD7090E5BEC0DF03F
:1011D000680EDF5C07E1D6EC0CF0680EDF5C1DE109
:1011E000030E18D0740EDF5C17E07A0EDF5C14E09B
:1011F000480EDF5C06E0540EDF5C03E05A0EDF5C55
:1012000002E1020E07D06C0EDF5C03E06A0EDF5CC9
:1012100004E1010EAEEC0DF0C9DBDF506E0A01E116
:101220007FD31E0A01E192D1200A01E18FD13F0A4A
:1012300001E149D11A0A01E146D10D0A01E143D188
:10124000200A01E140D13A0A01E13DD1200A01E141
:101250003AD1260A01E135D10D0A01E132D11A0A4B
:1012600001E1D9D0200A4AE0300A1FE0460A0EE028
:10127000250A01E083D3D950F90FE96EFF0EDA2079
:10128000EA6E010EEE5E000EEE5AEE5ABCEC0DF068
:10129000250EE66E95DB03E1151C01E169D3B8EC80
:1012A0000DF001E26BD3DB2A69D3080EDB6A040E72
:1012B000DB50010806E2040EDB0480EC0DF0DB508D
:1012C0008BDB080EDB5009E0030EDB50010B05E160
:1012D00072DB01E04DD3080EDB6A64DBEFCFDFFF8A
:1012E00030EC0EF003E1151C01E142D3B8EC0DF037
:1012F00001E3DB2A60DB01E141D33AD3070EDB5087
:1013000002080FE1FCEC0DF0030EC3EC0DF00E0E25
:10131000EECFDBFF0F0EEECFDBFF100EEECFDBFFCD
:1013200020D0F70EDBCF17F0F80EDBCF18F0020E4F
:10133000175E000E185AF70E17C0DBFFF80E18C024
:10134000DBFF17C0E9FF18C0EAFFB3EC0DF0166A27
:101350000E0E14C0DBFF0F0E15C0DBFF100E16C003
:10136000DBFF0E0EDBCFE6FF0F0EDBCFE6FF100E2E
:10137000DBCFE6FF88ECADF0E552E552E552130E07
:1013800007C0DBFF140E08C0DBFF060EDB5005E0D4
:10139000130EF7EC0DF001E26ADB1BEC0EF002E23B
:1013A000130E37DBDEEC0DF006E0040EF7EC0DF06B
:1013B00002E2050E2EDB030EDBB005D0FCDA01E005
:1013C000D7D2080EDB6A090EDB6A0E0EDBCFF6FF02
:1013D0000F0EDBCFF7FF100EDBCFF8FF0800F55044
:1013E000DF6EDF5014E021EC0EF011E230EC0EF075
:1013F00003E1151C01E1BCD2BBDB01E3DB2A090ED2
:10140000DB2AD9500E0FE96E000ECBDBE7D7D3DA1B
:1014100001E1B4D2ADD2C6DA110EEECFDBFF120E6F
:10142000EDCFDBFF110EDBCFE6FF120EDBCFE6FFC9
:101430007AECADF0E552E552130EF3CFDBFF140E5C
:10144000F4CFDBFF060EDB5004E0130ED0DB01E22D
:101450000EDB1BEC0EF002E2130EDBDAAFDB05E075
:10146000040EC5DB02E2050ED4DA030EDBB005D0B4
:10147000A2DA01E07DD2080EDB6A090EDB6A110EEA
:10148000DBCFE9FF120EDBCFEAFFEFCFDFFFDF504C
:1014900014E0D7DB12E2E4DB03E1151C01E168D2C2
:1014A00067DB01E3DB2A090EDB2A110EDB2ADBCF27
:1014B000E9FF120EE8E3DB2AE6D77DDA01E15ED22E
:1014C00057D2030EDB8E070EDB0410E195DB040E12
:1014D0005ADB0A0EEECFDBFF0B0EEECFDBFF0C0E5E
:1014E000EECFDBFF0D0EEECFDBFF6CD0070EDB5037
:1014F00003082CE1030EDBAE0DD0B2DA020E76DA71
:10150000EFCF14F0156A166A176A14AE39D0156851
:10151000166835D0F70EDBCF15F0F80EDBCF16F0DE
:10152000020E155E000E165AF70E15C0DBFFF80E00
:1015300016C0DBFF15C0E9FF16C0EAFFEFCF14F0BD
:101540000A0E14C0DBFF0B0EDB6A38D0070EDB502F
:10155000020809E1030EDBAE04D059DB16AE10D051
:101560000ED055DB0DD0030EDBAE12D079DA020EB1
:101570003DDAF9DA166A176A15AE02D016681768EE
:10158000E2DA0C0E16C0DBFF0D0E17C0DBFF1AD01F
:10159000F70EDBCF16F0F80EDBCF17F0020E165E5B
:1015A000000E175AF70E16C0DBFFF80E17C0DBFF50
:1015B00016C0E9FF17C0EAFFD6DAC5DA0C0EDB6AFF
:1015C0000D0EDB6A060EDB5005E1010EF36E050E13
:1015D000F3CFDBFF150EDB6A160EDB6AD950370F2F
:1015E000146E000EDA20156E390E14C0DBFF3A0EB1
:1015F00015C0DBFF380EDB6A080EDB6A0A0EAEDAB6
:10160000DF50780A12E0200A10E0280A0CE0200AD5
:101610000AE03F0A06E00D0A02E0200A08E1020E95
:1016200005D0080E03D0080EDF26100E97DA030E41
:10163000DBBE02D0DB92DB94DB50800B24E08ADA45
:10164000D890030EEB50000A08E6000EEE5C000E88
:10165000EE58000EEE58000EEE5815E213DA0B6845
:101660000C680D680E6818ECBBF00A0E02C0DBFFB8
:101670000B0E03C0DBFF0C0E04C0DBFF0D0E05C01C
:10168000DBFF2D0E08D0030EDBA202D02B0E03D001
:10169000DBA408D0200EF36E170EF3CFDBFF150E80
:1016A000DB2A02D0170EDB6A050EDB5003E1B7D947
:1016B00001E189D0CC0E146E770E156E010E166EF8
:1016C000070EDBCF17F0186A196A1A6A17C00BF0F9
:1016D00018C00CF019C00DF01AC00EF0D3D950ECA0
:1016E000BBF014500224F36E15500320F46E165014
:1016F0000420F86EF4CFF7FFF3CFF6FF0800090ED1
:10170000F5CFDBFF580EDF5C0FE1610EF36E090EC3
:101710007BD90AE3200E146E090EDBCFE7FF1450CD
:10172000E75E090EE7CFDBFF070EDBCF14F0156A8B
:10173000166A176A0FDA14C00BF015C00CF016C049
:101740000DF017C00EF0EECF06F0EECF07F0EECFA3
:1017500008F0EFCF09F050ECBBF009C0EDFF08C076
:10176000EDFF07C0EDFF06C0EFFF390EDBCFE9FF4D
:10177000DB063A0EDBCFEAFF01E2DB06090EDBCF28
:10178000EFFF150EDB2A4BD995E1030EDBA61DD02A
:101790006F0EDF5C06E1C1D918E3150EDB285BDABA
:1017A00014D0780EDF5C09E0580EDF5C06E0620EB4
:1017B000DF5C03E0420EDF5C08E1020EF36E160E02
:1017C000F3CFDBFF02D0150EDB6A030EDB50100BEC
:1017D0000EE0040EDBCF14F0050EDB50D88014545D
:1017E00006E2060EDB5003E1040EDB5034DA95D935
:1017F0000AE2050EDBCFE7FF150EDB50E75E050EB4
:10180000E7CFDBFF02D0050EDB6A040EDBCF14F05E
:10181000160E45D9D880145414E2160EDBCFE6FF1D
:10182000150EDBCFE6FF040EDBCFE6FF050EDB5027
:10183000E552E75CE552D880E754E552D880E7549A
:101840005FD9030EDB50010B0BE1080EDB5008E003
:10185000B2D801E08DD0080EDB50BED8080EDB6A8E
:10186000170EDB5007E088D9170EF1D903E1151CDC
:1018700001E17ED0160EDB5016E07ED9300EE66E0A
:101880009FD802E1151C74E077D9DFCFE6FFD6ECD4
:10189000BAF0E552E552E552F4CF15F00001F31C21
:1018A00002E1151C65E0050EDBCF14F0160EDB50CF
:1018B000D880145409E2050EDBCFE7FF160EDB508B
:1018C000E75E050EE7CFDBFF300EE66E050ECBD9E7
:1018D0004FE1390EDB2ADBCFE9FF3A0E01E3DB2AC9
:1018E000DBCFEAFF090EEFCFDBFFDB500EE044D980
:1018F000090EADD902E1151C3BE0390EDB2ADBCF26
:10190000E9FF3A0EEDE3DB2AEBD755D831E1160EAD
:10191000DBCFE6FF080EC3D8E552E7245DD82ED012
:10192000070EDB50030A1CE0010A14E0030A07E07B
:101930007BD9DBCFEEFF020EDBCFEDFF1FD0F5D85A
:10194000196A17AE02D0186819682CD8BCD819C00B
:10195000EEFF14D0EAD817BE186824D8B4D80ED039
:1019600063D9DBCFEFFF0AD07BD905E1151C03E17A
:10197000F368F46810D0FCD801E3DB2A79D95DEF75
:1019800008F0010EDBCF14F0020EDBCF15F014C00F
:10199000F3FF15C0F4FF3B0EE15C02E2E16AE552A1
:1019A000E16ECBD029D9020EC3EF0DF061D908004A
:1019B000F550DF6E1200200EE66E080E33EF0EF0CB
:1019C000D6ECBAF0E552E552E552F3CF14F0F4CF7D
:1019D00015F00001F31C1200146E156AD950010FA6
:1019E0004DD91450EE261550ED221200185E000E4F
:1019F000195AF70E18C0DBFFF80E19C0DBFF18C02C
:101A0000E9FF19C0EAFF1200DBCFF4FFF350F45CEA
:101A10001200DB50E76E040EE7CFDBFF12000A0E68
:101A2000DBCF14F00B0EDBCF15F00C0EDBCF16F076
:101A30000D0EDBCF17F014501510161017101200F2
:101A4000130EEECFDBFF140EEDCFDBFF130EDBCF5B
:101A500014F0140EDBCF15F00001800E15141200E7
:101A6000F70EDBCF18F0F80EDBCF19F01200050EE1
:101A7000DB50E66ED950130F01D9E552E750EE6EF8
:101A8000ED6A12000A0EDBCF06F00B0EDBCF07F07B
:101A90000C0EDBCF08F00D0EDBCF09F01200DBCF10
:101AA000E6FF150EDBCFE6FF050EDB50E552E7241F
:101AB000E552E7241200DB50CED8010EF36E060E7D
:101AC000F3CFDBFF1200EE50EFCFEAFFE96E16C056
:101AD000EEFF17C0EEFF18C0EEFF1200D9CFE6FFF1
:101AE000DACFE6FFE1CFD9FFE2CFDAFF1200DFCF96
:101AF000E6FFE66AC3EC17F0E552E552F350120038
:101B0000E76E080EE7CFDBFF1200EECF14F0EECF4A
:101B100015F0EFCF16F0176A1200050EDBCF14F0A8
:101B2000150EDB50D88014541200010EDBCF16F0D6
:101B3000020EDBCF17F0186A1200E552E5CFDAFF8C
:101B4000E7CFD9FF12000A0E14C0DBFF0B0E15C041
:101B5000DBFF1200D9500A0F3EEF0EF0F36E070EB6
:101B6000F3CFDBFF1200EECF14F0EFCF15F0120031
:101B7000010EDB2A020E1200FC0EDBCFE6FFFD0E8B
:101B8000DBCFE6FF1200145E000E155AF70E14C0EC
:101B9000DBFFF80E15C0DBFF14C0E9FF15C0EAFF3C
:101BA0001200DA20EA6EEF2AEECFF6FF000EEF22E7
:101BB000EECFF7FFEF22EECFF8FF1200040EDBCFDF
:101BC000E6FF130EDB50E552E75C9ADFDB5004DFE3
:101BD000060EDB501200090EDB500A0DF350DF2415
:101BE000D00FE76E090EE7CFDBFFD6EF0CF0DB502E
:101BF000F36E050E04EF0DF0F70EDBCF14F0F80EC8
:101C0000DBCF15F01200DFCFE6FFE0EF0CF028DFAE
:101C1000030EECDE85EF0DF032EC08F0E552E552F4
:101C2000E552E55200091200BDDEEE50EFCFEAFFAB
:101C3000E96E010E1200130EDB50F36E040E04EF7A
:101C40000DF0040EDB50F36E090E04EF0DF0DBCF48
:101C5000E6FFE0EF0CF0E76E050EE7CFDBFF1200CA
:101C60008BDF03EF0EF0DBCFE6FF86DF0CEF0EF02D
:101C7000D950F90FE96EFF0ED1EF0DF0E96E000EAD
:061C8000DA20EA6E1200FA
:0A1C86009D989D9AC6D808019D6B39
:101C9000949C948E9F9A9F98240EAC6E900EAB6E7F
:101CA0007E86800EE66E250EE66EE66AE66A36D819
:101CB000CCEF0FF061D9186A2D0E196E310E1A6E25
:101CC000010E1B6E18C006F019C007F01AC008F00C
:101CD000096EFB0EDBCF0BF0FC0EDBCF0CF0FD0E24
:101CE000DBCF0DF0FE0EDBCF0EF050ECBBF006C0EC
:101CF00014F007C015F008C016F009C017F014065C
:101D0000000E155A165A175AD89017321632153235
:101D1000143214C0F3FF15C0F4FF33D12DD9030ED4
:101D2000E126D950FB0FE96EFF0EDA20EA6EEECF06
:101D3000E6FFEECFE6FFEECFE6FFEFCFE6FFBADF3E
:101D40002BD9F3CFDEFFF4CFDDFF9D50200B03E155
:101D50009D50100B06E0010EF36E020EF3CFDBFF79
:101D600002D0020EDB6A9D989D9ADECF14F0DDCF83
:101D700015F015C014F0156A14507F6EDF50AF6E69
:101D8000020EDB5002E09D889D8A030EE15C02E2B8
:101D9000E16AE552E16EF5D09E50100B05E09D50D2
:101DA000100B02E00AD8010C9E50200B05E09D505C
:101DB000200B02E010D8010C000CDED8E65207D947
:101DC00076D8E552E552000903E0DF50AD6E01D050
:101DD0009D98E552D6D0D0D8E652ABA203D0AB98AE
:101DE000AB880BD0AE50DF6EABB407D0DFCFE6FFD1
:101DF000A80EE66E080EDDD802D008019D81E552DE
:101E0000C0D0EAD801E1000C010CE6D803E1A751EB
:101E1000010B01E1000C010C320EE66EC90EE66EFC
:101E2000050EE66EA80EE66E080EBBD8640EE66ED2
:101E3000660EE66E070EE66EA20EE66E080ED1EF97
:101E40000FF09AD89D9AA1D8A80EE66E080EE66EFD
:101E5000EBECB8F0A1D8000903E09D8A010E02D096
:101E60009D8A000E8ED088D80801ADB113D0AC5138
:101E7000EA6AA825E96EA951EA22EF50E66EFD0E46
:101E8000DBCFE9FFFE0EDBCFEAFFE552E750EF6E56
:101E9000010E01D0000E75D06FD89D98FE0EDBCFDD
:101EA000E6FFA20EE66E080E84D89D886AD064D83C
:101EB0006CD8A20EE66E080EE66EEBECB8F06CD8AD
:101EC00060D05AD889D80DE17BD85FD87AECADF0D4
:101ED000E552E552F3CFA0F8F4CFA1F813D8010EE4
:101EE00001D0000E4ED048D877D80AE169D8FB0E51
:101EF000DBCFA0F8FC0EDBCFA1F804D8010E01D097
:101F0000000E3FD069D81BE0A051A11113E0A751EA
:101F1000020B10E19EC8E9FF9FC8EAFF9E2B000E4E
:101F20009F23EF50E66EB8DFE5520801A007000ED0
:101F3000A15BEAD7A051A11102E19E6B9F6B120039
:101F400008019E6B9F6B0CEF0FF016D8E65208014C
:101F5000ADB110D03CD887DFE552E552DFCFE6FFC8
:101F6000A8EC19F0E552000905E131D86ADFE55225
:101F7000E552EDD7E55205D0D9CFE6FFE1CFD9FF45
:101F80001200E552E7CFD9FF1200FD0EDBCFE6FFCE
:101F9000FE0EDBCFE6FF1200E552E552E552E552B8
:101FA0001200E66EB5ECB8F0146E050EE15E14504A
:101FB0001200E66ECFECB8F0E552E552E5521200A1
:101FC000FD0EDBCF9EF8FE0EDBCF9FF81200D9CFBF
:101FD000E6FFDACFE6FF120008019E519F111200C2
:101FE0001EEE00F02EEE00F0F86A019CEFECBBF064
:101FF00087ECBAF0FFEC17F0B6ECB7F0FBD71200A5
:10200000303030007878005000303031007878017E
:1020100050003030320078780250003030330010F9
:1020200010035000303034007878045000303035E0
:10203000006868055000303036007878065000306F
:10204000303700C0C0075000303038007878085072
:10205000003030390078780950003031300078781D
:102060000A50003031310078780B500030313200A6
:1020700078780C50003031330078780D50003031D2
:10208000340010100E50003031350078780F5000B9
:1020900030313600707010500030313700787811D0
:1020A00050003031380078781250003031390078E3
:1020B00078135000303230007878145000303231CC
:1020C00000787815500030323200787816500030A1
:1020D000323300B8B81750003032340078781850D6
:1020E0000030323500181819500030323600787838
:1020F0001A50003032370078781B500030323800E8
:1021000078781C50003032390078781D5000303318
:10211000300078781E50003033310078781F50003E
:102120003033320060602050003033330078782143
:10213000500030333400C0C02250003033350078B6
:1021400078235000303336002020245000303337BD
:1021500000787825500030333800787826500030E9
:1021600033390078782750003034300078782850A0
:1021700000303431007878295000303432007878DB
:102180002A50003034330060602B5000303434006B
:1021900078782C500030343500C0C02D50003034D9
:1021A000360078782E50003034370078782F500081
:1021B0003034380078783050003034390078783155
:1021C0005000343730007878325000343739007896
:1021D0007833500034374100909034500034393710
:1021E000007878355000343938007878365000342B
:1021F000394100D8D837500036303100787838501F
:1022000000363032007878395000363033002828D4
:102210003A50003630340078783B50003630350084
:1022200078783C50003630360070703D50003630C3
:10223000370078783E50003631300078783F5000D3
:1022400036323000B8B8405000363330007878412C
:10225000500036343000787842500036353000086F
:102260000843500036363000787844500036373016
:1022700000787845500036314100505046500036C5
:102280003241007878475000363341007878485022
:10229000003634410098984950003635410078782E
:1022A0004A50003636410078784B500036374100AE
:1022B000E8E84C50003637330078784D5000363718
:1022C000340078784E50003734300030304F5000B2
:1022D00037343100787850500037343200787851F4
:1022E000500037343300787852500037353000785A
:1022F00078535000373531007878545000373532F4
:1023000000C8C8555000373533007878565000372C
:102310003534007878575000373535001010585054
:1023200000373536007878595000373537007878DF
:102330005A50003738390058585B50003830380050
:1023400078785C50003830390078785D5000383942
:10235000440078785E50003934310078785F50005E
:10236000393432007878605000393433007878613D
:1023700050003630410078786250003035420078A5
:102380007863500030353000787864500030353153
:102390000078786550003035410078786650003418
:1023A00036300078786750003937300078786850D8
:1023B0000039373100787869500039373200787841
:1023C0006A50003937330078786B50003937340061
:1023D000A8A86C50003937350078786D500039372F
:1023E000360078786E500039373700F0F06F5000C3
:1023F0003139380078787050003435390078787188
:102400005000383732004040725000383930007880
:10241000787350003839380078787450003631427B
:102420000088887550003632420078787650003641
:10243000334200787877500036344200D0D078505C
:102440000036354200787879500036364200787888
:102450007A50003637420020207B5000363038005A
:1024600078787C50003638300078787D50003638E7
:10247000410068687E50003638420078787F50000E
:1024800036304200787880500038353200B0B08164
:102490005000323430007878825000323431007885
:1024A0007883500039393930000484500039393983
:1024B000310001855000656E640078780000006589
:1024C0006E64007878000000656E64007878000023
:1024D00000656E64007878000000656E64007878AE
:1024E000000000656E64007878000000656E64008E
:1024F0007878000000656E64007878000000656EF2
:102500006400787800000000000000000000000077
:1025100000000000000000000000000000000000BB
:1025200000000000000000000000000000000000AB
:10253000000000000000000000000000000000009B
:10254000000000000000000000000000000000008B
:10290000060007780100FB080000040000000278C0
:102910000100FB05000005000000DD770100FF025B
:10292000000001000000F8770100000900000A0023
:102930000000EE770100F10800000A000000EC77CB
:0A2940000100F20700000200000091
:06294A0086DAE6526EDAA7
:102950007AECADF0E552E552F350DF6EDF501E0821
:1029600002E21E0EDF6E07DB06E2A0DAF9DA86DA93
:10297000FEE1010E69DA5ADADFCFE6FFF1DA7EDA3C
:10298000FEE1020E61DAE5526CD266DA040EE1264F
:1029900094DAEF500EE091DAEFCF16F0176A16BE18
:1029A0001768D4DA06E0FD0EDB2AFE0EF1E3DB2A1F
:1029B000EFD78ADA42DAEFCF16F0176A16BE176839
:1029C000CADA08E0C0DA06E0020EDB2A030EF2E300
:1029D000DB2AF0D7B8DA04E094DA01E3DB2A58DA2C
:1029E000C3DA0BE2B0DA09E094DADECFE6FFDDCF3E
:1029F000E6FFABDFE55294DA01D0010E146E040E4F
:102A0000E15C02E2E16AE552E16E14502AD224DA76
:102A1000040EE12652DAEF500EE04FDAEFCF16F057
:102A2000176A16BE176892DA06E0FD0EDB2AFE0E64
:102A3000F1E3DB2AEFD748DA00DAEFCF16F0176AB6
:102A400016BE176888DA08E07EDA06E0020EDB2A96
:102A5000030EF2E3DB2AF0D776DA04E052DA01E380
:102A6000DB2A16DA81DA10E26EDA0EE052DA87EC4F
:102A7000B4F0E552E552F350E66EDECFE6FFDDCF6F
:102A8000E6FF3CD84DDA01D0010E146E040EE15C75
:102A900002E2E16AE552E16E1450E3D14CDA1EE243
:102AA0004EDAECD9FEE1010EB2D9DF5009E0BED911
:102AB000DFCFE6FFB4D9050EE1D9FEE1020EA7D9BA
:102AC000DF50E76EFB0EDBCFE9FFFC0EDBCFEAFF4A
:102AD000E750E926000EEA22EF6A0DD07D0EE66E81
:102AE000660EE66E010EE66EA1D961ECADF0146ED5
:102AF000050EE15E1450000EE552B3D1ADD93BDABC
:102B00000DE2D950FC0FE66EFF0EDA20E66E010EE4
:102B1000E66E26DAB3D9FEE1000E96D9A2D10BDA21
:102B200014E20DDAABD9FEE1000E71D9DFCFE6FF7A
:102B3000E66A760EE66E660EE66E010EE66E76D9F3
:102B400031ECBAF0146E070E0BD0670EE66E660E0F
:102B5000E66E010EE66E6AD92AECADF0146E050E33
:102B6000E15E1450000EE5527CD1E5D92EE2E7D9A2
:102B700085D9FEE1010E4BD9DF5027E0290EE66E24
:102B8000D9EC24F0E552000909E10601FE2BDFCF64
:102B9000E6FFA4EC24F0E552000902E0010E16D095
:102BA000000EE66E070EE66EDFCFE6FF38D9050EA3
:102BB00065D9FEE1020E2BD939D9010EE66E2FD967
:102BC000050E5CD9FEE1000E22D9000EE55249D176
:102BD00043D9E652DF6AFE0EDB50290826E10601E2
:102BE000FE5123E0FE07FE511EE1FF51040A12E0F0
:102BF000070A0CE0010A06E0030A13E1B8D9B9ECB0
:102C000029F00ED0B4D9D0EC29F00AD0B0D9E7EC35
:102C100029F006D0020EE66EAAD9FEEC29F0E552A4
:102C2000E5520601FF6B010EDF6EDF50E55219D150
:102C300013D9E652DF6A0601FE5128E001017851FE
:102C4000791124E04ED9250816E1010EDF6EFEEC65
:102C500022F047D908E045D9290805E00701642B8F
:102C6000000E6523F6D73DD92908ECE10701642B56
:102C7000000E6523E7D7010E0101AE1507E0DF5016
:102C800005E0AFC1E6FFA5EC23F0E552E552E9D03F
:102C9000E3D8C5D8000E145C500E155817E3D95070
:102CA000FD0FE96EFF0EDA20EA6E8F0ED880EE542B
:102CB000510EED540BE3BAD8B2D8000E145E500E8C
:102CC000155A5CD952DFE5522BD901D0010EC9D07B
:102CD000C3D8020EE126DE6ADD6A46D915E2E66A4D
:102CE000200EE66EE66A03D9050EC8D8FEE1000E96
:102CF0001CD979ECA2F0166E060EE15E1650DF2AA2
:102D0000010EEBE3DB2AE9D7146E020EE15C02E26E
:102D1000E16AE552E16E1450A4D09ED8020EE1267D
:102D2000FD0EDBCFDEFFDBCFDDFFE1D8F80EDBCF22
:102D300018F0F90EDBCF19F0FD0EDB501824166EDB
:102D4000FE0EDB501920176E1650145C17501558E4
:102D500055E2DECF1AF0DDCF1BF01C6A050ED890CD
:102D60001A361B361C36E806FAE1D950FA0FE96E1E
:102D7000FF0EDA20EA6EEE501A24176EEE501B207A
:102D8000186EEE501C20196EFD0EDBCF1DF0FE0EEE
:102D9000DBCF1EF01F6A050ED8901D361E361F367B
:102DA000E806FAE11D50175C146E1E501858156E97
:102DB0001F501958166EE2D8E66E200EE66EE66ACF
:102DC000DECF20F0DDCF21F0050ED8902036213661
:102DD000E806FBE1000E2026040E212220C0E6FFBB
:102DE00021C0E6FFE66A43ECA2F0226E080EE15E27
:102DF0002250DF2A010E99E3DB2A97D7146E020EC8
:102E0000E15C02E2E16AE552E16E14502AD08DD80D
:102E100031ECA3F0166E060EE15E16501200FD0EA8
:102E2000DBCF14F0FE0EDBCF15F01200FB0EDBCF74
:102E3000E6FFFC0EDBCFE6FF1200020EDBCFE9FF60
:102E4000030EDBCFEAFF120070D81CECA2F0166E66
:102E5000070EE15E16501200D9CFE6FFE1CFD9FF91
:102E60001200E552E7CFD9FF1200E552E552F3CF49
:102E700014F0F4CF15F0F350F4101200D89014367B
:102E80001536E8061200900E145C010E155812005B
:102E9000EF6A6DD8FE0EDBCFE6FFFCECB4F0E55236
:102EA000E55206C0DEFF07C0DDFF1200D9CFE6FF06
:102EB000DACFE6FF010EE66E1200FD0EDBCFE9FF72
:102EC000FE0EDBCFEAFF1200FD0EDBCF08F0FE0E98
:102ED000DBCF09F0020E08C0DBFF030E09C0DBFFE9
:102EE000120064C7E9FF65C7EAFFEF501200DECFAA
:102EF00014F0DDCF15F0120016C0E6FF17C0E6FF94
:102F00001200020EDBCFE9FFDB2A030EDBCFEAFF64
:102F10001200020EDBCFE6FF030EDBCFE6FF12004E
:102F2000E552E552E552000E12001426040E152259
:102F300025D8E66A120090DFE652BBEF17F0B6DF45
:102F40006EDF050E120079DFEF501200D5DFD5ECF1
:102F500017F035EF17F0D0DFC3EC17F035EF17F0AF
:102F6000E66A5DDF050E1200C2DF43EF17F0FD0ECB
:102F7000DBCFE6FF120053DF43EF17F014C0E6FF8C
:062F800015C0E6FF12007F
:0A2F8600F36AF46AFF0EE124E96E1D
:102F9000FF0EE220EA6EED6607D02F0EEF6404D03C
:102FA0003A0EEF6001D0F32A1200F36AF46AFF0EC2
:102FB000E124E96EFF0EE220EA6EED660AD0200EF3
:102FC000EF5C06E0080EEF6404D00E0EEF6001D057
:102FD000F32A1200FF0EE124E96EFF0EE220EA6EF2
:102FE000EDCFF4FFEFCFF3FFF46607D0600EF3648C
:0C2FF00004D07B0EF36001D0F39A1200B5
:022FFC001200C1
:022FFE001200BF
:1030000000000000000000000000000000000000C0
:1030100000000000000000000000000000000000B0
:1030200000000000000000000000000000000000A0
:103030000000000000000000000000000000000090
:103040000000000000000000000000000000000080
:103050000000000000000000000000000000000070
:103060000000000000000000000000000000000060
:103070000000000000000000000000000000000050
:103080000000000000000000000000000000000040
:103090000000000000000000000000000000000030
:1030A0000000000000000000000000000000000020
:1030B0000000000000000000000000000000000010
:1030C0000000000000000000000000000000000000
:1030D00000000000000000000000000000000000F0
:1030E00000000000000000000000000000000000E0
:1030F00000000000000000000000000000000000D0
:1031000000000000000000000000000000000000BF
:1031100000000000000000000000000000000000AF
:10312000000000000000000000000000000000009F
:10313000000000000000000000000000000000008F
:10314000000000000000000000000000000000007F
:10315000000000000000000000000000000000006F
:10316000000000000000000000000000000000005F
:10317000000000000000000000000000000000004F
:10318000D9CFE6FFE1CFD9FFDD52DD52DF50E84471
:10319000DF10E844DF10E844DF10E844DE14DE52BC
:1031A000E552E7CFD9FF1200000C8AEC8FF00D0139
:1031B0003D69FD0EDB50DF6E0D013D5109E079ECFC
:1031C00089F0010EE66E07EC89F010EC96F0F1E163
:1031D000010EDB50C4EC8DF002E2E16AE552E16ED3
:1031E000145094EF87F0B6EC8FF00D013D690D019E
:1031F0003D5110E0FA0EDBCFE6FF44EC88F014EC12
:1032000096F01FEC93F0D3ECA3F0EFEC8FF0DF6EB1
:10321000DF50EDE1DF50E55294EF87F0AEEC96F031
:1032200090EC93F040EF95F0AEEC96F0D8EC8DF08A
:1032300040EF95F0AEEC96F0DEEC8DF040EF95F0BF
:10324000F8EC90F00D013D69010EF36E040EF3CF22
:10325000DBFF0D013D512CE0040EDB5029E0FD0E9B
:10326000DB500BE0FD0EDB507EEC89F0D950030FF4
:103270005AEC93F0E5EC8AF002D0040EDB6ADB50E6
:10328000E8E1020EF36EDB6E79EC89F091EC95F0DB
:103290004AEC96F0E5EC8AF0020EDB0403E1FF0E47
:1032A000DE1604D0020EDB50D4E1DE6ADD6AD1D72F
:1032B000040EDB5003E0F368F46A06D0C1EC88F03A
:1032C00014C0F3FF15C0F4FF050EE15C02E2E16AF1
:1032D000E552E16E94EF87F0D8EC8FF00D013D6977
:1032E000010EFBEC8BF00D013D5119E0020EDB509D
:1032F00016E0FD0EDB5026EC88F0D950010F5AEC99
:1033000093F05AEC92F0EFE1500EDF6E44EC88F04F
:1033100079EC89F04AEC96F0A7EC88F0E4D7020E3D
:10332000DB5002E0FF0E01D0000E0FEC8CF002E249
:10333000E16AE552E16E145094EF87F061EC92F08F
:103340000F0EB4EF95F061EC92F0100EB4EF95F023
:1033500096EC93F014BE1568A6EC8BF00101080EF4
:10336000AF6F010EA76F000E94EF87F096EC93F00D
:1033700014BE1568A6EC8BF00101AEB302D0080EA6
:10338000AF6F94EF87F0B6EC8FF0FE0EDB98DB9A10
:10339000DB9CDB9EDB5002E1440E07D00A0EF6EC0C
:1033A00087F005E2FE0EDB50300FDF6E1AD0FE0E06
:1033B000DB500F0A14E0010A10E0030A0CE0010AD6
:1033C00008E0070A04E0010A0CE1300E09D02A0ED9
:1033D00007D0230E05D0410E03D0420E01D0430E7C
:1033E000DF6EDF50E55294EF87F02FEC90F000C1D4
:1033F000DFFFDF5001E1AAD051EC91F0DB502AEC65
:103400008CF0020EEFCFDBFF01010C510DE0010E3D
:10341000F36EDB5003E003EC89F0FDE1F3500101B2
:10342000B21502E1020EDB8829EC92F07EEC89F005
:10343000DB5029E1020EDB1C100B05E122EC89F0C8
:1034400031C1EFFF30D030EC8EF00B0808E030ECEB
:103450008EF00C0804E0E7EC88F0EF500CE022EC72
:1034600089F0EFCF14F03051D880145404E222ECEC
:1034700089F030C1EFFF22EC89F0EF5014E11FEC2E
:1034800088F0EF8810D0020EDB1C100B05E022EC58
:1034900089F032C1EFFF07D022EC89F0EF5003E151
:1034A0001FEC88F0EF98030EDB5016E029EC92F049
:1034B00013E0020EDB1C100B0FE0B2EC96F00F0BCA
:1034C000146E30EC8EF0145C07E01FEC88F0EF987F
:1034D00022EC89F030C1EFFF29EC92F015E0020EEA
:1034E000DB1C100B11E0B2EC96F0200B0DE130EC80
:1034F0008EF0146EB2EC96F0F00B1410E66E1FEC2A
:1035000088F0E552E750EF6E030EDB501DE029EC2A
:1035100092F01AE11FEC88F0EF8A0BA515D03C0E53
:10352000AEEC8CF0010EDB50300FAEEC8CF03A0EAE
:10353000AEEC8CF0B2EC96F0E66E25DFE552AEEC28
:103540008CF03E0EAEEC8CF0DF0653D7040EE15C3F
:1035500002E2E16AE552E16E94EF87F02DEC92F021
:10356000C8EC8DF004E0010E0801BB1502E1000E6D
:1035700001D0010E94EC91F001018DEC8AF003E092
:103580009EEC8BF0FDE1E1EC96F0DF5001E1BFD065
:1035900051EC91F07AEC88F0EF5015E0010E7AECE6
:1035A00088F034EC8EF07AEC88F0EFCF15F0010E55
:1035B000DB502AEC8CF0EF1C1514145C04E161EC78
:1035C00095F0EF8003D061EC95F0EF90010EDB50A9
:1035D0002AEC8CF0EF1C400B04E0020EDB50B2131F
:1035E00003D0020EDB1CB217E4EC95F0030B020AC9
:1035F00021E0010A12E0020A08E0010A22E1DFEC00
:1036000091F04D0FE96E010E0DD0CBEC8BF0EF5029
:1036100018E161EC95F0EF8214D0DFEC91F0550FDA
:10362000E96E010EEA22EF50E66ECBEC8BF052EC25
:1036300089F007D0CBEC8BF0EF5003E161EC95F013
:10364000EF92050EDB5004E1E4EC95F0020B25E16E
:10365000010EDB5076EC8DF0EF5003E0050EDB50F1
:1036600042E0020EDB500801B31505E0AEC8E6FFEC
:10367000AFC8E6FF08D0020EDB50B41509E0B0C8B1
:10368000E6FFB1C8E6FF010E3EEC89F096EC92F041
:10369000020EDB1C0101A81726D0010EDB5076ECD0
:1036A0008DF0B2C8EFFF48EC8EF0A00E1626000E8B
:1036B000B6EC96F07DEC95F016E1020EDB500801B9
:1036C000B31103E0AE51AF1107E1020EDB50B411AC
:1036D0000AE0B051B11107E0050EDB5004E1020E23
:1036E000DB500101A813E4EC95F0020B09E0020E97
:1036F000DB500101A81504E1020EDB50B01304D029
:10370000020EDB1C0101B0171CEC96F03ED7060E32
:10371000E15C02E2E16AE552E16E94EF87F0CAEC07
:1037200094F003E003EC89F0FDE1F350DF6E01015A
:1037300092519311E81C146EF4EC8FF0DCEC94F0D1
:103740000315A51514141BE0DF50011509E0040E44
:103750000D1506E137EC91F0D10EE926060E0BD0DF
:10376000DF5002150CE0080E0D1509E137EC91F061
:10377000B90EE926060ED2EC8BF007EC8AF0DF508A
:10378000010101152BE0F4EC8FF0DCEC94F0021554
:1037900025E0DF50921506E037EC91F0000EE926A7
:1037A000080E21D0DF50931506E037EC91F0A10E02
:1037B000E926060E18D00BEC90F0BBEC27F0E55292
:1037C000000906E037EC91F0300EE926080E0BD028
:1037D00037EC91F0180EE926080E05D037EC91F081
:1037E000480EE926080ED2EC8BF007EC8AF0E55281
:1037F00094EF87F0B6EC8FF0070EB1EC95F069EC22
:1038000092F004E1155002E1CFDCDF6ADF5002E004
:10381000000E01D0010EE55294EF87F0D8EC8FF046
:1038200013EC8CF007E101010A5104E0010EFBECFE
:103830008BF009D08DEC88F003E003EC89F0FDE11A
:10384000F350A7EC88F000C1DFFFDF501FE051EC20
:1038500091F073EC8CF00FE001010A5110E011ECD3
:1038600089F033EC90F0D5EC96F009E033EC90F071
:10387000EE52EF0404E137EC90F0EF8A05D0A3514B
:1038800003E137EC90F0EF9ADF06DFD713EC8CF012
:1038900004E0020E01010B1551E00D01FA51010186
:1038A00096190EE10D01FB510101971909E1510E25
:1038B000E66EE66A5D0EE66E660EE66E010E2ED0D0
:1038C00008017551010196190EE1080176510101B7
:1038D000971909E1510EE66EE66A510EE66E660E24
:1038E000E66E010E1BD008017251010196190EE11E
:1038F000080173510101971909E1510EE66EE66A5C
:10390000410EE66E660EE66E010E08D0510EE66EB2
:10391000E66A3C0EE66E660EE66E010EE66EAD0ED3
:10392000E66E040EDAEC8BF07AEC8CF0E552E552A0
:1039300089EC90F003E301010A510BE098C1E6FF26
:1039400096C1E6FF97C1E6FFD0EC00F0E552E552E4
:10395000E552030EE15C02E2E16AE552E16E94EFAA
:1039600087F07BEC04F0000904E101EC0FF00009A2
:1039700001E0000C010CD8EC8FF013EC8CF007E1A7
:1039800001010A5104E0010EFBEC8BF009D08DEC33
:1039900088F003E003EC89F0FDE1F350A7EC88F038
:1039A00000C1DFFFDF5042E051EC91F073EC8CF08E
:1039B00031E001010A510CE011EC89F033EC90F098
:1039C000D5EC96F005E033EC90F0EE52EF0422E0F7
:1039D000A95124E001510211146E010EF36EDB5067
:1039E00003E003EC89F0FDE1F350141417E033EC2D
:1039F00090F0080EC0EC87F0EFCF15F011EC89F0D5
:103A000013EC8CF002E0000E01D0010EE552E7103D
:103A1000151404E037EC90F0EF8A06D00101A351B1
:103A200003E137EC90F0EF9ADF06BCD713EC8CF093
:103A300004E0020E01010B151CE04F0EE66EE66A73
:103A40003DEC94F024EC93F029EC93F024EC93F00B
:103A500038EC95F0500EF35C000EF45806E24FEC93
:103A60008EF024EC93F072EC96F07AEC8CF0E55248
:103A7000E55289EC90F005E30101AC5108E10A51EF
:103A800006E03DEC94F035EC03F0E552E552030E10
:103A9000E15C02E2E16AE552E16E94EF87F0AEECA0
:103AA00003F0000904E101EC0FF0000901E0000C53
:103AB000010C8FEC87F0F4EC8FF0C8EC95F09F0BC5
:103AC00007E1F4EC8FF0050E60EC8FF0010B02E0E3
:103AD000010E01D0000E94EF87F043DF000904E0EF
:103AE000DEDF000901E0000C010C32EC92F0060E62
:103AF000DB6A01018DEC8AF003E09EEC8BF0FDE1C6
:103B0000E1EC96F0DF5001E1ABD03CEC95F0800B9E
:103B100006E056EC8EF003E0CEEC94F0EF9E010E42
:103B2000010109150BE0020EDB50B01507E03CEC7B
:103B300095F0400B03E071EC92F0EF8A040E09154A
:103B40000BE0CBEC96F0010B07E03CEC95F0400B62
:103B500003E0CEEC94F0EF9C3CEC95F0620B69E056
:103B6000200A32E0220A19E0420A71E17EEC8CF070
:103B7000EF5073E1020E091504E0CBEC96F0010B57
:103B80006CE13CEC95F09F0B68E171EC92F0EF82F8
:103B9000DF04E66EC4DDE55260D056EC8EF05DE0E9
:103BA000020EDB500101B0150BE011EC89F0B4EC12
:103BB00087F0D5EC96F004E0CEEC94F0EF9243D091
:103BC000CEEC94F0EF9249D0020EDB50B01545E1F7
:103BD000CEEC94F0EF9A020EDB50A8150AE0060E28
:103BE000DBCFE7FF020EDB50E712060EE7CFDBFF6D
:103BF00034D0020EDB5001150CE143EC8FF02DE0C8
:103C0000B4EC87F0DCEC94F0A51527E0080E0D1558
:103C100024E1CEEC94F0EF8C43EC8FF005E07EECE9
:103C20008CF034C1EFFF19D07EEC8CF033C1EFFF84
:103C300014D011EC89F06E1D146E6D1DB0151414A6
:103C4000E552E7140AE0CEEC94F0EF8A06D09D0E20
:103C5000146ECEEC94F01450EF161CEC96F052D784
:103C600009EC8FF0F3CFDBFFCCEC8DF02CE2DF50D2
:103C7000A8EC87F0C8EC95F0620B22E1060EDBCFD2
:103C8000E6FFDF50A8EC87F0D5EC96F019E0010EC6
:103C90000E1504E0020EDB50011506E1020E0E15B2
:103CA0000FE043EC8FF00CE0FBC6E6FFFCC6E6FF3E
:103CB000FDC6E6FF18EC8DF0DF50E9EC95F0EF82E1
:103CC00085EC8CF0CFD7060EDB6A050EDB6A09ECBB
:103CD0008FF0F3CFDBFF0051DF5C1FE2EA6ADF34D5
:103CE0005DEC93F0EE52EF50800B11E1020EDB50D1
:103CF000BB1509E0050EDBCFE7FF020EDB50E71234
:103D0000050EE7CFDBFF020EDB1CBB1703D0020E54
:103D1000DB50BB1385EC8CF0DCD7D950030F8CEC57
:103D200090F0000EEE6E040EED6E09EC8FF0F3CF06
:103D3000DBFFCCEC8DF045E23CEC95F0620B36E11C
:103D40002B1DA511146E38EC8EF0B4EC87F0D5EC79
:103D500096F0031514142AE0010E0D1504E0020E6E
:103D6000DB50011506E1020E0D1520E043EC8FF04B
:103D70001DE0020EDB50011506E05EEC92F0D10E64
:103D8000E926060E08D043EC8FF009E05EEC92F0D5
:103D9000B90EE926060ED2EC8BF018EC8DF0020E6F
:103DA000DB1C06EC8BF0CEEC94F0EF82D950030FC5
:103DB0008CEC90F00B0EEE26000EEF2285EC8CF0D2
:103DC000B6D7B351400A68E0C00A66E0A00A4AE0EC
:103DD000300A2CE0180A22E00C0A19E0060A0BE06F
:103DE000030A01E097D0755117E0040EB36F080E77
:103DF000765D07E309D0755116E0080EB36F765D66
:103E000003E243C140FD86D044C140FD83D00D0193
:103E1000405101E07FD00101100E06D00D0140514C
:103E200001E078D00101200EB36F74D0E6EC8DF084
:103E300071E10101400EB36F080E765D04E29BEC68
:103E400093F0EF8404D00A5102E0040104850101DB
:103E5000756B76C1E6FFE2DCE5523BEC88F01EECC8
:103E60008DF058D0E6EC8DF055E10101800EB36F76
:103E7000080E765D04E29BEC93F0EF8606D00A51C3
:103E800004E0AC5102E1040104870101756B76C1C5
:103E9000E6FF71DDE5523ED020DE000907E10101B9
:103EA000B36BA96B60EC91F035E132D0400E0101AB
:103EB000B35D30E13AC114F0156A166A176A3AC167
:103EC000E6FF15C0E6FFC6EC88F03BEC88F05DEC41
:103ED0008EF064EC8EF001017F51065C186E80510B
:103EE0000758196E815108581A6E825109581B6E75
:103EF0001850145C195015581A5016581B50175862
:103F000009E25CEC04F00101B36B60EC91F002E1BA
:103F10000DEC3BF0070EE15C02E2E16AE552E16E76
:103F200094EF87F08FEC87F0010E76EC96F0050E9B
:103F300042EC94F094EF87F0B6EC8FF0020EB1EC07
:103F400095F069EC92F005E1155003E1D4EC18F01E
:103F5000DF6ADF5002E0000E01D0010EE55294EF5F
:103F600087F08FEC87F0180E76EC96F07AEC96F0EE
:103F700094EF87F0B2EC94F008E047EC94F03DE069
:103F80007EEC91F013EC8FF01BD083EC95F01BE0EE
:103F90002AEC95F032E001016A5102E124EC90F044
:103FA000C1EC88F014503B5D15503C5926E36A5132
:103FB00002E024EC90F03BC1E6FF3CC1E6FF020EBC
:103FC00048EC95F019D02AEC95F00EE04BEC94F00B
:103FD00011E004EC97F011E13CEC95F0DF0B0DE102
:103FE0009EEC93F00AE306D001016A5106E19EECD3
:103FF00093F003E34EEC94F0E552050EE15C02E22F
:10400000E16AE552E16E94EF87F0B2EC94F00BE0D8
:1040100047EC94F024E024EC90F013EC8FF0020EC7
:1040200048EC95F018D02AEC95F017E083EC95F069
:104030000DE0C1EC88F001011450415D155042596A
:1040400002E3E9EC96F024EC90F009D04BEC94F00C
:1040500006E14EEC94F0E55202D07EEC91F0050EB4
:10406000E15C02E2E16AE552E16E94EF87F0B2ECC6
:1040700094F013E02AEC95F00AE124EC90F0030EA2
:104080000101695D32E011EC89F06BDF2AD047EC69
:1040900094F02BE024EC90F01FD02AEC95F023E074
:1040A00004EC97F020E083EC95F00CE0C1EC88F094
:1040B0004151145C4251155802E2E9EC96F024ECAF
:1040C00090F013D04BEC94F010E14EEC94F0E552EC
:1040D000030E0101695D09E113EC8FF0020E48EC5B
:1040E00095F0E55202D07EEC91F0050EE15C02E223
:1040F000E16AE552E16E94EF87F08FEC87F0050EF0
:1041000086EC95F08DEC8AF003E09EEC8BF0FDE1FF
:1041100052EC94F0DF5041E051EC91F001016E1D42
:10412000146E97EC8AF06D1DE552E71414146C15AB
:104130002DE0CFEC87F040EC8EF005E1690519E049
:10414000695124E01AD0CFEC87F0EE52EF0408E07A
:10415000CFEC87F0EE52EF50040814E16B0504E158
:10416000D0EC88F007DF0CD0020E6B5D0BE1690527
:1041700004E1D0EC88F049DF03D0D0EC88F077DFA1
:10418000E55204D0CFEC87F07AEC96F0040E7DEC8B
:1041900088F057EC94F0DF06BDD7050EE15C02E233
:1041A000E16AE552E16E94EF87F08FEC87F09BECCB
:1041B0008AF0FE0E48EC95F0E55294EF87F08FEC14
:1041C00087F0EEEC8DF0DF500EE0A5EC93F006E00A
:1041D000DF500101005DE66EE8DFE552010EC7EC3D
:1041E00089F0DF06F0D7020EE15C02E2E16AE552F7
:1041F000E16E94EF87F08FEC87F0EEEC8DF0DF50FE
:104200000FE0A5EC93F00101011505E0DF50005D22
:10421000E66ECBDFE552010EC7EC89F0DF06EFD783
:10422000020EE15C02E2E16AE552E16E94EF87F092
:10423000B6EC8FF0AAEC8DF003E003EC89F0FDE121
:10424000F350DF6EFE0EDB5005E0DF5001018B13F3
:10425000DF5002D0DF5001018C13E55294EF87F05C
:104260008FEC87F0F4EC8FF0070E42EC94F094EFB3
:1042700087F08FEC87F00BEC90F0E66A18EC8FF08B
:1042800094EF87F08FEC87F00101105105E00BEC03
:1042900090F0010EE66E03D00BEC90F0E66A18EC9D
:1042A0008FF094EF87F08AEC8FF08DEC88F003E0CC
:1042B00003EC89F0FDE1F35026EC88F0DF6A050E8F
:1042C000DF5C07E29FEC92F002E0DF5003D0DF2AD0
:1042D000F6D7FF0EC4EC8DF002E2E16AE552E16E22
:1042E000145094EF87F08FEC87F0060E86EC95F073
:1042F0008DEC8AF003E09EEC8BF0FDE152EC94F043
:10430000DF5001E18ED051EC91F0CFEC87F0070E39
:1043100060EC8FF001E07BD0010117050DE1040E88
:10432000DB50AB1509E0B21D1F15E81C146ED9EC6B
:1043300096F0B015141425D0CFEC87F040EC8EF039
:104340000FE097EC8AF003511515146E0451161501
:104350001410E552E71404E1040EDB50AB1506E03F
:10436000B21D1F15E81C156E8B1D05D0B21D1F1543
:10437000E81C156E8C1D146ED9EC96F0B015141453
:10438000151494EC91F0CFEC87F0EE52EF0422E19B
:10439000040EDB5092150DE0040EDB50B01509E061
:1043A000050EDBCFE7FF040EDB50E716050EE7CF67
:1043B000DBFF040EDB5093150DE097EC8AF0D9EC8F
:1043C00096F00115E552E710B01504E00151931580
:1043D00006EC8BF0D9EC96F09415B01511E097EC43
:1043E0008AF0D9EC96F0E552E710B015E66EC0EC15
:1043F00018F0E552000904E00101941D06EC8BF071
:10440000010EDDEC87F0050EDBCFEFFF04D0010ECF
:10441000DDEC87F0EF6A57EC94F0040EE3EC91F0DA
:104420006FD7060EE15C02E2E16AE552E16E94EFBD
:1044300087F0CAEC94F003E003EC89F0FDE1F3505F
:10444000DF6EDF1C01018B17DF1C8C174CDFE55280
:1044500094EF87F0B9EC96F086EC95F000C1DFFFA1
:10446000DF5009E0CFEC87F0070EDDEC96F057EC5B
:1044700094F0DF06F5D737DF040EE15C02E2E16A73
:10448000E552E16E94EF87F0F8EC90F08DEC88F057
:1044900003E003EC89F0FDE1F350DF6E0BEC90F0EC
:1044A00065EC93F002E3020EDB6A0101AFEC8DF0E4
:1044B000020E66EC95F0141415147EEC89F0020ED1
:1044C00066EC95F0DF1405E1DF50011505E01C51A5
:1044D00003E0010EDB6A03D0DE52020EDD6E020E37
:1044E000D5EC8FF0040EC0EC87F0040EEFCFDBFFAD
:1044F0001B5130E1FEEC8AF0EB50DF142BE1FAECBB
:1045000087F0011527E0FAEC87F0146E075102E0FE
:10451000000E01D0010E1402F3501CE1040EDB501A
:10452000DF1410E1010EF36E020EDB5003E003EC2A
:1045300089F0FDE1F3500101951504E0040EDB1C48
:10454000071508E1040EDB50DF1407E0040EDB5012
:10455000071503E0010EDB9402D0010EDB84DB5073
:10456000146E050EE15C02E2E16AE552E16E145060
:1045700094EF87F0B6EC8FF06BEC8EF0DF6EF1CD40
:10458000E6FFF2CDE6FFF3CDE6FF07EC8AF0DFA20F
:1045900007D0F4CDE6FFF5CDE6FFF6CDE6FF08D077
:1045A000DFA40DD0F7CDE6FFF8CDE6FFF9CDE6FFAD
:1045B0000BEC90F0A3EC19F0BAEC8FF0E552F4ECB0
:1045C0008FF0040E5BEC94F0E55294EF87F08FECE3
:1045D00087F01C0EC0EC89F01D0E76EC96F0C8EC4E
:1045E00095F0100B04E0F4EC8FF0FBEC94F094EFFA
:1045F00087F070EC8EF00601FE6B1200D8EC8FF0A5
:1046000064C7E9FF65C7EAFFEFCFDFFF010E64C7AC
:10461000DBFF020E65C7DBFF010EE76EDBCFE9FFB4
:10462000020EDBCFEAFFE75060EC8FF0E66E29EC7C
:1046300088F052EC89F006E0010EDB2A020EECE372
:10464000DB2AEAD7DF500FEC8CF002E2E16AE55298
:10465000E16E145094EF87F08AEC8FF06BEC8EF0E3
:1046600026EC88F00101B16F3BEC88F006C0BCF18C
:1046700007C0BDF108C0BEF109C0BFF10101A351DF
:1046800007E100C1DFFFDF5003E060EC94F0FBD7EF
:104690004FEC96F05BEC94F0F0CDE6FFEECDE6FF4C
:1046A000EFCDE6FFD0EC00F0BAEC8FF00101A351A2
:1046B00017E1010EDBA207D0F6CDE6FFF4CDE6FF51
:1046C000F5CDE6FF08D0DBA40BD0F9CDE6FFF7CDA2
:1046D000E6FFF8CDE6FF29EC01F0E552E552E552A0
:1046E000020EE15C02E2E16AE552E16E94EF87F0CE
:1046F0008AEC8FF00101B15120E0B16B5CEC04F069
:104700000101A35102E174EC04F000C1DFFFDF50AE
:1047100014E051EC91F00101A35103E137EC90F06A
:10472000EF9A33EC90F0C8EC95F0100B04E033EC0A
:1047300090F0FBEC94F0DF06EAD7020EE15C02E2B7
:10474000E16AE552E16E94EF87F0B6EC8FF001017B
:10475000A35107E100C1DFFFDF5003E060EC94F0FC
:10476000FBD789EC90F010E24FEC96F0C0EC87F0AC
:10477000040EEF6E65C8E6FF63C8E6FF64C8E6FF97
:10478000D0EC00F0E5520DD0370EE66E660EE66E08
:10479000010EE66EAD0EE66E040E2EEC89F07AEC9C
:1047A0008CF0BAEC8FF094EF87F0F8EC90F07BECA3
:1047B00004F0000904E145EC05F0000924E0D950BB
:1047C000040FF8EC8FF091EC95F00FEC01F0FBEC9E
:1047D00096F05CEC04F000C1DFFFDF5014E051EC18
:1047E00091F00101A35103E137EC90F0EF9A33EC23
:1047F00090F0C8EC95F0040B04E033EC90F0FBEC87
:1048000094F0DF06EAD7050EE15C02E2E16AE552C8
:10481000E16E94EF87F0B9EC96F03CEC8EF0F6EC9C
:1048200087F016E21F0EDF6E010E5DC1DBFF020E88
:104830005EC1DBFF030E5FC1DBFFD950010FE66EE7
:10484000000EDA2015EC88F01F0EAFEC89F019D0BD
:1048500013EC8CF016E1010EA36F5DC1E6FF5EC1A3
:10486000E6FFB7EC02F0E552E552F3CF16FDF4CFC8
:1048700017FD5FC11CFD9D900D0111899D80FFEC0E
:104880003AF0040EE15C02E2E16AE552E16E94EF77
:1048900087F08FEC87F013EC8CF00BE10101A35152
:1048A00008E0A36B9D900D0111999D800DEC3BF0EC
:1048B00006D099EC91F003E21E0EC0EC89F094EF63
:1048C00087F08FEC87F07DEC96F08AEC8BF0F3CFDD
:1048D000E6FFF4CFE6FF0FEC97F05DEC8EF016509C
:1048E000F324146E1750F420156E640E56EC93F0FA
:1048F00007E2C4EC87F0000EE66E070EDFEC8BF0EB
:1049000094EF87F08FEC87F03CEC92F0DCEC90F0C9
:104910001426000E1522640E56EC93F009E20BECFF
:1049200090F03CEC92F069EC05F0E552E552E5526E
:1049300094EF87F07DEC96F0320ED880F354000EA1
:10494000F45401E2010C000C8AEC8FF07DEC96F03F
:10495000F350DF6EFE0EDB50DF24010F146E640E89
:10496000145C1DE2010EDFCFDBFFDB5010E0010E17
:10497000DB507CEC8DF0EF50E66E8CEC8CF0E72495
:104980007CEC8DF052EC89F0010EDB06EED7FE0ECA
:10499000DB507CEC8DF000C7EFFF000E01D0010E64
:1049A000C4EC8DF002E2E16AE552E16E145094EF3E
:1049B00087F015EC95F0DB500BE0010EE66EC4DFDE
:1049C000E552000905E1FE0EDBCF00F7000E01D035
:1049D000010E94EF87F08FEC87F077EC8EF0EFCF3D
:1049E00014F0ABEC91F0145C0DE1ABEC91F00AE04B
:1049F000FB0EDB2AFC0E01E3DB2AC0EC8BF0EDE3BF
:104A0000DB2AEBD7ABEC91F002E0000E07D077EC9D
:104A10008EF0EF5002E0010E01D0020E94EF87F00D
:104A200032EC92F00101B15118E03BEC88F0010149
:104A3000BC51065C146EBD510758156EBE51085826
:104A4000166EBF510958176E45C118F0196A1A6AD7
:104A50001B6A27EC8DF001E24BDE34EC95F07EEC26
:104A60008EF08DEC8AF003E09EEC8BF0FDE152ECD1
:104A700094F0DF5001E1F9D151EC91F0F1EC96F0B6
:104A800006E0C8EC8DF003E119EC95F0EF6A1FEC3D
:104A900088F0020EEFCFDBFF97EC8AF001010351A3
:104AA0000411E552E7141DE097EC8AF00451121549
:104AB000146E035111151410E552E71412E1020EA1
:104AC000DBA805D0D0EC88F0E66E18EC8FF0020E73
:104AD000DBAA07D01FEC88F0EF9A65EC94F0020E89
:104AE000DB6A020EDBA853D065EC94F032EC93F055
:104AF000040804E032EC93F0080813E197EC8AF024
:104B0000010104511415146E035113151410E552CC
:104B1000E71407E1D0EC88F0E66E18EC21F0E552DE
:104B20000CD001010FB107D0020E0F1507E030ECD9
:104B30008EF00B0803E037EC93F0E552F1EC96F0C1
:104B400004E00101B15101E0D3DD30EC8EF00B083F
:104B50000FE132EC93F0010B05E0D0EC88F042EC71
:104B600021F005D001010FA503D037EC93F0E552F9
:104B7000020EDB5023080BE100EC8CF005E18A51BA
:104B800003E0010EAE1503E137EC93F0E552020E9F
:104B9000DBAAACD0DBCFE6FFC3EC19F0E552A7EC03
:104BA00088F01FEC88F0EF9AF1EC96F005E0010137
:104BB000B15102E09DDD0CD0D2EC94F0200B08E066
:104BC00019EC95F0EF6A9DEC91F002E0CFEC92F0D9
:104BD000020EDB502A0811E132EC93F0010B07E0E2
:104BE000F1EC96F03FE0C8EC8DF06DE13BD0F1ECDC
:104BF00096F063E00101AE9360D0D2EC94F0080827
:104C000036E111EC89F0E7EC91F081EC96F03BECA9
:104C100091F0E7EC91F0DFDEFBEC96F07EEC89F0B2
:104C2000DB501CE1010EDB50050D8AEC8BF0CA0E47
:104C30001626070EB6EC96F038EC95F0F3CFE6FFAB
:104C4000F4CFE6FF3BEC91F088EC88F064EC8EF05A
:104C500082EC8DF0145CF45015582FE2030EDB50FB
:104C6000020831E167EC90F05BEC94F02CD0020E7E
:104C7000DB50230828E100EC8CF005E18A5103E0C9
:104C8000010EAE1520E137EC93F0E55200EC8CF00C
:104C900004E1020EAE1501E0AE939DEC91F00DE043
:104CA00019EC95F0080EEF6E010EDB50050D41EC8E
:104CB00092F0CA0EE926070E04D067EC90F0E926C0
:104CC000000EEA22EF6AF1EC96F010E011EC89F0A8
:104CD00019DEE5521DEC8FF003E071EC8AF0FDE186
:104CE0000101B01502E0899101D08981D2EC94F0E4
:104CF000100B2CE000EC8CF00BE0010EAE1515E172
:104D0000B15113E10701005110E130EC8DF00DE1DC
:104D1000F4EC96F0AE839DEC91F058E0010EAE15E8
:104D200055E10701005152E14DD019EC95F0200EEC
:104D3000EF6E9DEC91F001E185D0D0EC88F01ADCAB
:104D4000E552E7EC88F038C1EFFF7CD0D2EC94F06C
:104D5000200B4AE0010E0101AE153CE1B1513AE1F0
:104D60000701005137E130EC8DF034E1010EDB50EA
:104D7000AF5D1FE0080EAF5D1CE2AF51A8EC87F0FD
:104D80001FEC97F0020B15E0AF51A8EC87F0020E74
:104D9000C0EC87F0EF92320E176E440E186E000EC4
:104DA000196E010EDBCF1AF01B6A1C6A030E8DEC24
:104DB00089F0F4EC96F00101AE839DEC91F006E0F1
:104DC000CFEC92F0D0EC88F047DCE5522A0EE66E8C
:104DD00099DD37D0E7EC88F0EF5034E19DEC91F0AD
:104DE00029E0CFEC92F026D0F1EC96F01FE000EC39
:104DF0008CF009E1E7EC88F0EF500EE1B1510CE1E5
:104E0000010EAE1509E119EC95F0EF6A010EDB50C9
:104E1000AF5D13E1AE9311D0B35103E1010EAE15B6
:104E200011E039510FE065EC94F00CD0E7EC88F01C
:104E3000EF5008E119EC95F0EF6AD0EC88F019EC2E
:104E400022F0E55200EC8CF008E1010EAE1505E011
:104E500029EC92F002E047C141FDD950050F60EC0A
:104E600088F0040EE3EC91F004D6070EE15C02E258
:104E7000E16AE552E16E94EF87F02FEC90F00101CA
:104E80008DEC8AF003E09EEC8BF0FDE10AEC97F0EC
:104E9000DF5010E06AEC94F008E1030EC4EC90F0EF
:104EA00004E0D5EC92F036C1EFFFDAEC92F0E3ECDF
:104EB00091F0EED7040EE15C02E2E16AE552E16EA8
:104EC00094EF87F02FEC90F001018DEC8AF003E075
:104ED0009EEC8BF0FDE10AEC97F0DF5017E06AECF6
:104EE00094F00FE1030EC4EC90F00BE0BDEC96F0F3
:104EF0000101061DE552E71404E0D5EC92F035C13E
:104F0000EFFFDAEC92F0E3EC91F0E7D7040EE15C0E
:104F100002E2E16AE552E16E94EF87F08FEC87F0F0
:104F2000030E3CEC8EF0DDEC8FF04BEC8BF0DF50A1
:104F30001AE06AEC94F011E10101061D156EDF0420
:104F4000146E010E145203E09EEC8BF0FDE115147B
:104F500004E0D5EC92F035C1EFFFD950010F60ECC1
:104F600088F0DF06E4D7030EE15C02E2E16AE55275
:104F7000E16E94EF87F0F8EC90F0040EDB6A0BEC36
:104F800090F0A6EC92F002E3000E2AD0010E6FEC36
:104F900095F0010102155AEC92F020E0010EF36E3B
:104FA000030EF3CFDBFFDF6A0051DF5C17E2030E75
:104FB00088EC8DF0E7140DE0DF50A8EC87F0090EC7
:104FC00060EC8FF0355D05E1010EF36E040EF3CF5A
:104FD000DBFF030EC7EC89F0DF2AE6D7040EDB50B7
:104FE000146E050EE15C02E2E16AE552E16E1450D6
:104FF00094EF87F06EEC94F0DF5004E1010E0101B4
:10500000011506E091EC8CF0400EEF6E000E01D021
:10501000010EE55294EF87F06EEC94F0DF5004E15E
:10502000010E0101011506E091EC8CF0600EEF6EAF
:10503000000E01D0010EE55294EF87F08AEC8FF05C
:10504000E7EC8BF0DF5004E1010E0101011518E0DF
:1050500091EC8CF0EF50200B10EC96F006E02E0E49
:10506000E66E660EE66E010E05D0240EE66E660E46
:10507000E66E010EB1EC95F02FDABAEC8FF0E55246
:10508000020EE15C02E2E16AE552E16E94EF87F024
:10509000E0EC92F0400EEF6E94EF87F0E0EC92F0CF
:1050A000600EEF6E94EF87F0D8EC8FF089EC90F003
:1050B00043E2FDEC90F0020EEFCFDBFF010EF36E4A
:1050C000020EDB5003E003EC89F0FDE1F35026EC27
:1050D00088F0020E7AEC88F0EF50200BDF6EDF5084
:1050E0000CE0010ED0EC8DF008E0FAEC88F0170E21
:1050F000E66E660EE66E010E1DD0DF5008E0FAEC9B
:1051000088F00A0EE66E660EE66E010E13D0010EF2
:10511000D0EC8DF008E0FAEC88F0FC0EE66E650E3F
:10512000E66E010E07D0FAEC88F0EE0EE66E650E24
:10513000E66E010E3BEC93F0030EE15C02E2E16AE5
:10514000E552E16E94EF87F0E0EC92F0EF50C7EC9F
:105150008CF0156A940F146E020EC8EC87F0A4EC64
:1051600087F094EF87F02DEC92F0010E4DEC89F072
:10517000DF6E020E4DEC89F026EC88F0030E4DEC4C
:1051800089F0A7EC88F0060E4DEC89F094EC91F0D4
:10519000DBCFE6FFD0EC88F0040E4DEC89F0D88030
:1051A000DF54E552D880E754E552D880E7547EECCE
:1051B00089F0050E4DEC89F0E5EC8AF0010187518C
:1051C00008E06BEC90F0D60EE66E650EE66E010E12
:1051D00007D06BEC90F0BF0EE66E650EE66E010E2A
:1051E00010EC95F0146E130EE15E145085EC96F001
:1051F000060EE15C02E2E16AE552E16E94EF87F0AF
:105200002DEC92F00A0E4DEC89F0DE6EDD6A0B0E8D
:10521000E3EC92F0CBEC88F01450EE121550ED1246
:105220000C0E4DEC89F0E66E95EC95F072EC94F076
:105230000D0EE3EC92F0D950020FF6EC8DF00E0E4D
:105240004DEC89F0E66ED950040F8CEC90F072ECC6
:1052500094F00F0EE3EC92F0D950040FF6EC8DF0C1
:1052600077EC94F06AEC93F0B10EE66E650EE66EA4
:10527000010E20EC8BF0ACEC88F0060EE15C02E253
:10528000E16AE552E16E94EF87F08AEC8FF075ECFD
:105290007CF003EC92F0A60EE66E650EE66E010E53
:1052A00009EC92F002E2E16AE552E16E94EF87F0D8
:1052B0008AEC8FF07EEC7CF003EC92F09B0EE66EB5
:1052C000650EE66E010E09EC92F002E2E16AE5522B
:1052D000E16E94EF87F08AEC8FF085EC7CF003ECC4
:1052E00092F0900EE66E650EE66E010E09EC92F0FD
:1052F00002E2E16AE552E16E94EF87F08FEC87F00D
:10530000020E3CEC8EF0C8EC8AF01AE2210EE66E3A
:1053100014EC96F020EC19F066EC8BF0FEEC88F0C3
:10532000FD0EDBCFE6FFE66A830EE66E650EE66EE7
:10533000010EE66EBEEC8FF06DEC8BF085EC96F016
:10534000020EE15C02E2E16AE552E16E94EF87F061
:105350008FEC87F001010051E66EE66A7E0EE66E84
:10536000650EE66E010E19EC88F0ACEC88F094EF57
:1053700087F001EC91F00FE10601FE5103E001011D
:10538000775109E1CEEC89F060C896F161C897F1D8
:1053900062C898F103D00601010EFF6F94EF87F009
:1053A00001EC91F00FE10601FE5103E0010177519C
:1053B00009E1CEEC89F06CC896F16DC897F16EC822
:1053C00098F103D00601020EFF6F94EF87F001EC15
:1053D00091F00FE10601FE5103E00101775109E16F
:1053E000CEEC89F06FC896F170C897F171C898F14A
:1053F00003D00601030EFF6F94EF87F001EC91F0EC
:1054000015E10601FE5103E0010177510FE1CEECF9
:1054100089F0FD0EDB50060B07E0FACD96F1FBCDCF
:1054200097F1FCCD98F10CD0B36B0AD0FD0EDB5098
:10543000060B04E00601040EFF6F02D00601FF69AF
:1054400094EF87F001EC91F00FE10601FE5103E0CB
:105450000101775109E1CEEC89F072C896F173C869
:1054600097F174C898F103D00601050EFF6F94EF11
:1054700087F001EC91F00FE10601FE5103E001011C
:10548000775109E1CEEC89F075C896F176C897F1AD
:1054900077C898F103D00601060EFF6F94EF87F0EE
:1054A0008FEC87F0CEEC89F0FC0EDBCF96F1FD0E91
:1054B000DBCF97F15FC198F194EF87F001EC91F0A9
:1054C00009E14F0E50EC8BF03DEC94F029EC93F099
:1054D00085EC8EF094EF87F001EC91F00AE14F0E2D
:1054E00017EC8CF0000EE66E050EDAEC8BF085EC16
:1054F0008EF094EF87F08FEC87F0FB0EDBCFE9FFA7
:10550000DB2AFC0EDBCFEAFF01E3DB2AEF50E66E7D
:1055100045EC8AF001E3DB2A52EC89F0EEE194EFEE
:1055200087F042EC96F0AEB106D0A0EC88F0EF6ABE
:10553000C36B15EC89F00D01415103E1D5EC23F06B
:1055400069D00101C2516BE0E0EC88F0EF5067E0F8
:1055500030EC8CF003E146C141FD02D047C141FD72
:105560003FEC93F02A0EDF5C55E0230EDF5C52E047
:10557000FEEC22F00101C35113E0C36BDF50390A86
:105580000DE00E0A09E0760A0EE0030A0CE0010ABB
:105590000AE0070A3FE107D02A0E22D0230E20D0CE
:1055A00099EC95F003E0DFCFE6FF1BD0DF50430A14
:1055B00024E0020A1DE0030A0BE0620A09E0290A5E
:1055C00007E04D0A11E04E0A0FE0070A23E10CD074
:1055D000A0EC88F0EF5020E0FB0EDB5005E1200E40
:1055E000E66E61EC89F018D00101010EC26F14D093
:1055F0000101410EC36FC22B0FD0FE0EDB50010123
:10560000C25D08E2FE0EDB28C26FA0EC88F0300E0F
:10561000EF6E02D0FF0E05D00101C20792D7010143
:10562000C251E55294EF87F042EC96F0AEB107D04C
:10563000A0EC88F0EF6A010EAA6F15EC89F00D015D
:10564000415106E1D5EC23F00101AA6BFF0E52D0C7
:105650000101C2513DE0E0EC88F0EF5039E030EC60
:105660008CF003E146C141FD02D047C141FD3FEC52
:1056700093F0FEEC22F001017251DF5C02E12A0E90
:105680001ED07351DF5C02E1230E19D0FB0EDB50FC
:10569000DF5C0DE099EC95F014E1DF50200A0AE0A0
:1056A000290A08E0030A02E0070A0BE10101010EE2
:1056B000C26F0BD0A0EC88F0EF5007E0200EE66E32
:1056C00002D0DFCFE6FF61EC89F00101C207C0D74D
:1056D000FB0EDB500AE11DEC8FF003E071EC8AF069
:1056E000FDE10101B01501E1C26B0101C25101E10F
:1056F000AA6BC251E55294EF87F032EC92F0FE0EA5
:10570000DB50146E156A060ED8801454000E155422
:1057100005E2060EF36EFE0EF3CFDBFF010EE66E22
:10572000F90EE66E030EB1EC95F0FBDEE55274EC7B
:105730008BF03CE1D950050F8CEC90F0F90EEE6E39
:10574000030EED6EDF68D6EC87F0EF5025E0D6EC67
:1057500087F0A2EC8BF016BE1768F5EC94F001E030
:10576000DF6AD6EC87F0A2EC8BF016BE1768F5EC7A
:1057700094F00CE1D6EC87F0EFCF1AF01B6A1ABE5A
:105780001B6875EC92F002E1FF0E11D0050EDB2ACA
:10579000060ED9E3DB2AD7D7F90EE66E030EE66EC6
:1057A000FFEC95F006C0C0F107C0C1F1DF50146EE8
:1057B000070EE15C02E2E16AE552E16E145094EFFB
:1057C00087F0B6EC8FF0E66AE9EC92F0AADEE552DB
:1057D00074EC8BF002E0DF5020D0A0EC88F0EF50AA
:1057E0001BE0A0EC88F0A2EC8BF016BE1768F5EC7D
:1057F00094F00CE1A0EC88F0EFCF1AF01B6A1ABE0F
:105800001B6875EC92F002E1FF0E07D0FC0EDB2A5C
:10581000FD0EE3E3DB2AE1D7000EE55294EF87F0BB
:1058200042EC96F0AEB106D0A0EC88F0EF6AC46B03
:1058300015EC89F00D01415103E1D5EC23F072D054
:105840000101C25101E17BD0E0EC88F0EF5001E1B1
:1058500076D030EC8CF003E146C141FD02D047C167
:1058600041FD3FEC93F099EC95F033E00101C45118
:1058700005E1300EDF5C010FC46F56D0E80E176EE5
:10588000760E186E010E196EC4051A6E1B6A1C6A1C
:105890001AAE02D01B681C68050E8DEC89F0300E24
:1058A000DF5C1D6E1E6A1F6A14501D24F36E1550B6
:1058B0001E20F46E16501F20F86EF4CFF7FFF3CFC2
:1058C000F6FF0800F550E66E61EC89F00101C46B4B
:1058D0002BD0440EDF5C06E00D0EDF5C03E00A0E09
:1058E000DF5C04E10101010EC26F1ED02A0EDF5CF5
:1058F00019E0430EDF5C09E1FE0EDB280101C26FF7
:10590000A0EC88F0300EEF6E0FD00101C45108E119
:10591000200EDF5C03E0090EDF5C02E1C22B04D045
:10592000FEEC22F0FF0E0DD0FEEC22F00101C4517E
:1059300004E0440EDF5C01E083D7C20781D7010198
:10594000C251E55294EF87F042EC96F0AEB105D02B
:10595000A0EC88F0EF6A15EC89F00D01415103E1EC
:10596000D5EC23F020D00101C25128E0E0EC88F012
:10597000EF5024E030EC8CF003E146C141FD02D051
:1059800047C141FD3FEC93F00D0EDF5C03E00A0ED2
:10599000DF5C04E10101010EC26F0BD0210EDF5C60
:1059A00004E1FEEC22F0FF0E0BD0DFCFE6FF61EC4E
:1059B00089F0FEEC22F00101C207D5D70101C251E6
:1059C000E55294EF87F02FEC90F0C70EE66E010ED3
:1059D000E66E080EE66E7BEC94F040E1D950010FC4
:1059E0008CEC90F0C70EEE6E010EED6E0101C66BF1
:1059F00029EC88F0EF5032E029EC88F0A2EC8BF033
:105A000016BE1768F5EC94F023E0090E186E29EC29
:105A100088F0EF50D00F7EEC89F0DB50D88018541E
:105A200017E2FE0EDB5009E0030EDB50ACEC93F006
:105A30000DE09EEC8BF0FDE109D0010EF36E030E3C
:105A4000DB5003E003EC89F0FDE1F3500101C613E4
:105A5000010EDB2A020ECCE3DB2ACAD7DF5046EC6C
:105A60008CF002E2E16AE552E16E145094EF87F0A7
:105A7000AEEC96F0FD0F7FEC94F0FF0ED880EE5464
:105A8000350EED5438E38CEC8EF0E40E145C010E10
:105A900015580BE3FD0EDBCF16F0FE0EDBCF17F033
:105AA000700E165C010E175826E3FD0EDBCF18F0C2
:105AB000FE0EDBCF19F0010E185C000E195808E33A
:105AC000CCEC8AF0040ED880EE54000EED5413E2B4
:105AD000CCEC8AF0A00EEE1802E1020EED180BE0FD
:105AE000CCEC8AF09F0EEE1808E1020EED1805E1ED
:105AF00001018E5102E1000E01D0010E94EF87F0FA
:105B0000E4EC90F00CE0ACEC92F002E6D1EC91F019
:105B100006E328EC8BF002E6B3EC93F002E2010E10
:105B200004D06FEC93F0B9EC93F0146E080EE15CC6
:105B300002E2E16AE552E16E145094EF87F0E4EC82
:105B400090F010E0ACEC92F002E6D1EC91F00AE3B8
:105B500028EC8BF006E6D880FF0E0754FF0E3CECD5
:105B60008CF002E2010E04D039EC8DF0B9EC93F028
:105B7000146E080EE15C02E2E16AE552E16E145037
:105B800094EF87F08FEC87F0100EE12662EC8AF03C
:105B9000C4EC87F020EC8AF0D9500A0F79EC8BF036
:105BA00074E00A0EDBCFE9FF0B0EDBCFEAFFEF500C
:105BB0006CE052EC8CF0B5EC89F023EC91F002E64D
:105BC000D1EC91F062E3B2EC8BF009E6D880000EE4
:105BD0000754000E0854010E0954000E0A5455E3F0
:105BE00023EC91F005E6200EEE5CA20E13EC8AF099
:105BF0000AE2B2EC8BF006E6D880FF0E0754350EB1
:105C00003CEC8CF042E317EC91F020EC8AF0040EAF
:105C1000DB6A050EDB6AD9500A0F79EC8BF04AE09B
:105C2000D0EC8AF0D890155004E6100E145C000EEB
:105C3000155840E252EC8CF00C0E06C0DBFF0D0E46
:105C400007C0DBFF0E0E08C0DBFF0F0E09C0DBFF35
:105C5000D9500C0F8CEC90F089EC96F002E6D1EC68
:105C600091F013E30C0EDBCF07F00D0EDBCF08F045
:105C70000E0EDBCF09F00F0EDBCF0AF00A34000E58
:105C80000A1802E6B3EC93F002E2010E24D1E1EC33
:105C900087F0D00EE926010EEA220C0EDBCFEFFFD3
:105CA000040EDB2A050E01E3DB2A17EC91F020EC51
:105CB0008AF0B1D7080EDB6A090EDB6A8EEC8DF034
:105CC000040EDBCF1CF0050EDBCF1DF01E6A1F6A31
:105CD0001DAE02D01E681F682BEC8AF0CBEC88F05A
:105CE000030EEBCFF3FF1750F318E8AE02D0F334F6
:105CF00008D0EE50145CEE501558EE501658EE5089
:105D0000175808E28EEC8DF0CBEC88F038EC8AF076
:105D1000D7EC8AF023EC91F005E6EB0EEE5C010E79
:105D200013EC8AF001E392D0D0EC8AF0166A176A7D
:105D300015AE02D01668176846EC96F01426EE50A1
:105D40001522EE501622EE5017221734000E1718A7
:105D500004E6D880E40EFCEC8DF001E377D0040E6D
:105D6000DBCF08F0050EDBCF09F0060E08C0DBFF25
:105D7000070E09C0DBFF23EC91F005E6E40EEE5CB4
:105D8000010E13EC8AF024E2E40E7FEC92F0D7ECE3
:105D90008AF0060EDBCF16F0070EDBCF17F0040EED
:105DA000DB50165C146E050EDB501758156E070E8F
:105DB000145E000E155A060E14C0DBFF070E15C048
:105DC000DBFF10EC92F00001800E151443E03ED092
:105DD000040EDBCF18F0050EDBCF19F01A6A1B6A30
:105DE00019AE02D01A681B68EB0E206E010E216EF0
:105DF000226A236A46EC96F0205C1C6EEE50215815
:105E00001D6EEE5022581E6EEE5023581F6E2BEC66
:105E10008AF0D7EC8AF0EB0E7FEC92F0080E14C0FB
:105E2000DBFF090E15C0DBFFD0EC8AF00001800E0D
:105E3000151404E0040EDB6A050EDB6AEB0EDE6E61
:105E4000010EDE6EDE6ADD6ADD52DD52060EDB6AB1
:105E5000070EDB6AD950040F79EC8BF00FE0080EC7
:105E6000DBCF14F0090EDBCF15F0D00E1426010E97
:105E7000C8EC87F077EC94F073EC93F0D0EC8AF0F8
:105E8000070E1426000E1522166A176A15AE02D0E8
:105E9000166817681450DE261550DE221650DE22D2
:105EA0001750DD22DD52DD52D950060F79EC8BF010
:105EB00011E0D0EC8AF0D00E1426010E1522070E48
:105EC00004EC96F0060EDBCFE6FF070EDBCFE6FF15
:105ED00073EC93F0000E146E100EE15C02E2E16AC6
:105EE000E552E16E145094EF87F0D8EC8FF06AEC35
:105EF00091F002E1010E10D06FEC93F086EC91F07E
:105F000011EC89F0E66AFEEC88F06A0EE66E650E2A
:105F1000E66E010EC0EC93F00FEC8CF002E2E16A49
:105F2000E552E16E145094EF87F02FEC90F06AEC9C
:105F300091F002E1010E0DD039EC8DF086EC91F07C
:105F40006AEC93F0610EE66E650EE66E010EC0EC33
:105F500093F046EC8CF002E2E16AE552E16E1450F7
:105F600094EF87F046EC92F0D3EC95F0C1EC88F01A
:105F7000166AD8901650000A06E6200E145CA20E8F
:105F80001558000E165808E2CBEC88F0FF0ED880AA
:105F9000EE54350EED540BE317EC91F0FEEC87F068
:105FA000C5EC93F0D950020F79EC8BF002E1010EB1
:105FB000DBD095EC95F0100ED880EE54000EED5429
:105FC00005E2100EFBEC8BF0030EDB6AFEEC88F0B2
:105FD0005C0EE66E650EE66E010EC1EC96F031ECDD
:105FE000BAF040EC91F0C1EC88F0166A176A1C6AAE
:105FF0001D6A010E1E6E1F6A020EDBCF20F0030E1B
:10600000DBCF21F0226A236A20501C5C186E2150DD
:106010001D58196E22501E581A6E23501F581B6EA1
:10602000E8501718E8AE02D0173402D027EC8DF0F4
:106030000CE28EEC8DF0DECF1CF0DDCF1DF01E6A81
:106040001F6A2BEC8AF0BDEC90F0E00EE66E010EBC
:10605000E66E11EC89F086EC91F0C1EC88F0EA0E66
:10606000D8801454010E15544BE3020EDBCF18F008
:10607000030EDBCF19F0DE501824166EDD50192008
:10608000176E1606000E175AE40ED8801654010E2D
:10609000175436E2C1EC88F0E40ED8801454010E97
:1060A000155411E3C1EC88F0E40ED8801456010EAB
:1060B0001556080E14C0DBFFDB50070FE76E090E04
:1060C000E7CFDBFF0ED0080EDB6AC1EC88F0E40EF0
:1060D000145E010E155A070EB4EC8DF0090E14C0B3
:1060E000DBFF090EDB5093EC8EF00AE2100E93EC0E
:1060F0008EF006E200EC8EF0EF6A080EDB2AF1D794
:10610000080EDB6ADBCF14F0020EDBCF15F0030EB6
:10611000DBCF16F01550145C000E165424E200EC90
:106120008EF0EF50E66EE66A580EE66E650EE66E8D
:10613000010E10EC95F040EC91F013EC97F0500E3E
:10614000B4EC8DF01406155A4BEC92F0BEEC8FF0C7
:10615000C4EC87F0ADECADF0166E060EE15E1650A5
:10616000080EDB2ACFD7000E146E0A0EE15C02E2A5
:10617000E16AE552E16E145094EF87F08FEC87F0FE
:1061800001010051C8EC8AF00AE2BEEC8FF00C0E5F
:10619000E66E14EC96F097EC8EF085EC96F094EFAA
:1061A00087F0B6EC8FF0DF6A080EDF5C0BE2DF50A1
:1061B0009AEC88F0EF50F36EFE0EDB50F35C02E0D9
:1061C000DF2AF2D7DF50E55294EF87F08FEC87F0AB
:1061D000140EE126FDEC90F0EFCFDFFFDFCFE6FFFE
:1061E000CBEC95F094EC91F0DB5092EC8AF004E16A
:1061F000155002E1050EDB6A010EDF5205E0DFCF2C
:10620000F3FF38EC8BF0FDE1A7EC88F0DBCFE6FF85
:10621000050E66EC95F0E552E71426EC88F0020EC8
:10622000DB500101021506E0560EE66E650EE66EC5
:10623000010E19D0020EDB50041506E0540EE66E76
:10624000650EE66E010E0FD0020EDB50031506E060
:10625000510EE66E650EE66E010E05D04F0EE66E2F
:10626000650EE66E010EE66ED950110FE66E000E59
:10627000DA202EEC89F0FD0EDB5010E0DF507AECD6
:106280008FF056EC96F0450EE66E650EE66E010E4A
:106290003EEC8DF00B0EE15E16500CD056EC96F0F5
:1062A0003E0EE66E650EE66E010EE66EBEEC8FF0FB
:1062B0006DEC8BF0010EDB5027E0020EDB1C146E40
:1062C000050E66EC95F0141422EC8FF0080EDB6AD4
:1062D000070EDB6A080EF36E070ED1EC90F00EE2AB
:1062E000060EDBA005D0070EDB50300FC4EC8BF0A0
:1062F000070EDB2A060E7DEC88F0ECD7080EDB508B
:1063000003E0200EC4EC8BF0020EDB5001016D1592
:1063100002E1000E01D0010E7EEC89F0020EDB508E
:106320006E1502E1000E01D0010E020D42EC8DF05F
:10633000020EDB50701502E1000E01D0010E040DBB
:1063400042EC8DF0DB50030B13E0030EDBA207D011
:10635000370EE66E650EE66E010E92EC88F0030EC7
:10636000DBA02ED0320EE66E650EE66E010E26D054
:10637000010EDB501EE02E0EE66E650EE66E010E7F
:1063800092EC88F0FD0EDB501BE0080EDB5018E0AD
:106390002A0EE66E650EE66E010E92EC88F0D9507C
:1063A000080FF8EC8FF0970EE66E050EDFEC8BF021
:1063B00007D0250EE66E650EE66E010E92EC88F0B3
:1063C000030EDBA407D01E0EE66E650EE66E010E10
:1063D00092EC88F01C0EE66E650EE66E010E92ECF5
:1063E00088F0BEEC8FF033EC89F0010E146E140EC1
:1063F000E15C02E2E16AE552E16E145094EF87F04D
:106400008EEC96F03AE292EC96F005E0DFCFF3FFE7
:1064100038EC8BF0FDE110EC96F001016D15EEEC1F
:1064200090F00BE0020EDB5008E0FAEC88F0120E60
:10643000E66E650EE66E010E1DD0030EDB5008E021
:10644000FAEC88F0070EE66E650EE66E010E12D0CD
:10645000020EDB5008E0FAEC88F0FE0EE66E640EE9
:10646000E66E010E07D0FAEC88F0F50EE66E640ECB
:10647000E66E010E3BEC93F001D0000E46EC8CF082
:1064800002E2E16AE552E16E145094EF87F08EEC7F
:1064900096F03AE292EC96F005E0DFCFF3FF38ECAD
:1064A0008BF0FDE110EC96F001016E15EEEC90F032
:1064B0000BE0020EDB5008E0FAEC88F0E90EE66E25
:1064C000640EE66E010E1DD0030EDB5008E0FAEC00
:1064D00088F0DC0EE66E640EE66E010E12D0020E3F
:1064E000DB5008E0FAEC88F0D10EE66E640EE66E42
:1064F000010E07D0FAEC88F0C60EE66E640EE66E6A
:10650000010E3BEC93F001D0000E46EC8CF002E261
:10651000E16AE552E16E145094EF87F08EEC96F04C
:106520003AE292EC96F005E0DFCFF3FF38EC8BF027
:10653000FDE110EC96F001017015EEEC90F00BE02F
:10654000020EDB5008E0FAEC88F0BD0EE66E640E39
:10655000E66E010E1DD0030EDB5008E0FAEC88F069
:10656000B30EE66E640EE66E010E12D0020EDB5024
:1065700008E0FAEC88F0A80EE66E640EE66E010EF6
:1065800007D0FAEC88F09D0EE66E640EE66E010E02
:106590003BEC93F001D0000E46EC8CF002E2E16A95
:1065A000E552E16E145094EF87F008EC96F013E298
:1065B0008DEC88F003E003EC89F0FDE17DEC8AF0DE
:1065C0009CEC95F0DF5001016D1514EC90F018EC87
:1065D0008BF0A4EC87F0020EE15C02E2E16AE55286
:1065E000E16E94EF87F008EC96F015E28DEC88F000
:1065F00003E003EC89F0FDE17DEC8AF0B9EC8DF06D
:10660000A0EC87F0DF5001016E1514EC90F0B9ECAE
:106610008DF0A4EC87F0020EE15C02E2E16AE55243
:10662000E16E94EF87F008EC96F013E28DEC88F0C1
:1066300003E003EC89F0FDE17DEC8AF04A0E71EC99
:106640008FF0DF5001016F1514EC90F04A0E64ECEE
:106650008FF0020EE15C02E2E16AE552E16E94EF36
:1066600087F008EC96F015E28DEC88F003E003EC7F
:1066700089F0FDE17DEC8AF0BCEC8DF0A0EC87F0B8
:10668000DF500101701514EC90F0BCEC8DF0A4EC1F
:1066900087F0020EE15C02E2E16AE552E16E94EFFE
:1066A00087F001017051E66EE66A6E51E66EE66AA9
:1066B0006D51E66EE66A920EE66E640EE66E010EAF
:1066C00020EC8BF033EF89F04CEC95F0080E7EEC6B
:1066D0008BF010E20101011D146E090EC4EC90F064
:1066E000141402E090EC90F0080EDB2A090EC7ECBF
:1066F00089F0ECD70A0EE15C02E2E16AE552E16E54
:1067000094EF87F04CEC95F0080E7EEC8BF00EE2E7
:10671000090EC4EC90F00101011502E090EC90F03C
:10672000080EDB2A090EC7EC89F0EED70A0EE15CF1
:1067300002E2E16AE552E16E94EF87F0A0EC95F099
:106740001DE2080EC8EC8AF019E2FDEC90F0EF5063
:10675000156E010E155204E0E846FE0B1506FCE12D
:10676000146EFD0EDB509AEC88F0EF5084EC8BF049
:106770001450EF12E8EC87F0000E01D0030E94EFF6
:1067800087F0B6EC8FF0DF6A080EDF5C14E2FE0ED5
:10679000DB5005E0DF5084EC8BF0EF6A08D0CFECE3
:1067A00095F0146EDF5084EC8BF01450EF16E8EC8B
:1067B00087F0DF2AE9D7E55294EF87F002EC8BF0FF
:1067C000EB5001010715166E010EEB50156E071DFB
:1067D000151416100FEC90F0FEEC8AF0C0EC87F068
:1067E0000151EF16CFEC95F054EC8BF0E8EF87F009
:1067F000E5DF8FEC8BF003E071EC8AF0FDE1E81C43
:1068000001019517CFEC95F005EC8CF021B15CDF20
:10681000010121A302D062EC27F0010121A902D0DD
:106820000AEC8CF0E8EF87F0F8EC90F0DF6A89EC86
:1068300090F03AE2F4EC8FF0EE52EF0404E1FE0E39
:10684000DB50DF6E31D00BEC90F0A6EC92F002E35F
:10685000010EDB6A010E17EC97F05AEC92F024E07F
:10686000030EDB6A040EDB6A58EC8CF016E211ECC6
:1068700089F0CCEC93F0EF50166E010E165204E046
:10688000E846FE0B1606FCE1E552E71406E1030EAE
:10689000DB2A040EE9E3DB2AE7D758EC8CF004E2AC
:1068A000CCEC93F0EFCFDFFFDF50146E050EE15C10
:1068B00002E2E16AE552E16E145094EF87F02FECAA
:1068C00090F0FD0EDB501CE00BEC90F0FCEC89F03E
:1068D00004E3020EDB6A030EDB6A19EC8AF037E18F
:1068E000B551151834E1CFEC87F0F4EC89F0EF5096
:1068F000011510EC96F09313010EDB1C921729D0B2
:10690000E7EC8BF0DF5004E1010E010101151FE0FF
:10691000DFCFE6FFFCEC89F004E3020EDB6A030E36
:10692000DB6A19EC8AF013E1B551151810E1010E7C
:10693000DF5205E0DFCFF3FF38EC8BF0FDE110EC28
:1069400096F001019213010EDB1C931702D0010E89
:106950000ED08FEC8BF003E071EC8AF0FDE10101C9
:106960009513A3EC90F0C8EC87F0EEEC92F046ECB7
:106970008CF002E2E16AE552E16E145094EF87F088
:10698000D8EC8FF0E7EC8BF0010EDF5205E0DFCFA3
:10699000F3FF38EC8BF0FDE126EC88F0DFCFE6FF6B
:1069A00065EC93F002E3020EDB6A020EDB508CEC26
:1069B00095F015220101B451141802E1B5511518D2
:1069C00002E0010E13D0010EDB50931507E0020E1A
:1069D0006FEC95F09315E81C931703D0010EDB1CA8
:1069E0009217020E8FEC8FF0EEEC92F00FEC8CF021
:1069F00002E2E16AE552E16E145094EF87F0B6ECE2
:106A00008FF0010122B17EDE010122A302D062ECEF
:106A100027F0010122A902D00AEC8CF0D3EC93F00C
:106A2000011D10EC8EF0011515100FEC90F0011DFA
:106A3000156EFEEC8AF0EB5015140111EFEC8AF0A4
:106A400022EC97F074EC91F0E8EC87F0E55294EFCB
:106A500087F08AEC8FF001018D6B8E6B8F6B010ECE
:106A6000776F996B9E6BDF6ACCEC8DF003E29BEC49
:106A70008EF0FAD7080EE66E49EC24F0E5520101DB
:106A800023B140DE010123A302D062EC27F0010113
:106A900023A527D0CFEC95F005EC8CF0071D10EC6A
:106AA0008EF0071515100FEC90F0071D166EFEEC1A
:106AB0008AF0EB501614156E01515CEC96F0A51798
:106AC000A4EC95F09CEC95F0010EDB1C146EFAEC36
:106AD00087F094EC8DF023A902D00AEC8CF0E8EC5E
:106AE00087F00101AB6B020EE15C02E2E16AE55264
:106AF000E16E94EF87F015EC95F0DBA602D05EDE38
:106B000018D002EC8BF0EB50166E0101015104110C
:106B100003111614156E010EEB50021515100FEC33
:106B200090F0021D146EFEEC8AF0C0EC87F0145059
:106B3000EF16CFEC95F0010154EC8BF0FE0EDBB0BC
:106B4000C3DDFE0EDBA202D062EC27F0FE0EDBA45A
:106B500002D0D3EC93F0FE0EDBA802D00AEC8CF04E
:106B6000E8EC87F094EF87F0A2EC8EF0176E01014D
:106B7000071D166EEF5016141714156E020EEB500B
:106B8000071515100FEC90F0071D0115156EFEECA2
:106B90008AF0EB505CEC96F005EC8CF08FEC8BF00F
:106BA00003E071EC8AF0FDE10101951325B18CDD64
:106BB000010125A302D062EC27F0010125A902D032
:106BC0000AEC8CF00101996B9E6BE8EF87F08FEC7B
:106BD0008BF003E071EC8AF0FDE1E81C01019517F0
:106BE000E8EF87F08FEC8BF003E071EC8AF0FDE1C9
:106BF00001019513E8EF87F0D6EC91F005E0DFCFC7
:106C0000F3FF38EC8BF0FDE144EC93F009E0E2ECAB
:106C10008FF0010EDB5001016D1396EC96F001D060
:106C2000010E46EC8CF002E2E16AE552E16E14508E
:106C300094EF87F0D6EC91F005E0DFCFF3FF38EC6E
:106C40008BF0FDE144EC93F00BE0E2EC8FF0010EF1
:106C5000DB1C01016D17CFEC87F088EC92F001D0BE
:106C6000010E46EC8CF002E2E16AE552E16E14504E
:106C700094EF87F08FEC87F0050E56EC89F005E075
:106C8000DFCFF3FF38EC8BF0FDE126EC88F0040E4B
:106C9000DB6A080EF36E040ED1EC90F00AE2040EEB
:106CA000DB509AEC88F0EF50DF5C03E0040EDB2A47
:106CB000F0D7010ED0EC8DF046E0E2EC8FF0010E43
:106CC000DB5001016E1508E023EC95F07E0EE66EB8
:106CD000640EE66E010E31D0010EDB506D1509E138
:106CE000D0EC88F0CFEC87F060EC8FF0E552E71045
:106CF00008E123EC95F0710EE66E640EE66E010E6F
:106D00001CD0D0EC88F0CFEC87F01FEC97F002E0BD
:106D1000000E01D0010EE552E71408E023EC95F0D7
:106D2000630EE66E640EE66E010E07D023EC95F05E
:106D3000570EE66E640EE66E010E3EEC8DF0090E07
:106D4000E15E165009D0500EE66E640EE66E010E3E
:106D500010EC95F0EFEC8FF0BEEC8FF033EC89F097
:106D6000050EE15C02E2E16AE552E16E94EF87F024
:106D7000D6EC91F005E0DFCFF3FF38EC8BF0FDE1CE
:106D800044EC93F00DE0E2EC8FF0010EDB1C146E8E
:106D9000CFEC87F050EC92F0EF1696EC96F001D025
:106DA000010E46EC8CF002E2E16AE552E16E14500D
:106DB00094EF87F0D6EC91F005E0DFCFF3FF38ECED
:106DC0008BF0FDE144EC93F00FE0E2EC8FF0CFECC0
:106DD00087F0C0EC87F0010EDB50EF12CFEC87F0AC
:106DE000020E88EC92F001D0010E46EC8CF002E22B
:106DF000E16AE552E16E145094EF87F0CAEC94F02A
:106E000003E003EC89F0FDE13CEC90F00EE099EC3E
:106E100091F00BE2FAEC87F0DF14146E48EC93F07B
:106E2000EF12E8EC87F0000E01D0010EE55294EF6E
:106E300087F0CAEC94F003E003EC89F0FDE13CEC50
:106E400090F00FE099EC91F00CE2FAEC87F0DF148F
:106E5000E81C146E48EC93F0EF16E8EC87F0000E97
:106E600001D0010EE55294EF87F0B6EC8FF0DF6AA7
:106E7000050EDF5C14E2FEEC94F0030EC0EC87F02C
:106E800001010151EF1625EC97F00115146EFEEC8F
:106E900094F048EC93F0EF1253EC8FF0E9D7E55201
:106EA00094EF87F0CAEC94F003E003EC89F0FDE185
:106EB0003CEC90F012E099EC91F00FE2DF50AB1354
:106EC000BCC8E6FFBDC8E6FF420EE66E0D0EE66EDC
:106ED00044EC89F0E552000E01D0010EE55294EF2A
:106EE00087F0B6EC8FF064EC33F082EC33F062ECB8
:106EF00027F0A2EC8EF00FEC90F0FAEC87F0010195
:106F00000115E66E1FEC91F005EC8CF074EC91F03D
:106F1000EF50E81C54EC8BF0AB6B8FEC8BF003E084
:106F200071EC8AF0FDE101012615146E8FEC8BF0F7
:106F300003E071EC8AF0FDE1E81C010195151410E5
:106F4000956F0AEC8CF0E8EC87F083DDE55294EF66
:106F500087F0B6EC8FF09FEC8AF0B0EC87F08EEC07
:106F600027F00101926B936B89EC83F079EC89F047
:106F70009CEC95F0DF1C01010115E81C6D17A56B59
:106F800023EC96F0010127510315946F26C195F16A
:106F9000010EE66EC1EC33F0E552DF6A050EDF5CF0
:106FA00006E294EC8FF0E8EC87F0DF2AF7D70101D6
:106FB000010E776F996B9E6BAB6BDF6ACCEC8DF03B
:106FC00003E29BEC8EF0FAD7080EE66E49EC24F053
:106FD000E5523FDDE55294EF87F0A0EC95F00FE22B
:106FE000FD0EDB501F0B146E37EC92F0EF50A00B30
:106FF0001410E66E37EC92F052EC89F02CD013ECC2
:107000008CF029E1FD0EDBA002D08E8801D08E9895
:10701000DBA202D08E8A01D08E9ADBA402D08E8CA5
:1070200001D08E9CDBA602D08E8E01D08E9EDBA876
:1070300002D08F8001D08F90DBAA02D08D8001D04A
:107040008D90DBAC02D08D8201D08D92DBAE02D070
:10705000908601D0909694EF87F0B6EC8FF089EC93
:1070600090F030E2050EC8EC8AF02CE2AAEC8DF02C
:1070700003E003EC89F0FDE1F350DF6EFC0EDB5022
:107080000CE0AAEC8DF003E003EC89F0FDE1F35095
:10709000E76EFC0EE7CFDBFF02D0FC0EDB6ADBCF36
:1070A000E6FFFE0EDDEC87F0EECF14F0EFCF15F02B
:1070B000DF1C1514E552E710E66E37EC92F052EC47
:1070C00089F077D013EC8CF001E073D0080EC8EC97
:1070D0008AF06FE2FC0EDB5006E0010EF36EFC0E50
:1070E000F3CFDBFF02D0FC0EDB6AAAEC8DF003E0ED
:1070F00003EC89F0FDE1F35001012A150AE0FC0ED2
:10710000DB5002E0000E01D0010EE76EFC0EE7CF6F
:10711000DBFFFD0EDB50070A46E0010A3CE0030AF4
:1071200032E0010A28E0070A1EE0010A14E0030A1F
:107130000AE0010A3EE1FC0EDB50E8B08E88E8B0C0
:1071400038D08E9836D0FC0EDB50E8B08E8AE8B08E
:1071500030D08E9A2ED0FC0EDB50E8B08E8CE8B08A
:1071600028D08E9C26D0FC0EDB50E8B08E8EE8B086
:1071700020D08E9E1ED0FC0EDB50E8B08F80E8B091
:1071800018D08F9016D0FC0EDB50E8B08D80E8B0A0
:1071900010D08D900ED0FC0EDB50E8B08D82E8B0A0
:1071A00008D08D9206D0FC0EDB50E8B09086E8A0A7
:1071B0009096E55294EF87F08FEC87F099EC91F080
:1071C00010E203010D0EC66FFD0EDBCFC7F3FC0E00
:1071D000DBCFC8F38CEC93F0DFEC94F00D0EAFEC4A
:1071E00089F094EF87F015EC95F062EC96F0EEECF8
:1071F00095F0FC0EDBCFEFFF010EC7EC8CF0040D19
:10720000D7EC93F0FD0EDB50B4EC92F0C7EC8CF0B1
:10721000040DA6EC8EF0FD0EDB503CEC8BF094EFF1
:1072200087F08FEC87F0E9EC92F0DDDFBAEC8FF0BD
:1072300013EC8CF005E127EC91F01FEC6BF004D01F
:10724000E9EC92F0B9DFE552E552E55294EF87F0B0
:107250008FEC87F013EC8CF007E10EEC91F014EC5E
:1072600096F01FEC6BF006D00EEC91F0C4EC87F0BA
:10727000A3DFE552E552E55294EF87F08AEC8FF0F8
:107280000101AEA1F56BF55139E1F20EE66E010E8A
:10729000DFEC94F07BEC94F029E1F20EE66E010E47
:1072A000E66E88EC88F0F4CF15F0020EF3181EE1BC
:1072B00015501CE10101010EF56F300EF25DF06F0B
:1072C000300EF35DF16F000EF05D43E3F0510808FE
:1072D00040E3000EF15D3DE3F15103083AE3CBECEE
:1072E00090F0EFCFF6F146C141FD92D0C4EC96F09C
:1072F00001E08ED0155001E08BD02AD00D01415114
:1073000004E12AEC96F019E01DD0010178517911C1
:1073100001E17ED0E0EC88F0B8EC8CF001E178D0AF
:1073200046C141FD010EDB502A0804E0010EDB508E
:10733000230812E12AEC96F005E1CBEC90F0ADECDD
:107340008EF004D0CBEC90F0CBEC8CF0E552E55213
:107350000101786B796B5CD0010EDB50440A31E09F
:107360007D0A28E00A0A1FE00B0A19E00D0A12E064
:10737000070A0CE0050A06E0060A38E1EAEC8FF09D
:10738000EF2A34D0EAEC8FF0EF0630D0EAEC8FF041
:10739000EF682CD0EAEC8FF07F0EEF6E27D0EAEC8E
:1073A0008FF0EF6A23D00A0E166EEAEC8FF01650BB
:1073B000EF261CD00A0E166EEAEC8FF01650EF5E28
:1073C00015D0010EE66E4AEC8CF0D7EC93F0F1513B
:1073D000B4EC92F0E66E040E0101F003A6EC8EF020
:1073E000F15100013CEC8BF04BEC8DF0FEEC22F007
:1073F000080E0101F05D05E1CBEC90F0ADEC8EF0F4
:1074000004D0CBEC90F0CBEC8CF0E552E55282D777
:10741000020EE15C02E2E16AE552E16E94EF87F070
:107420008AEC8FF00101AEB102D00001F46B0001D3
:10743000F45139E1F10EE66E000E0AEC88F07BECB7
:1074400094F029E1F10EE66E000EE66EDCEC90F0B1
:10745000F31821E115501FE10001010EF46F300E09
:10746000F15DF06F000EF05D41E3080EF05D3EE26D
:10747000F0519AEC88F0EFCFF0F04BEC8FF0E66A29
:10748000370E8DEC91F00001F56FF66BF76BF86B32
:1074900046C141FDACD0C4EC96F001E0A8D0155037
:1074A00001E0A5D023D00D01415120E00101785128
:1074B000791101E19CD0E0EC88F0B8EC8CF001E1AE
:1074C00096D046C141FD010EDB502A0804E0010EB2
:1074D000DB5023080FE1F5C0E6FFF6C0E6FFF7C07A
:1074E000E6FFF8C0E6FF340E8DEC91F00101786BF9
:1074F000796B7DD0010EDB50440A69E0710A5EE0D1
:10750000010A52E0020A46E0010A3BE0060A30E0C6
:10751000090A1CE00A0A11E00B0A0BE00A0A59E109
:107520000001E051F927E151FA23E251FB23E35135
:1075300039D0E00EE96E000E0CD00001E451F927BD
:10754000E551FA23E651FB23E7512CD0E40EE96E16
:10755000000EEA6EEE500001F95D146EEE50FA591D
:10756000156EEE50FB59166EEE50FC59176E31D069
:107570000001E851F927E951FA23EA51FB23EB51C5
:1075800011D00001E851F95FE951FA5BEA51FB5B68
:10759000EB5112D00001EC51F927ED51FA23EE51D5
:1075A000FB23EF51FC2315D00001EC51F95FED51A5
:1075B000FA5BEE51FB5BEF51FC5B0BD0F5C0F9F0D1
:1075C000F6C0FAF0F7C0FBF0F8C0FCF002D04BECCC
:1075D0008DF0F9C0E6FFFAC0E6FFFBC0E6FFFCC095
:1075E000E6FF340E8DEC91F0FEEC22F064D7020E33
:1075F000E15C02E2E16AE552E16E94EF87F0B6ECFD
:107600008FF0080EDF6EDF5005E0D4EC88F0EF8AD3
:10761000DF06F9D7E55294EF87F0B6EC8FF0080E4D
:10762000DF6EDF5003E060EC94F0FBD7E55294EF9F
:1076300087F068EC96F0CBEC88F001018351EE5CAA
:10764000146E8451EE58156E8551EE58166E8651A3
:10765000EE58A8EC8AF00BE3DFCF83F1010EDBCF0D
:1076600084F1020EDBCF85F1030EDBCF86F1040E31
:10767000E15C02E2E16AE552E16E94EF87F0AFC1AE
:1076800091F1AFC1E6FFCBEC95F00101B66F050EAD
:10769000B65D01E3B66BB651B3EC8EF0B427060EBF
:1076A000B523120001019151AF5D11E13BEC88F06F
:1076B00001018351065C146E84510758156E855183
:1076C0000858166E86510958A8EC8AF001E2D7DFF7
:1076D00012008FEC87F0AFC191F1050EF6EC87F048
:1076E00002E3010E0FD0FE0EDBCFB6F1DB50B3ECA0
:1076F0008EF00101B427060EB5233BEC88F054EC64
:107700008DF0000E94EF87F0A0EC95F002E3FE0EF2
:10771000DB6AFDEC90F0EF50E66ECBEC95F0E66E98
:10772000D8DFE55294EF87F042EC96F0AEB116D078
:10773000F76BCCEC8AF0770EEE1802E1030EED1831
:1077400008E0CCEC8AF0710EEE1808E1370EED1867
:1077500005E1A388A38A0201010EFF6F0101F75121
:107760003FE1DEEC8AF0610E081802E1370E0918DD
:107770001BE0710E081802E1370E091815E0760EAD
:10778000081802E1030E091806E0770E081815E143
:10779000030E091812E1E66A44EC88F04B0EE66E1F
:1077A00091EC2AF0E55206D044EC88F04B0EE66EE0
:1077B000A4EC2CF0BAEC8FF0DF6EDF500AE101018F
:1077C000010EF76F4FEC8EF044EC88F072EC96F0FF
:1077D00057D0C4EC96F054E1155052E1FF0E51D051
:1077E000F70529E1DEEC8AF0770E081802E1030EB6
:1077F000091817E0710E081802E1370E091811E098
:10780000760E081802E1030E091806E0610E08184A
:107810000EE1370E09180BE144EC88F061EC0FF033
:1078200004D044EC88F03EECB1F0E552E5520101A1
:10783000020EF76F25D0DEEC8AF0770E081802E111
:10784000030E091817E0710E081802E1370E091827
:1078500011E0760E081802E1030E091806E0610E29
:1078600008180EE1370E09180BE105EC0FF00009BE
:1078700007E004D0E2ECB0F0000902E0000E01D015
:10788000010EE55294EF87F042EC96F0AEA1F86B52
:10789000F8511CE1060EE66E7DEC2BF0E552DF6E32
:1078A000DF500EE10101FF0ED880C055000EC1551A
:1078B00002E2C069C16BC0C13FFD010EF86F0CD080
:1078C000C4EC96F009E1155007E103D00D013F51DA
:1078D00003E10101786B796BE55294EF87F0D9CF22
:1078E000E6FFE1CFD9FF130EE12601018D51010121
:1078F0008E1128E0460EE66E0D0EE66EA3EC00F04B
:10790000E552E55201017B51065C146E01017C5188
:107910000758156E01017D510858166E01017E5100
:107920000958176ED8802C0E1454010E1554000EF1
:107930001654000E175406E201018D6B01018E6B87
:1079400001018F6B040EDB6A0601FE5102E10F019B
:107950005D6B0701005101E06CDE010E0101AE1507
:1079600002E0D7EF41F00101B35102E0D7EF41F05F
:107970000701005102E1D7EF41F0FEEC22F0DF6E8B
:107980002A0EDF5C0EE0DFCFE6FFE66AD5EC17F0EB
:10799000E552E552F3CF14F0F4CF15F01450151062
:1079A00006E00101786B796B0F01006B80D3AFC1EA
:1079B000E6FFDFCFE6FFE8EC15F0E552E5520009FF
:1079C0000BE00101786B796B0F01006B0601FE5132
:1079D00002E10F015D6B6BD3DFCFE6FF000EE66EB9
:1079E0000F0EE66E69EC05F0E552E552E552010135
:1079F0008D5101018E110BE00101AF510101905D2C
:107A000006E001018D6B01018E6B01018F6BD95076
:107A1000080FE66E000EDA20E66E000EE66E0F0E20
:107A2000E66E070EE66E140EE66E620EE66E0D0E44
:107A3000E66E4AEC85F0146E080EE15E1450E76EB7
:107A4000050EE7CFDBFF050EDB50020850E1010E0B
:107A5000F36E040EF3CFDBFF0F01006B0101786BB7
:107A6000796B080EDBCF14F0090EDBCF15F015345F
:107A700004E214500108000E155408E20101010E41
:107A80008D6F01018E6B01018F6B11D00101010E11
:107A90008E6FD950080FE96EDACFEAFFEE50ED1085
:107AA00003E10101010E8F6F0101010E8D6F460E82
:107AB000E66E0D0EE66EA3EC00F0E552E55206C050
:107AC0007BF107C07CF108C07DF109C07EF1AFC138
:107AD00090F1080E0101AF5D09E1010E01010B15E6
:107AE00005E0AFC1E6FFB9EC29F0E552E0D2050EA2
:107AF000DB0409E1010EF36E040EF3CFDBFF01019D
:107B0000786B796BD4D2D950060FE66E000EDA206E
:107B1000E66E000EE66E0F0EE66E040EE66E010EC9
:107B2000E66E100EE66E390EE66E010EE66EB2ECF3
:107B300084F0146E090EE15E1450E76E050EE7CF77
:107B4000DBFF110EDB6A050EDB5001E0A8D0D95037
:107B5000060FE66E000EDA20E66E000EE66E0F0EE1
:107B6000E66EFA0EE66EE66A000EE66E200EE66E31
:107B7000000EE66EB2EC84F0146E090EE15E145055
:107B8000E76E050EE7CFDBFF010EF36E110EF3CFAC
:107B9000DBFF050EDB50020801E081D0000E166EFF
:107BA000200E176E000E186E060EDBCF19F0070EB2
:107BB000DBCF1AF01B6A1ABE1B68090E0C6E0D6A29
:107BC0000E6A19C007F01AC008F01BC009F0E4ECF7
:107BD000B6F004C019F005C01AF006C01BF016502C
:107BE0001924F36E17501A20F46E18501B20F86EEB
:107BF000F4CFF7FFF3CFF6FF060EF626000EF722BE
:107C0000000EF8220900F5CF14F00800F5CF15F0AA
:107C1000150E141802E1010E15183FE0000E1E6E3D
:107C2000200E1F6E000E206E060EDBCF21F0070E19
:107C3000DBCF22F0236A22BE2368090E0C6E0D6A88
:107C40000E6A21C007F022C008F023C009F0E4EC5E
:107C5000B6F004C021F005C022F006C023F01E508B
:107C60002124F36E1F502220F46E20502320F86E42
:107C7000F4CFF7FFF3CFF6FF060EF626000EF7223D
:107C8000000EF8220900F5CF1CF00800F5CF1DF01A
:107C90001C5002E1010E1D1802E1050EDB6A050E03
:107CA000DB500AE10101786B796B0101AE6B0F01CA
:107CB000006BF9EC22F0FBD1050EDB50020801E06D
:107CC000EED1040EDB6A0F01006B110EDB5001E0F8
:107CD000F3D0100E146E390E156E010E166E060ED0
:107CE000DBCF17F0070EDBCF18F0196A18BE196842
:107CF000090E0C6E0D6A0E6A17C007F018C008F066
:107D000019C009F0E4ECB6F004C017F005C018F093
:107D100006C019F014501724F36E15501820F46E95
:107D200016501920F86EF4CFF7FFF3CFF6FF060ECA
:107D3000F626000EF722000EF8220900F5CF78F1A2
:107D40000A00F5CF79F10601FE5138E1100E146EEC
:107D5000390E156E010E166E060EDBCF17F0070EEC
:107D6000DBCF18F0196A18BE1968090E0C6E0D6A7F
:107D70000E6A17C007F018C008F019C009F0E4EC4B
:107D8000B6F004C017F005C018F006C019F0145082
:107D90001724F36E15501820F46E16501920F86E43
:107DA000F4CFF7FFF3CFF6FF080EF626000EF7220A
:107DB000000EF8220800F5CF0CFF05D00601FE05E5
:107DC00002E108CF0CFF100E156E390E166E010E73
:107DD000176E060EDBCF18F0070EDBCF19F01A6A0C
:107DE00019BE1A68090E0C6E0D6A0E6A18C007F0EB
:107DF00019C008F01AC009F0E4ECB6F004C018F09D
:107E000005C019F006C01AF015501824F36E16506C
:107E10001920F46E17501A20F86EF4CFF7FFF3CF45
:107E2000F6FF080EF626000EF722000EF8220800D4
:107E3000F5500F010C15146E800E14140F010A6F0B
:107E4000100E146E390E156E010E166E060EDBCF77
:107E500017F0070EDBCF18F0196A18BE1968090E63
:107E60000C6E0D6A0E6A17C007F018C008F019C032
:107E700009F0E4ECB6F004C017F005C018F006C035
:107E800019F014501724F36E15501820F46E165084
:107E90001920F86EF4CFF7FFF3CFF6FF080EF626A1
:107EA000000EF722000EF8220800F5500F010C1109
:107EB000100B0F010B6FF2D0000E146E200E156E1A
:107EC000000E166E060EDBCF17F0070EDBCF18F094
:107ED000196A18BE1968090E0C6E0D6A0E6A17C071
:107EE00007F018C008F019C009F0E4ECB6F004C0BF
:107EF00017F005C018F006C019F014501724F36EDF
:107F000015501820F46E16501920F86EF4CFF7FFB4
:107F1000F3CFF6FF060EF626000EF722000EF8222B
:107F20000900F5CF78F10A00F5CF79F10601FE518D
:107F300038E1000E146E200E156E000E166E060E41
:107F4000DBCF17F0070EDBCF18F0196A18BE1968DF
:107F5000090E0C6E0D6A0E6A17C007F018C008F003
:107F600019C009F0E4ECB6F004C017F005C018F031
:107F700006C019F014501724F36E15501820F46E33
:107F800016501920F86EF4CFF7FFF3CFF6FF080E66
:107F9000F626000EF722000EF8220800F5CF0CFF9F
:107FA00005D00601FE0502E108CF0CFF000E156E9C
:107FB000200E166E000E176E060EDBCF18F0070EA1
:107FC000DBCF19F01A6A19BE1A68090E0C6E0D6A19
:107FD0000E6A18C007F019C008F01AC009F0E4ECE6
:107FE000B6F004C018F005C019F006C01AF015501C
:107FF0001824F36E16501920F46E17501A20F86EDC
:10800000F4CFF7FFF3CFF6FF080EF626000EF722A7
:10801000000EF8220800F5500F010C15146E800EAA
:1080200014140F010A6F000E146E200E156E000E50
:10803000166E060EDBCF17F0070EDBCF18F0196AAD
:1080400018BE1968090E0C6E0D6A0E6A17C007F08B
:1080500018C008F019C009F0E4ECB6F004C017F03D
:1080600005C018F006C019F014501724F36E15500F
:108070001820F46E16501920F86EF4CFF7FFF3CFE6
:10808000F6FF080EF626000EF722000EF822080072
:10809000F5500F010C11100B0F010B6F08D0010EE2
:1080A000F36E040EF3CFDBFF0101786B796B0101F6
:1080B0007851791101E17BD10101781D01E1791D30
:1080C00004E10101786B796B62D1080E0101AF5DAB
:1080D00021E10101896B01018D5103E001018997C3
:1080E00002D00101898701018E5103E001018999C4
:1080F00002D0010189890F010C510F010B110101FF
:1081000089150F01096F0F01095103E00101786B17
:10811000796B3DD1010EAFC1E7FFE75204E0E846BD
:10812000FE0BE706FCE1E76E0A0EE7CFDBFF0A0E67
:10813000DBCFE6FFB4C1E9FFB5C1EAFF020EEB50A9
:10814000E552E71408E10A0EDB500101011506E0D3
:1081500001011C5103E00101899302D001018983CF
:1081600001016E1D156E01016D1D146EB4C1E9FF94
:10817000B5C1EAFF020EEB5014141514E76E120E8F
:10818000E7CFDBFFB4C114F0B5C115F0880E145E63
:10819000060E155A050E0D6E0E6A14C008F015C0B5
:1081A00009F08AECB6F008C014F009C015F00B0E07
:1081B00014C0DBFFB4C1E9FFB5C1EAFF040EEB5008
:1081C000E76E0C0EE7CFDBFF01011B5143E10A0E06
:1081D000DBCFE6FFB4C1E9FFB5C1EAFF030EEB5008
:1081E000E552E71437E1B4C1E9FFB5C1EAFFEF504A
:1081F000010101152FE0B4C1E9FFB5C1EAFFEF505D
:108200000101071527E00C0EDBCFE6FF0A0EDB505D
:10821000E552E71412E1010EF36E0B0EDB5004E0A1
:10822000D890F336E806FCE1F3500101951505E01E
:108230000C0EDB1C010107150DE10C0EDBCFE6FF78
:108240000A0EDB50E552E71408E00C0EDB5001018A
:10825000071503E00101899502D00101898501011B
:108260008D5103E00101899702D001018987010145
:108270008E5103E00101899902D0010189890F0122
:108280000C510F010B11010189150F01096F0A0E25
:10829000DB5001016D1503E00F01098B02D00F01C6
:1082A000099B0A0EDB5001016E1503E00F01098DD9
:1082B00002D00F01099D0F015D5103E0400E0F0137
:1082C00009170101000E785D500E79590AE301018A
:1082D0008F0ED8807855510E795503E39F0E0F010C
:1082E000091701011D510EE001018D5101018E118F
:1082F00009E0500E0F01091701018E5103E0100E25
:108300000F0109170601FE5106E00F01095103E1B3
:108310000F01010E5D6F01017A510EE00101030EA4
:10832000781901E1795104E1180E0F01091503E0F4
:108330000101786B796B2BD00F0109511BE0800E86
:108340000F010C150F010A15146E156A1450151043
:1083500011E10101AE810101AE93F9EC22F009CFE8
:10836000E6FFAFC1E6FFFEEC29F0E552E552010160
:10837000786B796B0A0EDB500101701508E0010182
:108380008D5101018E1103E10101786B796B080EAB
:108390000101AF5D0AE10101010E781901E1795196
:1083A00004E10101010EAC6F02D00101AC6B0101CF
:1083B0007851791102E137EF68F052EC3BF0460E4C
:1083C000E66E0D0EE66EA3EC00F0E552E55206C037
:1083D0007BF107C07CF108C07DF109C07EF101018D
:1083E000781D01E1791D02E00601FF6B040EDB50F0
:1083F00018E1080EE66E0F0EE66E78C1E6FF79C151
:10840000E6FF48EC16F0E552E552E552E552000968
:1084100008E1010EF36E040EF3CFDBFF0101786B70
:10842000796B18EC16F0040EDB5002E050EF46F0CA
:10843000010EF36E040EF3CFDBFF210E010178195C
:1084400002E1030E791901E165D3230E01017819C8
:1084500002E1030E791901E15DD3240E01017819BF
:1084600002E1030E791901E155D3020E01017819D9
:1084700002E1030E791901E14DD3030E01017819D0
:1084800002E1030E791901E145D3050E01017819C6
:1084900002E1030E791901E13DD3070E01017819BC
:1084A00002E1030E791901E135D30101785102E1AE
:1084B000030E791901E12ED3010E0101781902E1B1
:1084C000030E791901E1EFD2040E0101781902E1DE
:1084D000030E791901E1E7D2580E0101781902E182
:1084E000030E791901E1DFD2590E0101781902E179
:1084F000030E791901E1D7D2260E0101781902E1A4
:10850000030E791901E1BFD2250E0101781902E1AC
:10851000030E791901E166D2060E0101781902E114
:10852000030E791901E137D2080E0101781902E131
:10853000030E791901E122D2330E0101781902E10B
:10854000030E791901E1D2D13B0E0101781902E144
:10855000030E791901E1CAD1380E0101781902E13F
:10856000030E791901E17BD13A0E0101781902E17C
:10857000030E791901E173D1360E0101781902E178
:10858000030E791901E140D1370E0101781902E19A
:10859000030E791901E138D1310E0101781902E198
:1085A000030E791901E1A9D0320E0101781902E117
:1085B000030E791901E1A1D0390E0101781902E108
:1085C000030E791901E199D0300E0101781902E109
:1085D000030E79195BE0210E0101781901E179514F
:1085E00026E0010E0101781901E179510CE0E868FB
:1085F0000101781902E1E868791901E04ED301011F
:10860000786B796B4DD30101AE81440EE66E640E3A
:10861000E66E010EE66EAFC1E6FF6CEC2AF0E552A5
:10862000E552E552E5520101786B796B39D3010EC1
:10863000E66E7DEC2BF0E552E76E050EE7CFDBFF33
:10864000050EDB5016E101010051146E156A01019F
:108650001450C05D1550C15908E2C0C1E6FFAFC15A
:10866000E6FFBEEC30F0E552E5520101786B796B24
:108670000CD0050EDB50146E156AFF0E141801E1C4
:10868000155003E10101786B796B0AD3010EE66E98
:108690007DEC2BF0E552E76E050EE7CFDBFF050E14
:1086A000DB501EE10101080EC05D000EC15914E24D
:1086B0000A0E0101C025E96E090E0101C121EA6E11
:1086C000EF50E66E16EC81F0E552000905E0AFC10F
:1086D000E6FFB9EC29F0E5520101786B796B0CD01B
:1086E000050EDB50146E156AFF0E141801E11550CB
:1086F00003E10101786B796BD3D2010EE66E7DEC5C
:108700002BF0E552E76E050EE7CFDBFF050EDB50E1
:108710006EE10101080EC05D000EC15964E20F0157
:10872000095117E00F010C51146E156A1450800B9B
:108730004EE0F80E0F0109154AE10A0E0101C025AD
:10874000E96E090E0101C121EA6EEF500101AF5D32
:108750003EE10F01010E5D6F310E0101781902E15A
:10876000030E791915E10A0E0101C025E96E090E03
:108770000101C121EA6EEF50E66EF8EC80F0E5529F
:10878000000905E0AFC1E6FFB9EC29F0E5521ED0C3
:10879000320E0101781902E1030E791908E1E66A47
:1087A000C0C1E6FFE6EC30F0E552E5520FD0390EDD
:1087B0000101781902E1030E791908E1010EE66E54
:1087C000C0C1E6FFE6EC30F0E552E5520CD0010105
:1087D000AE93F9EC22F009CFE6FFAFC1E6FFFEEC65
:1087E00029F0E552E5520101786B796B0CD0050E4A
:1087F000DB50146E156AFF0E141801E1155003E1E9
:108800000101786B796B4CD20101AE8101010051FD
:108810000101AF5D20E2370E0101781902E1030E7C
:1088200079190EE0360E0101781902E1030E79196B
:1088300001E00CD0AFC1E6FF16EC81F0E55206D0A6
:10884000AFC1E6FFF8EC80F0E55200D0AFC1E6FF23
:10885000B9EC29F0E5520101786B796B21D2010165
:10886000AE810B0EDB6A0B0EDB50EA6A0A0FE96E73
:10887000090EEA22EF500101AF5D0CE0080EF36E25
:108880000B0EDBCFF4FFF350F45C04E200D00B0ED0
:10889000DB2AE9D7080EF36E0B0EDBCFF4FFF350A3
:1088A000F45C20E2380E0101781902E1030E791917
:1088B00009E1E66A0B0EDBCFE6FFE6EC30F0E552AD
:1088C000E55210D03A0E0101781902E1030E791930
:1088D00009E1010EE66E0B0EDBCFE6FFE6EC30F0B1
:1088E000E552E5520101786B796BDAD10D0EE66E37
:1088F0000F0EE66E4F0EE66EE1EC2BF0E552E55200
:10890000E552E76E050EE7CFDBFF050EDB5029E1F0
:10891000330E0101781902E1030E79190DE10D0EF4
:10892000E66E0F0EE66E98EC83F0E552E552E66EC9
:1089300040EC81F0E5520CD00D0EE66E0F0EE66EA7
:1089400098EC83F0E552E552E66E54EC81F0E55286
:10895000AFC1E6FFB9EC29F0E5520101786B796B04
:108960000CD0050EDB50146E156AFF0E141801E1D1
:10897000155003E10101786B796B92D10101AE8151
:1089800033EC81F0AFC1E6FFB9EC29F0E55201010B
:10899000786B796B85D1010EE66E7DEC2BF0E5529C
:1089A000E76E050EE7CFDBFF050EDB500EE1C0C121
:1089B000E6FF7BEC35F0E552AFC1E6FFB9EC29F0FC
:1089C000E5520101786B796B0CD0050EDB50146E0B
:1089D000156AFF0E141801E1155003E10101786BCF
:1089E000796B5ED10D0EE66E0F0EE66E020EE66E30
:1089F000E1EC2BF0E552E552E552E76E050EE7CFCC
:108A0000DBFF050EDB5032E10D0EE66E0F0EE66E5B
:108A10007AECADF0E552E552F3CF14F0F4CF15F057
:108A2000020E141801E1155020E1300E0F010E5D09
:108A3000E66E300E0F010D5DE66E9EEC33F0E552F2
:108A4000E552E76E050EE7CFDBFF050EDB500AE1CE
:108A5000010EF36E050EF3CFDBFFAFC1E6FFB9ECFD
:108A600029F0E5520101786B796B0CD0050EDB50D3
:108A7000146E156AFF0E141801E1155003E101018F
:108A8000786B796B0DD10101AE81010EE66EC1EC00
:108A900033F0E552AFC1E6FFB9EC29F0E552010130
:108AA000786B796BFDD00101AE81590E0101781907
:108AB00002E1030E791922E0580E0101781902E152
:108AC000030E791918E0040E0101781902E1030E72
:108AD00079190BE0010E0101781902E1030E7919F1
:108AE00001E00FD0F8EC33F00CD024C1E6FF7BECB2
:108AF00035F0E55206D064EC33F003D082EC33F06D
:108B000000D0AFC1E6FFB9EC29F0E5520101786B66
:108B1000796BC6D00101AE81D9500B0FE66E000E05
:108B2000DA20E66E9E0EE66E020EE66ECDEC6BF07F
:108B3000E552E552E552E5520F01095127E0180EC2
:108B40000F01091501E099D001018E5105E1400E98
:108B50000F01091501E091D00B0EDB1C146E0A0EFB
:108B6000DB5001016D15141401E187D0070E0101DE
:108B7000AF150B0DF3CFE9FFF4CFEAFF000EE926A6
:108B8000040EEA22EE52EF0401E077D00F01010E4D
:108B90005D6F0B0EDB6A0101785102E1030E79195A
:108BA00054E0070E0101781902E1030E79194AE039
:108BB000050E0101781902E1030E791940E0030E58
:108BC0000101781902E1030E791936E0020E010164
:108BD000781902E1030E79192CE0240E01017819AD
:108BE00002E1030E79191DE0230E0101781902E15B
:108BF000030E79190FE0210E0101781902E1030E2D
:108C0000791901E025D01AEC36F0E76E0B0EE7CFAC
:108C1000DBFF1ED0DAEC36F0E76E0B0EE7CFDBFFA2
:108C200017D03AEC36F0010EF36E0B0EF3CFDBFFEC
:108C30000FD0B4EC35F00CD029EC35F009D0FFECB6
:108C400034F006D071EC37F003D0A9EC37F000D047
:108C50000B0EDB5011E10101785102E1030E79198D
:108C600006E1AFC1E6FFE7EC29F0E55205D0AFC160
:108C7000E6FFB9EC29F0E5520CD00101AE93F9EC16
:108C800022F009CFE6FFAFC1E6FFFEEC29F0E55286
:108C9000E5520101786B796B03D0040EDB6A00D0DA
:108CA000040EDB5002E0F0EF51F0010EF36E040E03
:108CB000F3CFDBFF060E0101781902E1040E7919EA
:108CC00002E1EAEF51F00101785102E1040E791955
:108CD00001E1D7D3010E0101781902E1040E7919DF
:108CE00001E1CFD3020E0101781902E1040E7919D6
:108CF00001E1C7D3030E0101781902E1040E7919CD
:108D000001E1BFD3040E0101781902E1040E7919C3
:108D100001E1B7D3050E0101781902E1040E7919BA
:108D200001E1AFD3070E0101781902E1040E7919B0
:108D300001E1A7D3080E0101781902E1040E7919A7
:108D400001E19FD3100E0101781902E1040E791997
:108D500001E197D3090E0101781902E1040E791996
:108D600001E18FD3110E0101781902E1040E791986
:108D700001E187D30A0E0101781902E1040E791985
:108D800001E17FD3D20E0101781902E1400E791979
:108D900001E177D30B0E0101781902E1040E791974
:108DA00001E16FD3D30E0101781902E1400E791968
:108DB00001E167D30C0E0101781902E1040E791963
:108DC00001E15FD3D00E0101781902E1400E79195B
:108DD00001E157D3D10E0101781902E1400E791952
:108DE00001E14FD3140E0101781902E1040E791943
:108DF00001E147D3150E0101781902E1040E79193A
:108E000001E13FD3160E0101781902E1040E791930
:108E100001E137D3190E0101781902E1040E791925
:108E200001E12FD31A0E0101781902E1040E79191C
:108E300001E127D31B0E0101781902E1040E791913
:108E400001E11FD31C0E0101781902E1040E79190A
:108E500001E117D31D0E0101781902E1040E791901
:108E600001E10FD3200E0101781902E1040E7919F6
:108E700001E107D3210E0101781902E1040E7919ED
:108E800001E1FFD2220E0101781902E1040E7919E5
:108E900001E1F7D2230E0101781902E1040E7919DC
:108EA00001E1EFD2240E0101781902E1040E7919D3
:108EB00001E1E7D2250E0101781902E1040E7919CA
:108EC00001E1DFD2200E0101781902E1030E7919C8
:108ED00001E1ADD2220E0101781902E1030E7919E8
:108EE00001E1A5D2820E0101781902E1030E791980
:108EF00001E18FD2800E0101781902E1030E791988
:108F000001E1F5D1810E0101781902E1030E791911
:108F100001E1EDD1170E0101781902E1040E791972
:108F200001E1E5D1180E0101781902E1040E791969
:108F300001E1DDD1570E0101781902E1030E791923
:108F400001E19FD1550E0101781902E1030E791953
:108F500001E161D1540E0101781902E1030E791982
:108F600001E1E3D0560E0101781902E1030E7919EF
:108F700001E1DBD0510E0101781902E1030E7919EC
:108F800001E1C3D0500E0101781902E1030E7919F5
:108F900066E0520E0101781902E1030E79195FE0D3
:108FA000130E0101781902E1030E791946E0120E41
:108FB0000101781902E1030E79192DE0110E01016A
:108FC000781902E1030E79191FE0100E01017819DA
:108FD00002E1030E791911E0A00E0101781902E1F6
:108FE000020E791902E0EDEF51F00101786B796B17
:108FF0000101010EA96FF0EF51F00101786B796B5F
:10900000DFEC20F0F0EF51F00101786B796BFBECB5
:1090100020F0F0EF51F00101AE81580EE66E040E23
:10902000E66EAFC1E6FF5EEC2AF0E552E552E5528E
:109030000101786B796BF0EF51F00101AE81800E88
:10904000E66E040EE66EAFC1E6FF5EEC2AF0E55276
:10905000E552E5520101786B796BF0EF51F00101B7
:10906000AE810F0109511AE00F010C51146E156AFF
:109070001450800B39E0F80E0F01091535E1070E89
:109080000101AF150B0DF3CFE9FFF4CFEAFF000E9E
:10909000E926040EEA22EE52EF0426E10F01010E4A
:1090A0005D6F520E0101781902E1030E791912E089
:1090B000500E0101781902E1030E791901E013D075
:1090C000FAEC27F0000905E1AFC1E6FFB9EC29F0A1
:1090D000E55209D0AFC1E6FF1EEC28F0E5520101D0
:1090E000786B796B00D00CD00101AE93F9EC22F0D3
:1090F00009CFE6FFAFC1E6FFFEEC29F0E552E552ED
:109100000101786B796BF0EF51F00101AE810CEC4D
:1091100028F0000905E1AFC1E6FFB9EC29F0E552FE
:109120000101786B796BF0EF51F0010EE66E7DEC8A
:109130002BF0E552E76E050EE7CFDBFF050EDB50A7
:109140005CE10101080EC05D000EC15952E20F0141
:10915000095117E00F010C51146E156A1450800B61
:109160003CE0F80E0F01091538E10A0E0101C02597
:10917000E96E090E0101C121EA6EEF500101AF5DF8
:109180002CE10F01010E5D6F560E0101781902E10D
:10919000030E79191BE0540E0101781902E1030E48
:1091A000791901E019D00A0E0101C025E96E090EF6
:1091B0000101C121EA6EEF50E66E48EC28F0E5525D
:1091C000AFC1E6FFB9EC29F0E55206D0C0C1E6FF19
:1091D00054EC28F0E55200D00CD00101AE93F9EC2C
:1091E00022F009CFE6FFAFC1E6FFFEEC29F0E55221
:1091F000E5520101786B796B0CD0050EDB50146ED3
:10920000156AFF0E141801E1155003E10101786B96
:10921000796BF0EF51F0010EE66E7DEC2BF0E5522C
:10922000E76E050EE7CFDBFF050EDB501CE1010109
:10923000080EC05D000EC15912E20A0E0101C025E0
:10924000E96E090E0101C121EA6EEF50E66E4EECA7
:1092500028F0E552AFC1E6FFB9EC29F0E552010173
:10926000786B796B0CD0050EDB50146E156AFF0E0F
:10927000141801E1155003E10101786B796BF0EFEF
:1092800051F0010EE66E7DEC2BF0E552E76E050E17
:10929000E7CFDBFF050EDB501CE10101080EC05DCE
:1092A000000EC1590DE20A0E0101C025E96E090E3A
:1092B0000101C121EA6EEF50E66EA4EC28F0E55200
:1092C000AFC1E6FFD0EC29F0E5520101786B796B74
:1092D0000CD0050EDB50146E156AFF0E141801E158
:1092E000155003E10101786B796BF0EF51F0010E3D
:1092F000E66E7DEC2BF0E552E76E050EE7CFDBFF67
:10930000050EDB5001E077D00101080EC05D000EB4
:10931000C15965E2180E0101781902E1040E7919AC
:109320004CE0170E0101781902E1040E791933E0BF
:10933000810E0101781902E1030E79191AE0800EFD
:109340000101781902E1030E791901E048D00A0EF3
:109350000101C025E96E090E0101C121EA6EEF503D
:10936000E66E86EC81F0E552E76E050EE7CFDBFF97
:1093700036D00A0E0101C025E96E090E0101C12196
:10938000EA6EEF50E66EA1EC81F0E552E76E050E55
:10939000E7CFDBFF24D00A0E0101C025E96E090EDC
:1093A0000101C121EA6EEF50E66EB5EC81F0E552A5
:1093B000E76E050EE7CFDBFF12D00A0E0101C025D4
:1093C000E96E090E0101C121EA6EEF50E66EC7ECAD
:1093D00081F0E552E76E050EE7CFDBFF00D0050E0A
:1093E000DB5005E1AFC1E6FFB9EC29F0E552010120
:1093F000786B796B0CD0050EDB50146E156AFF0E7E
:10940000141801E1155003E10101786B796BF0EF5D
:1094100051F00101AE81D9EC81F00101786B796BDB
:10942000AFC1E6FFB9EC29F0E552F0EF51F00101D0
:10943000AE81220E0101781902E1030E791912E0C2
:10944000200E0101781902E1030E791901E014D010
:10945000FCEC35F0000905E1AFC1E6FFB9EC29F0FD
:10946000E5520AD0B8EC36F0000905E1AFC1E6FFDD
:10947000B9EC29F0E55200D00101786B796BF0EF7F
:1094800051F00101AEB102D00F015E6B0F015E51D0
:10949000040A02E166EF51F0070A02E150EF51F0D1
:1094A000010A02E1E6EF4FF0030A01E17ED1010A71
:1094B00002E0E3EF51F0090E0101781902E1040E18
:1094C000791901E14BD1110E0101781902E1040E65
:1094D000791901E143D10A0E0101781902E1040E64
:1094E000791901E13BD1D20E0101781902E1400E58
:1094F000791901E133D10B0E0101781902E1040E53
:10950000791901E12BD1D30E0101781902E1400E46
:10951000791901E123D10C0E0101781902E1040E41
:10952000791901E11BD1D00E0101781902E1400E39
:10953000791901E113D1D10E0101781902E1400E30
:10954000791901E10BD11B0E0101781902E1040E1A
:10955000791901E103D11C0E0101781902E1040E11
:10956000791901E1FBD0230E0101781902E1040E03
:10957000791901E1F3D0240E0101781902E1040EFA
:10958000791901E1EBD0250E0101781902E1040EF1
:10959000791901E1E3D0080E0101781902E1040E06
:1095A000791901E1CBD0050E0101781902E1040E11
:1095B000791901E1B3D0040E0101781902E1040E1A
:1095C000791901E19BD0140E0101781902E1040E12
:1095D000791901E193D0150E0101781902E1040E09
:1095E000791901E18BD0030E0101781902E1040E13
:1095F000791974E0020E0101781902E1040E79195B
:109600005DE00101785102E1040E791947E0010E95
:109610000101781902E1040E791940E0070E0101F9
:10962000781902E1040E791939E0160E0101781952
:1096300002E1040E791932E0100E0101781902E1FD
:10964000040E79192BE0190E0101781902E1040EBC
:10965000791924E01A0E0101781902E1040E791932
:109660001DE01D0E0101781902E1040E791916E0C2
:10967000200E0101781902E1040E79190FE0210E84
:109680000101781902E1040E791908E0220E0101A6
:10969000781902E1040E791901E070D00D0EE66E22
:1096A0000F0EE66E050EE66EE1EC2BF0E552E5528C
:1096B000E552E76E050EE7CFDBFF60D00D0EE66EDC
:1096C0000F0EE66E070EE66EE1EC2BF0E552E5526A
:1096D000E552E76E050EE7CFDBFF50D00D0EE66ECC
:1096E0000F0EE66E0A0EE66EE1EC2BF0E552E55247
:1096F000E552E76E050EE7CFDBFF40D00D0EE66EBC
:109700000F0EE66E0C0EE66EE1EC2BF0E552E55224
:10971000E552E76E050EE7CFDBFF30D00D0EE66EAB
:109720000F0EE66E060EE66EE1EC2BF0E552E5520A
:10973000E552E76E050EE7CFDBFF20D00D0EE66E9B
:109740000F0EE66E070EE66EE1EC2BF0E552E552E9
:10975000E552E76E050EE7CFDBFF10D00D0EE66E8B
:109760000F0EE66E010EE66EE1EC2BF0E552E552CF
:10977000E552E76E050EE7CFDBFF00D0050EDB50AC
:1097800004E10F01010E5E6F0ED0050EDB50146E6A
:10979000156AFF0E141801E1155005E1F9EC22F0ED
:1097A0000101786B796BE9EF51F0300E0F010D5D1F
:1097B0000F015F6F080E0F015F5D09E20F015F513E
:1097C000EA6A0A0FE96E090EEA22EFCF5FFF010194
:1097D00000510F015F5D01E3F6D30E0EE66E0F0E32
:1097E000E66EFCECB4F0E552E5520D0E06C0DBFF70
:1097F0000E0E07C0DBFF0F0E08C0DBFF100E09C006
:10980000DBFF0101785102E1040E79195CE0010EE1
:109810000101781902E1040E791955E0020E0101E7
:10982000781902E1040E79194EE0030E010178194E
:1098300002E1040E791947E0040E0101781902E1F2
:10984000040E791940E0050E0101781902E1040EB9
:10985000791939E0070E0101781902E1040E79192E
:1098600032E0080E0101781902E1040E79192BE0AB
:10987000140E0101781902E1040E791924E0150E85
:109880000101781902E1040E79191DE0160E01019B
:10989000781902E1040E791916E0210E01017819F8
:1098A00002E1040E79190FE0250E0101781902E199
:1098B000040E791908E0240E0101781902E1040E62
:1098C000791901E00AD05FCFE6FFA1EC81F0E55203
:1098D000E76E050EE7CFDBFF00D0240E01017819FB
:1098E00002E1040E791901E151D3250E0101781925
:1098F00002E1040E791901E136D3230E0101781932
:1099000002E1040E791901E11BD3220E010178193D
:1099100002E1040E791901E1F7D2210E0101781953
:1099200002E1040E791901E1D3D20A0E010178197E
:1099300002E1040E791901E1B8D2D20E01017819C1
:1099400002E1400E791901E1B0D20B0E0101781944
:1099500002E1040E791901E1A8D2D30E01017819B0
:1099600002E1400E791901E1A0D20C0E0101781933
:1099700002E1040E791901E198D2D00E01017819A3
:1099800002E1400E791901E190D2D10E010178195E
:1099900002E1400E791901E188D2200E0101781907
:1099A00002E1040E791901E164D21D0E010178195A
:1099B00002E1040E791901E140D21C0E010178196F
:1099C00002E1040E791901E125D21B0E010178197B
:1099D00002E1040E791901E10AD21A0E0101781987
:1099E00002E1040E791901E1F4D1190E010178198F
:1099F00002E1040E791901E1D0D1160E01017819A6
:109A000002E1040E791901E1BAD1150E01017819AC
:109A100002E1040E791901E198D1140E01017819BF
:109A200002E1040E791901E176D1110E01017819D4
:109A300002E1040E791901E15BD1090E01017819E7
:109A400002E1040E791901E140D1100E01017819EB
:109A500002E1040E791901E11CD1080E0101781907
:109A600002E1040E791901E1F8D0070E010178191D
:109A700002E1040E791901E1D4D0050E0101781933
:109A800002E1040E791901E1B0D0040E0101781948
:109A900002E1040E791901E18CD0030E010178195D
:109AA00002E1040E791969E0020E0101781902E160
:109AB000040E791946E0010E0101781902E1040E45
:109AC000791923E00101785102E1040E791901E0CE
:109AD00070D2D9500D0FE96EDACFEAFFEECFE6FF74
:109AE000EECFE6FFEECFE6FFEFCFE6FF300EE66EFD
:109AF0005FCFE6FF1AEC19F0146E060EE15E14500B
:109B0000E76E050EE7CFDBFF54D2D9500D0FE96E9B
:109B1000DACFEAFFEECFE6FFEECFE6FFEECFE6FFCD
:109B2000EFCFE6FF310EE66E5FCFE6FF1AEC19F0DD
:109B3000146E060EE15E1450E76E050EE7CFDBFFF4
:109B400038D2D9500D0FE96EDACFEAFFEECFE6FF3B
:109B5000EECFE6FFEECFE6FFEFCFE6FF320EE66E8A
:109B60005FCFE6FF1AEC19F0146E060EE15E14509A
:109B7000E76E050EE7CFDBFF1CD2D9500D0FE96E63
:109B8000DACFEAFFEECFE6FFEECFE6FFEECFE6FF5D
:109B9000EFCFE6FF330EE66E5FCFE6FF1AEC19F06B
:109BA000146E060EE15E1450E76E050EE7CFDBFF84
:109BB00000D2D9500D0FE96EDACFEAFFEECFE6FF03
:109BC000EECFE6FFEECFE6FFEFCFE6FF340EE66E18
:109BD0005FCFE6FF1AEC19F0146E060EE15E14502A
:109BE000E76E050EE7CFDBFFE4D1D9500D0FE96E2C
:109BF000DACFEAFFEECFE6FFEECFE6FFEECFE6FFED
:109C0000EFCFE6FF350EE66E5FCFE6FF1AEC19F0F8
:109C1000146E060EE15E1450E76E050EE7CFDBFF13
:109C2000C8D1D9500D0FE96EDACFEAFFEECFE6FFCB
:109C3000EECFE6FFEECFE6FFEFCFE6FF380EE66EA3
:109C40005FCFE6FF1AEC19F0146E060EE15E1450B9
:109C5000E76E050EE7CFDBFFACD1D9500D0FE96EF3
:109C6000DACFEAFFEECFE6FFEECFE6FFEECFE6FF7C
:109C7000EFCFE6FF390EE66E5FCFE6FF1AEC19F084
:109C8000146E060EE15E1450E76E050EE7CFDBFFA3
:109C900090D1D9500D0FE96EDACFEAFFEECFE6FF93
:109CA000EECFE6FFEECFE6FFEFCFE6FF430EE66E28
:109CB0005FCFE6FF1AEC19F0146E060EE15E145049
:109CC000E76E050EE7CFDBFF74D1E66AE66AE66A67
:109CD000E66A3A0EE66E5FCFE6FF1AEC19F0146EF4
:109CE000060EE15E1450E76E050EE7CFDBFF61D193
:109CF000E66AE66AE66AE66A3B0EE66E5FCFE6FF74
:109D00001AEC19F0146E060EE15E1450E76E050EA3
:109D1000E7CFDBFF4ED1D9500D0FE96EDACFEAFF66
:109D2000EECFE6FFEECFE6FFEECFE6FFEFCFE6FFAA
:109D30005FCFE6FFC0ECABF0146E050EE15E145091
:109D4000E76E050EE7CFDBFF34D1D9500D0FE96E7A
:109D5000DACFEAFFEECFE6FFEECFE6FFEECFE6FF8B
:109D6000EFCFE6FF5FCFE6FFC6ECABF0146E050E5B
:109D7000E15E1450E76E050EE7CFDBFF1AD10D0E42
:109D8000DBCFE6FF5FCFE6FFCCECABF0E552E55270
:109D9000E76E050EE7CFDBFF0CD1D9500D0FE96E52
:109DA000DACFEAFFEECFE6FFEECFE6FFEECFE6FF3B
:109DB000EFCFE6FF440EE66E5FCFE6FF1AEC19F038
:109DC000146E060EE15E1450E76E050EE7CFDBFF62
:109DD000F0D00D0EDBCFE6FF5FCFE6FFD3ECABF0AC
:109DE000E552E552E76E050EE7CFDBFFE2D0E66A0B
:109DF000E66AE66AE66A450EE66E5FCFE6FF1AECB3
:109E000019F0146E060EE15E1450E76E050EE7CFF2
:109E1000DBFFCFD0E66AE66AE66AE66A460EE66EE1
:109E20005FCFE6FF1AEC19F0146E060EE15E1450D7
:109E3000E76E050EE7CFDBFFBCD0D9500D0FE96E02
:109E4000DACFEAFFEECFE6FFEECFE6FFEECFE6FF9A
:109E5000EFCFE6FF470EE66E5FCFE6FF1AEC19F094
:109E6000146E060EE15E1450E76E050EE7CFDBFFC1
:109E7000A0D0D9500D0FE96EDACFEAFFEECFE6FFA2
:109E8000EECFE6FFEECFE6FFEFCFE6FF480EE66E41
:109E90005FCFE6FF1AEC19F0146E060EE15E145067
:109EA000E76E050EE7CFDBFF84D0E66AE66AE66A76
:109EB000E66A370EE66E5FCFE6FF1AEC19F0146E15
:109EC000060EE15E1450E76E050EE7CFDBFF71D0A2
:109ED000D9500D0FE96EDACFEAFFEECFE6FFEECFF5
:109EE000E6FFEECFE6FFEFCFE6FF490EE66E5FCF6F
:109EF000E6FF1AEC19F0146E060EE15E1450E76EE0
:109F0000050EE7CFDBFF55D0D9500D0FE96EDACF44
:109F1000EAFFEECFE6FFEECFE6FFEECFE6FFEFCFB4
:109F2000E6FF4A0EE66E5FCFE6FF1AEC19F0146EFC
:109F3000060EE15E1450E76E050EE7CFDBFF39D069
:109F4000E66AE66AE66AE66A4B0EE66E5FCFE6FF11
:109F50001AEC19F0146E060EE15E1450E76E050E51
:109F6000E7CFDBFF26D0E66AE66AE66AE66A4C0ED1
:109F7000E66E5FCFE6FF1AEC19F0146E060EE15E96
:109F80001450E76E050EE7CFDBFF13D0E66AE66AF2
:109F9000E66AE66A4D0EE66E5FCFE6FF1AEC19F050
:109FA000146E060EE15E1450E76E050EE7CFDBFF80
:109FB00000D0050EDB5004E10F01020E5E6F02D0EF
:109FC0000F015E6902D00F015E6903D2D9500D0FF7
:109FD000E66E000EDA20E66E5FCFE6FFC1ECAAF077
:109FE000E552E552E552E76E050EE7CFDBFF050EC1
:109FF000DB5001E154D10101785102E1040E7919DD
:10A0000047E0020E0101781902E1040E791940E0DF
:10A01000030E0101781902E1040E791939E0040EEA
:10A020000101781902E1040E791932E0050E0101EF
:10A03000781902E1040E79192BE0070E0101781955
:10A0400002E1040E791924E0080E0101781902E1F9
:10A05000040E79191DE0210E0101781902E1040EA8
:10A06000791916E0230E0101781902E1040E79191D
:10A070000FE0240E0101781902E1040E791908E0BD
:10A08000250E0101781902E1040E791901E01CD0B6
:10A09000050EDB040CE1010E5FCFE7FFE75204E0A1
:10A0A000E846FE0BE706FCE10101A6130CD0010E09
:10A0B0005FCFE7FFE75204E0E846FE0BE706FCE16E
:10A0C000E81C0101A61700D0050EDB50030A01E1D0
:10A0D000CDD0010A09E0030A01E0D0D0AFC1E6FF0C
:10A0E000B9EC29F0E552D2D0D10E0101781902E184
:10A0F000400E79194CE0D00E0101781902E1400EB2
:10A1000079193FE00C0E0101781902E1040E79196A
:10A1100032E0D30E0101781902E1400E791925E0F1
:10A120000B0E0101781902E1040E791918E0D20E24
:10A130000101781902E1400E79190BE00A0E0101C4
:10A14000781902E1040E791901E027D00B0EDB6AC1
:10A1500027D0200EF36E0B0EF3CFDBFF21D0080EBD
:10A16000F36E0B0EF3CFDBFF1BD0280EF36E0B0E3E
:10A17000F3CFDBFF15D0090EF36E0B0EF3CFDBFF31
:10A180000FD00A0EF36E0B0EF3CFDBFF09D0190EC2
:10A19000F36E0B0EF3CFDBFF03D00B0EDB6A00D0A8
:10A1A000D20E0101781902E1400E79192EE0D30E8A
:10A1B0000101781902E1400E791927E00A0E010128
:10A1C000781902E1040E79191DE00B0E01017819CE
:10A1D00002E1040E791916E00C0E0101781902E172
:10A1E000040E79190FE0D00E0101781902E1400E3A
:10A1F000791908E0D10E0101781902E1400E7919B0
:10A2000001E02DD00F01030E5E6FD9500D0FE96EE6
:10A21000DACFEAFFEECFE6FFEECFE6FFEECFE6FFC6
:10A22000EFCFE6FF0B0EDBCFE6FF0D0EE66E0F0E57
:10A23000E66EF8ECAAF0146E070EE15E1450030E01
:10A240000F015E5D0BE20D0EE66E0F0EE66EAFC106
:10A25000E6FF5EEC2AF0E552E552E55206D0AFC1CA
:10A26000E6FFB9EC29F0E55200D010D0F9EC22F06D
:10A27000AFC1E6FF22EC2AF0E55208D0F9EC22F05B
:10A28000AFC1E6FF39EC2AF0E55200D0030E0F0112
:10A290005E5D05E20101786B796B0F015E6B99D011
:10A2A0004E0EE66E5FCFE6FFD5EC18F0E552E552B4
:10A2B000E76E050EE7CFDBFF050EDB5004E10F0173
:10A2C000040E5E6F02D00F015E6983D0D9500D0F6E
:10A2D000E66E000EDA20E66E5FCFE6FFC1ECAAF074
:10A2E000E552E552E552E76E050EE7CFDBFF050EBE
:10A2F000DB5002085BE1D9500D0FE96EDACFEAFFBF
:10A30000010EEE1805E1EE5003E1EE5001E1EE50D2
:10A310000EE0D9500D0FE96EDACFEAFF030EEE180A
:10A3200005E1EE5003E1EE5001E1EE500CE16D0E5F
:10A33000E66E0D0EE66E0F0EE66E69EC05F0E55268
:10A34000E552E55227D0D9500D0FE96EDACFEAFF7A
:10A35000020EEE1805E1EE5003E1EE5001E1EE5081
:10A360000EE0D9500D0FE96EDACFEAFF040EEE18B9
:10A3700005E1EE5003E1EE5001E1EE500BE1700E0D
:10A38000E66E0D0EE66E0F0EE66E69EC05F0E55218
:10A39000E552E5520D0EE66E0F0EE66EAFC1E6FF1A
:10A3A0005EEC2AF0E552E552E55207D0F9EC22F0D6
:10A3B000AFC1E6FF39EC2AF0E5520101786B796B09
:10A3C0000F015E6B06D00101786B796B0F015E6B3C
:10A3D00000D006D010EC3AF003D0040EDB6A00D0B7
:10A3E000040EDB5002E0B9EF5EF0010EF36E040ED6
:10A3F000F3CFDBFF160E0101781902E1020E791985
:10A4000002E1ABEF5EF0150E0101781902E1020ED8
:10A41000791902E172EF5EF0140E0101781902E180
:10A42000020E791902E145EF5EF0810E0101781903
:10A4300002E1210E791902E1F8EF5DF0800E0101D1
:10A44000781902E1210E791902E1F8EF5DF0100EA2
:10A450000101781902E1020E791902E1A4EF5DF021
:10A46000110E0101781902E1020E791902E1A4EF3F
:10A470005DF0130E0101781902E1020E791902E173
:10A4800097EF5DF0170E0101781902E1020E7919BC
:10A4900002E160EF5DF0120E0101781902E1020E97
:10A4A000791902E129EF5DF06C0E0101781902E1E2
:10A4B000030E791902E121EF5DF0610E01017819B7
:10A4C00002E1030E791902E11AEF5CF0650E010159
:10A4D000781902E1030E791902E11AEF5CF0690EB6
:10A4E0000101781902E1030E791902E11AEF5CF01B
:10A4F000620E0101781902E1030E791902E11AEFE7
:10A500005CF0660E0101781902E1030E791902E18F
:10A510001AEF5CF06B0E0101781902E1030E791954
:10A5200002E11AEF5CF0600E0101781902E1030EFE
:10A53000791902E1F7EF5AF0640E0101781902E18E
:10A54000030E791902E1F7EF5AF06D0E0101781947
:10A5500002E1030E791902E1F7EF5AF06E0E0101E4
:10A56000781902E1030E791902E1F7EF5AF0680E4B
:10A570000101781902E1030E791902E1F7EF5AF0AF
:10A58000630E0101781902E1030E791902E1F7EF78
:10A590005AF0670E0101781902E1030E791902E100
:10A5A000F7EF5AF06A0E0101781902E1030E7919EA
:10A5B00002E1F7EF5AF0330E0101781902E1010EC2
:10A5C000791902E1ADEF5AF0320E0101781902E17A
:10A5D000010E791902E17AEF5AF0310E0101781972
:10A5E00002E1010E791902E12FEF5AF0300E01015C
:10A5F000781902E1010E791902E1A0EF59F0010189
:10A60000785102E1130E791902E1A0EF59F0260EFC
:10A610000101781902E1010E791902E1A0EF59F068
:10A62000600E0101781902E1120E791902E1A0EF22
:10A6300059F0120E0101781902E1010E791902E1B7
:10A6400068EF59F0100E0101781902E1010E791935
:10A6500002E16BEF58F0150E0101781902E1010ECD
:10A66000791902E16BEF58F0140E0101781902E13B
:10A67000010E791902E16BEF58F0110E0101781902
:10A6800002E1010E791902E16BEF58F0130E01019E
:10A69000781902E1010E791902E16BEF58F00D0E05
:10A6A0000101781902E1010E791902E15BEF58F01E
:10A6B0000C0E0101781902E1010E791902E14BEF4C
:10A6C00058F0070E0101781902E1010E791902E133
:10A6D000DCEF57F0090E0101781902E1010E79193A
:10A6E00002E1DCEF57F00B0E0101781902E1010ED7
:10A6F000791902E1DCEF57F0060E0101781902E149
:10A70000010E791901E1EFD3080E0101781902E178
:10A71000010E791901E1E7D30A0E0101781902E16E
:10A72000010E791901E1DFD3300E0101781902E140
:10A73000020E791901E184D3310E0101781902E189
:10A74000020E791901E17CD3320E0101781902E180
:10A75000020E791901E174D3330E0101781902E177
:10A76000020E791901E16CD3340E0101781902E16E
:10A77000020E791901E164D3350E0101781902E165
:10A78000020E791901E15CD3360E0101781902E15C
:10A79000020E791901E154D3270E0101781902E163
:10A7A000020E791901E13CD32A0E0101781902E168
:10A7B000020E791901E10FD3250E0101781902E18A
:10A7C000020E791901E1F7D2260E0101781902E192
:10A7D000020E791901E1D3D2B00E0101781902E11C
:10A7E000020E791901E19FD2210E0101781902E1CF
:10A7F000010E791901E130D2170E0101781902E139
:10A80000010E791901E128D2190E0101781902E12E
:10A81000010E791901E120D2230E0101781902E11C
:10A82000010E791901E118D2250E0101781902E112
:10A83000010E791901E110D20101785102E1120EE5
:10A84000791901E18AD1600E0101781902E1110E36
:10A85000791901E182D1800E0101781902E1110E0E
:10A86000791901E17AD1200E0101781902E1120E65
:10A87000791901E172D1400E0101781902E1120E3D
:10A88000791901E16AD1200E0101781902E1010E66
:10A89000791901E1E2D0160E0101781902E1010EE9
:10A8A000791901E1DAD0180E0101781902E1010EDF
:10A8B000791901E1D2D0220E0101781902E1010ECD
:10A8C000791901E1CAD0240E0101781902E1010EC3
:10A8D000791901E1C2D00101785102E1020E791922
:10A8E00001E188D0010E0101781902E1020E791907
:10A8F0001EE0020E0101781902E1020E791917E03B
:10A90000030E0101781902E1020E791910E0040E1C
:10A910000101781902E1020E791909E0050E010121
:10A92000781902E1020E791902E0B6EF5EF0E66AEC
:10A93000E3EC2CF0E552E76E050EE7CFDBFF050EEA
:10A94000DB504AE1010E0101781902E1020E79198A
:10A9500006E1C6C1E6FFB1EC6DF0E55234D0020E5F
:10A960000101781902E1020E79190AE10101C61DFF
:10A9700001010517C6C1E6FFD3EC6DF0E55223D007
:10A98000030E0101781902E1020E791906E1C6C130
:10A99000E6FFFAEC6DF0E55216D0040E01017819CD
:10A9A00002E1020E791906E1C6C1E6FF23EC6EF062
:10A9B000E55209D00101C65101010513C6C1E6FFE8
:10A9C000D3EC6DF0E552AFC1E6FFD0EC29F0E552D3
:10A9D0000101786B796B0CD0050EDB50146E156A93
:10A9E000FF0E141801E1155003E10101786B796B3A
:10A9F000B9EF5EF00D0EE66E0F0EE66E080EE66E17
:10AA0000E1EC2BF0E552E552E552E76E050EE7CF9B
:10AA1000DBFF050EDB5013E10D0EE66E0F0EE66E4A
:10AA200068EC6CF0E552E552000905E1AFC1E6FFC4
:10AA3000D0EC29F0E5520101786B796B0CD0050E52
:10AA4000DB50146E156AFF0E141801E1155003E176
:10AA50000101786B796BB9EF5EF00D0EE66E0F0EAB
:10AA6000E66E4F0EE66E10EC2CF0E552E552E55224
:10AA7000E76E050EE7CFDBFF050EDB5060E1240E2D
:10AA80000101781902E1010E791941E0220E01015C
:10AA9000781902E1010E791931E0180E01017819D7
:10AAA00002E1010E791921E0160E0101781902E187
:10AAB000010E791911E0200E0101781902E1010E51
:10AAC000791901E02DD00D0EE66E0F0EE66ED2EC78
:10AAD0006EF0E552E55224D00D0EE66E0F0EE66ED6
:10AAE00058EC6EF0E552E5521BD00D0EE66E0F0EDF
:10AAF000E66E78EC6EF0E552E55212D00D0EE66E81
:10AB00000F0EE66E92EC6EF0E552E55209D00D0E96
:10AB1000E66E0F0EE66EB2EC6EF0E552E55200D036
:10AB20000D0EE66E0F0EE66EAFC1E6FF5EEC2AF08C
:10AB3000E552E552E5520101786B796B0CD0050EB8
:10AB4000DB50146E156AFF0E141801E1155003E175
:10AB50000101786B796BB9EF5EF00D0EE66E0F0EAA
:10AB6000E66E4F0EE66EA4EC2CF0E552E552E5528F
:10AB7000E76E050EE7CFDBFF050EDB505FE1400E11
:10AB80000101781902E1120E791940E0200E01014D
:10AB9000781902E1120E791930E0800E010178195E
:10ABA00002E1110E791920E0600E0101781902E12D
:10ABB000110E791910E00101785102E1120E791994
:10ABC00001E02DD00D0EE66E0F0EE66ED2EC6EF0AB
:10ABD000E552E55224D00D0EE66E0F0EE66E58ECEF
:10ABE0006EF0E552E5521BD00D0EE66E0F0EE66ECE
:10ABF00078EC6EF0E552E55212D00D0EE66E0F0EB7
:10AC0000E66E92EC6EF0E552E55209D00D0EE66E5E
:10AC10000F0EE66EB2EC6EF0E552E55200D00D0E6E
:10AC2000E66E0F0EE66EAFC1E6FF5EEC2AF0E5526F
:10AC3000E552E5520101786B796B0CD0050EDB50C3
:10AC4000146E156AFF0E141801E1155003E101019D
:10AC5000786B796BB9EF5EF00101AE81250E0101D1
:10AC6000781902E1010E79194DE0230E01017819DE
:10AC700002E1010E79193AE0190E0101781902E199
:10AC8000010E791927E0170E0101781902E1010E72
:10AC9000791914E0210E0101781902E1010E7919E8
:10ACA00001E03CD0A80EE66E040EE66EAFC1E6FFF2
:10ACB0005EEC2AF0E552E552E55230D0580EE66ED1
:10ACC000040EE66EAFC1E6FF5EEC2AF0E552E552F7
:10ACD000E55224D06C0EE66E040EE66EAFC1E6FFC0
:10ACE0005EEC2AF0E552E552E55218D0800EE66E91
:10ACF000040EE66EAFC1E6FF5EEC2AF0E552E552C7
:10AD0000E5520CD0940EE66E040EE66EAFC1E6FF7F
:10AD10005EEC2AF0E552E552E55200D00101786B75
:10AD2000796BB9EF5EF0040EE66E7DEC2BF0E55228
:10AD3000E76E050EE7CFDBFF050EDB5012E1080ED4
:10AD4000E66E0F0EE66EC0C1E6FFC1C1E6FFB5ECD0
:10AD500015F0E552E552E552E5520101786B796B49
:10AD60000CD0050EDB50146E156AFF0E141801E1AD
:10AD7000155003E10101786B796BB9EF5EF00101C9
:10AD8000AE810101010E0A6F440EE66E010EE66E01
:10AD9000430EE66EE66ACDEC6BF0E552E552E55205
:10ADA000E552AFC1E6FFB9EC29F0E5520101786B3D
:10ADB000796BB9EF5EF00101AE8101010A6B01010F
:10ADC000446BAFC1E6FFB9EC29F0E5520101786BA5
:10ADD000796BB9EF5EF0030EE66E7DEC2BF0E55279
:10ADE000E76E050EE7CFDBFF050EDB500BE1C0C1C0
:10ADF0000BF1AFC1E6FFB9EC29F0E5520101786B28
:10AE0000796B0CD0050EDB50146E156AFF0E14180A
:10AE100001E1155003E10101786B796BB9EF5EF048
:10AE20000101AE81E668F6EC76F0E552AFC1E6FFCF
:10AE3000D0EC29F0E5520101786B796BB9EF5EF047
:10AE40000101AE81360E0101781902E1020E791975
:10AE50003DE0350E0101781902E1020E791933E067
:10AE6000340E0101781902E1020E791929E0330E3E
:10AE70000101781902E1020E79191FE0320E010179
:10AE8000781902E1020E791915E0310E01017819E5
:10AE900002E1020E79190BE0300E0101781902E18E
:10AEA000020E791901E015D0CEEC6FF012D0E8EC6B
:10AEB0006FF00FD00BEC70F00CD02EEC70F009D0CE
:10AEC00051EC70F006D074EC70F003D097EC70F099
:10AED00000D0AFC1E6FFD0EC29F0E5520101786B5C
:10AEE000796BB9EF5EF00D0EE66E0F0EE66E4F0E4B
:10AEF000E66EE1EC2BF0E552E552E552E76E050E09
:10AF0000E7CFDBFF050EDB5049E10A0E010178199E
:10AF100002E1010E791929E0080E0101781902E118
:10AF2000010E791915E0060E0101781902E1010EF2
:10AF3000791901E027D00D0EE66E0F0EE66E80EC5B
:10AF40002DF0E552E552E76E050EE7CFDBFF1AD094
:10AF50000D0EE66E0F0EE66E9FEC2DF0E552E552FB
:10AF6000E76E050EE7CFDBFF0DD00D0EE66E0F0E80
:10AF7000E66EC2EC2DF0E552E552E76E050EE7CF26
:10AF8000DBFF00D0050EDB5005E1AFC1E6FFD0ECE2
:10AF900029F0E5520101786B796B0CD0050EDB507E
:10AFA000146E156AFF0E141801E1155003E101013A
:10AFB000786B796BB9EF5EF00D0EE66E0F0EE66EF4
:10AFC0004F0EE66EE1EC2BF0E552E552E552E76EEE
:10AFD000050EE7CFDBFF050EDB504FE10B0E010145
:10AFE000781902E1010E791929E0090E0101781999
:10AFF00002E1010E791915E0070E0101781902E14D
:10B00000010E791901E027D00D0EE66E0F0EE66EE7
:10B0100075EC2FF0E552E552E76E050EE7CFDBFF4A
:10B020001AD00D0EE66E0F0EE66E95EC2FF0E5527F
:10B03000E552E76E050EE7CFDBFF0DD00D0EE66E95
:10B040000F0EE66EB2EC2FF0E552E552E76E050EFC
:10B05000E7CFDBFF00D0050EDB500BE10D0EE66EF7
:10B060000F0EE66EAFC1E6FF5EEC2AF0E552E55248
:10B07000E5520101786B796B0CD0050EDB50146E34
:10B08000156AFF0E141801E1155003E10101786BF8
:10B09000796BB9EF5EF00101AE81DEECAEF0000934
:10B0A00005E1AFC1E6FFD0EC29F0E5520101786B74
:10B0B000796BB9EF5EF00101AE8181ECAFF0000970
:10B0C00005E1AFC1E6FFD0EC29F0E5520101786B54
:10B0D000796BB9EF5EF00D0EE66E0F0EE66E070EA1
:10B0E000E66EE1EC2BF0E552E552E552E76E050E17
:10B0F000E7CFDBFF050EDB5001E0DCD00B0EDB6A97
:10B100000D0EE66E0F0EE66E7AECADF0E552E552EE
:10B110000C0EF3CFDBFF0C0EDB50F36E0B0EDBCF10
:10B12000F4FFF350F45C20E20B0EDB50EA6A0D0FE3
:10B13000E96E0F0EEA22EFCF16F0176A16BE1768F7
:10B1400016C0E6FF17C0E6FFD5EC17F0E552E55252
:10B15000F3CF14F0F4CF15F01450151002E0050EE3
:10B16000DB680B0EDB2AD7D7050EDB50146E156A91
:10B17000FF0E141801E1155071E0130E010178194A
:10B1800002E1010E79195DE0110E0101781902E169
:10B19000010E791949E0150E0101781902E1010E3D
:10B1A00079192FE0140E0101781902E1010E7919C5
:10B1B00015E0100E0101781902E1010E791901E084
:10B1C0004DD00D0EE66E0F0EE66EC4EC85F0E55226
:10B1D000E552E76E050EE7CFDBFF40D001010051DD
:10B1E0000DE10D0EE66E0F0EE66E05EC86F0E552F3
:10B1F000E552E76E050EE7CFDBFF02D0050EDB68F8
:10B200002DD001018F510DE00D0EE66E0F0EE66E92
:10B2100005EC86F0E552E552E76E050EE7CFDBFF61
:10B2200002D0050EDB681AD00D0EE66E0F0EE66E2C
:10B230004BEC86F0E552E552E76E050EE7CFDBFFFB
:10B240000DD00D0EE66E0F0EE66E2FEC86F0E55279
:10B25000E552E76E050EE7CFDBFF00D0050EDB50B1
:10B26000146E156AFF0E141801E115501FE0050E4B
:10B27000DBCFE6FFE66A3F0EE66E640EE66E010E79
:10B28000E66E0D0EE66E0F0EE66E31ECBAF0146E41
:10B29000070EE15E14500D0EE66E0F0EE66EAFC1A6
:10B2A000E6FF5EEC2AF0E552E552E5520101786BCB
:10B2B000796B0CD0050EDB50146E156AFF0E141856
:10B2C00001E1155003E10101786B796BB9EF5EF094
:10B2D0000D0EE66E0F0EE66E020EE66EE1EC2BF042
:10B2E000E552E552E552E76E050EE7CFDBFF050EAE
:10B2F000DB5018E10D0EE66E0F0EE66E87ECB4F033
:10B30000E552E552F350E66E73EC86F0E552000923
:10B3100005E0AFC1E6FFD0EC29F0E5520101786B02
:10B32000796B0CD0050EDB50146E156AFF0E1418E5
:10B3300001E1155003E10101786B796BB9EF5EF023
:10B340000101785102E1130E791926E0600E010126
:10B35000781902E1120E79191FE0300E01017819F7
:10B3600002E1010E791908E0260E0101781902E1C7
:10B37000010E791901E020D00D0EE66E0F0EE66E7B
:10B380004F0EE66E10EC2CF0E552E552E552E76EFA
:10B39000050EE7CFDBFF10D00D0EE66E0F0EE66E4A
:10B3A0004F0EE66EA4EC2CF0E552E552E552E76E46
:10B3B000050EE7CFDBFF00D0050EDB5042E1260E85
:10B3C0000101781902E1010E791922E0600E0101F4
:10B3D000781902E1120E79191BE0300E010178197B
:10B3E00002E1010E791907E00101785102E1130E23
:10B3F000791901E01AD00D0EE66E0F0EE66EC5EC5F
:10B4000014F0E552E552E76E050EE7CFDBFF0DD0F5
:10B410000D0EE66E0F0EE66E05EC6FF0E552E5528E
:10B42000E76E050EE7CFDBFF00D0050EDB5005E130
:10B43000AFC1E6FFD0EC29F0E5520101786B796BE2
:10B440000CD0050EDB50146E156AFF0E141801E1C6
:10B45000155003E10101786B796BB9EF5EF00D0EC9
:10B46000E66E0F0EE66E030EE66EE1EC2BF0E55293
:10B47000E552E552E76E050EE7CFDBFF050EDB5028
:10B480002BE10D0EE66E0F0EE66E0D0EE66E0F0E44
:10B49000E66E87ECB4F0E552E552F3CF14F0F4CF4A
:10B4A00015F014C0E6FF15C0E6FF4EEC15F0E552AE
:10B4B000E552E552E55200090BE10D0EE66E0F0E66
:10B4C000E66EAFC1E6FF5EEC2AF0E552E552E552CA
:10B4D0000101786B796B0CD0050EDB50146E156A88
:10B4E000FF0E141801E1155003E10101786B796B2F
:10B4F000B9EF5EF00D0EE66E0F0EE66E4F0EE66EC5
:10B50000E1EC2BF0E552E552E552E76E050EE7CF90
:10B51000DBFF050EDB5013E10D0EE66E0F0EE66E3F
:10B5200007EC15F0E552E552000905E1AFC1E6FF71
:10B53000D0EC29F0E5520101786B796B0CD0050E47
:10B54000DB50146E156AFF0E141801E1155003E16B
:10B550000101786B796BB9EF5EF00D0EE66E0F0EA0
:10B56000E66E4F0EE66EE1EC2BF0E552E552E55249
:10B57000E76E050EE7CFDBFF050EDB502BE10D0E6E
:10B58000E66E0F0EE66E0D0EE66E0F0EE66E87ECA3
:10B59000B4F0E552E552F3CF14F0F4CF15F014C037
:10B5A000E6FF15C0E6FF8FEC15F0E552E552E552D7
:10B5B000E55200090BE10D0EE66E0F0EE66EAFC10F
:10B5C000E6FF5EEC2AF0E552E552E5520101786BA8
:10B5D000796B0CD0050EDB50146E156AFF0E141833
:10B5E00001E1155003E10101786B796BC2D3010EC3
:10B5F000E66E7DEC2BF0E552E76E050EE7CFDBFF44
:10B60000050EDB5001E009D10101080EC05D000EFE
:10B61000C15901E3FED00A0E0101C025E96E090EF1
:10B620000101C121EA6EEF500101C06FC16B010E33
:10B63000C0C1E7FFE75204E0E846FE0BE706FCE185
:10B64000E76E0B0EE7CFDBFFC0C1E6FF53EC21F046
:10B65000E552E76E0C0EE7CFDBFF6A0E01017819A9
:10B6600002E1030E791901E1C9D0670E01017819D1
:10B6700002E1030E791901E1B1D0630E01017819DD
:10B6800002E1030E791901E199D0680E01017819E0
:10B6900002E1030E791901E187D0640E01017819E6
:10B6A00002E1030E79194BE06E0E0101781902E1F7
:10B6B000030E791944E0600E0101781902E1030ECE
:10B6C000791908E06D0E0101781902E1030E79196C
:10B6D00001E09FD00B0EDB5001016D13600E0101E4
:10B6E000781902E1030E791905E10B0EDB1C01014B
:10B6F0006F1704D00B0EDB5001016F13050EF36EB4
:10B700000C0EDBCFF4FFF350F45C13E20C0EDB50B5
:10B71000050DF3CF14F0F4CF15F0880E1426060EA5
:10B72000152214C0E6FF15C0E6FF3BEC80F0E552A1
:10B73000E552AFC1E6FFB9EC29F0E5526AD00B0E35
:10B74000DB5001016E13640E0101781902E1030E52
:10B75000791905E10B0EDB1C01016F1704D00B0EEC
:10B76000DB5001016F13050EF36E0C0EDBCFF4FFFF
:10B77000F350F45C13E20C0EDB50050DF3CF14F024
:10B78000F4CF15F0880E1426060E152214C0E6FF1D
:10B7900015C0E6FF3BEC80F0E552E552AFC1E6FF95
:10B7A000B9EC29F0E55235D00B0EDB5001017013D6
:10B7B000AFC1E6FFB9EC29F0E5522BD0C0C1E6FFDE
:10B7C000D5EC32F0E552C0C1E6FF13EC33F0E552A0
:10B7D000AFC1E6FFD0EC29F0E5521BD0C0C1E6FFB7
:10B7E000F3EC32F0E552C0C1E6FF13EC33F0E55262
:10B7F000AFC1E6FFD0EC29F0E5520BD0C0C1E6FFA7
:10B8000031EC33F0E552AFC1E6FFD0EC29F0E55260
:10B8100000D00101786B796B0CD0050EDB50146EF3
:10B82000156AFF0E141801E1155003E10101786B50
:10B83000796B9FD2010EE66E7DEC2BF0E552E76E40
:10B84000050EE7CFDBFF050EDB5001E0EDD0010177
:10B85000080EC05D000EC15901E3E2D00A0E0101DD
:10B86000C025E96E090E0101C121EA6EEF50010108
:10B87000C06FC16B010EC0C1E7FFE75204E0E846AC
:10B88000FE0BE706FCE1E76E0B0EE7CFDBFFC0C166
:10B89000E6FF53EC21F0E552E76E0C0EE7CFDBFF3D
:10B8A0000F0109511AE00F010C51146E156A145062
:10B8B000800B01E1A9D0980E0F01091501E0A4D079
:10B8C0000A0E0101C025E96E090E0101C121EA6ECF
:10B8D000EF500101AF5D01E097D00F01010E5D6FE8
:10B8E0006B0E0101781902E1030E791901E185D08F
:10B8F000660E0101781902E1030E791901E177D092
:10B90000620E0101781902E1030E79196AE0690EED
:10B910000101781902E1030E791959E0650E010160
:10B92000781902E1030E79192DE0610E01017819F1
:10B9300002E1030E791901E066D00B0EDB1C010158
:10B940006D17050EF36E0C0EDBCFF4FFF350F45CB5
:10B9500013E20C0EDB50050DF3CF14F0F4CF15F00D
:10B96000880E1426060E152214C0E6FF15C0E6FF49
:10B970003BEC80F0E552E552AFC1E6FFB9EC29F0AF
:10B98000E55241D00B0EDB1C01016E17050EF36E64
:10B990000C0EDBCFF4FFF350F45C13E20C0EDB5023
:10B9A000050DF3CF14F0F4CF15F0880E1426060E13
:10B9B000152214C0E6FF15C0E6FF3BEC80F0E5520F
:10B9C000E552AFC1E6FFB9EC29F0E5521CD00B0EF1
:10B9D000DB1C01017017AFC1E6FFB9EC29F0E5529D
:10B9E00012D0C0C1E6FF00EC32F0E5520CD0C0C16D
:10B9F000E6FF47EC32F0E55206D0C0C1E6FF8EEC20
:10BA000032F0E55200D00CD009CFE6FFAFC1E6FF1F
:10BA1000FEEC29F0E552E5520101AE93F9EC22F07B
:10BA20000101786B796B0CD0050EDB50146E156A32
:10BA3000FF0E141801E1155003E10101786B796BD9
:10BA400098D10101AE8151EC33F00101786B796B33
:10BA500090D10D0EE66E0F0EE66E080EE66EE1EC6E
:10BA60002BF0E552E552E552E76E050EE7CFDBFF1E
:10BA7000050EDB5018E10D0EE66E0F0EE66EA1EC22
:10BA800082F0E552E552E76E050EE7CFDBFF050ECB
:10BA9000DB5005E1AFC1E6FFB9EC29F0E552010149
:10BAA000786B796B0CD0050EDB50146E156AFF0EA7
:10BAB000141801E1155003E10101786B796B59D13C
:10BAC0000D0EE66E0F0EE66E0A0EE66EE1EC2BF042
:10BAD000E552E552E552E76E050EE7CFDBFF050EB6
:10BAE000DB5018E10D0EE66E0F0EE66E0BEC83F0E8
:10BAF000E552E552E76E050EE7CFDBFF050EDB50A2
:10BB000005E1AFC1E6FFB9EC29F0E5520101786B20
:10BB1000796B0CD0050EDB50146E156AFF0E1418ED
:10BB200001E1155003E10101786B796B22D101012C
:10BB3000AE8189EC83F0AFC1E6FFB9EC29F0E552A4
:10BB40000101786B796B15D10D0EE66E0F0EE66E66
:10BB50000A0EE66EE1EC2BF0E552E552E552E76E97
:10BB6000050EE7CFDBFF050EDB5035E1110E0101BD
:10BB7000781902E1020E791915E0100E0101781909
:10BB800002E1020E791901E01AD00D0EE66E0F0ED9
:10BB9000E66EC7EC83F0E552E552E76E050EE7CF9F
:10BBA000DBFF0DD00D0EE66E0F0EE66E27EC84F077
:10BBB000E552E552E76E050EE7CFDBFF00D0050E3C
:10BBC000DB5005E1AFC1E6FFD0EC29F0E552010101
:10BBD000786B796B0CD0050EDB50146E156AFF0E76
:10BBE000141801E1155003E10101786B796BC1D0A4
:10BBF000010EE66E7DEC2BF0E552E76E050EE7CF09
:10BC0000DBFF050EDB5034E1800E0101781902E103
:10BC1000210E791915E0810E0101781902E1210E3A
:10BC2000791901E019D0010EE66EC0C1E6FF60ECA3
:10BC300084F0E552E552E76E050EE7CFDBFF0CD04E
:10BC4000E66AC0C1E6FF60EC84F0E552E552E76EBB
:10BC5000050EE7CFDBFF00D0050EDB5005E1AFC1DD
:10BC6000E6FFB9EC29F0E5520101786B796B0CD055
:10BC7000050EDB50146E156AFF0E141801E1155005
:10BC800003E10101786B796B74D0010EE66E7DECF7
:10BC90002BF0E552E76E050EE7CFDBFF050EDB501C
:10BCA00014E10101050EC05D000EC1590AE2C0C1D8
:10BCB000E6FF69EC3BF0E552AFC1E6FFB9EC29F0D5
:10BCC000E5520101786B796B0CD0050EDB50146ED8
:10BCD000156AFF0E141801E1155003E10101786B9C
:10BCE000796B47D0010EE66E7DEC2BF0E552E76EE6
:10BCF000050EE7CFDBFF050EDB5020E1010100510F
:10BD0000146E156A01011450C05D1550C15912E23C
:10BD10000A0E0101C025E96E090E0101C121EA6E7A
:10BD2000EF50E66E84EC3BF0E552AFC1E6FFB9ECB4
:10BD300029F0E5520101786B796B0CD0050EDB50D0
:10BD4000146E156AFF0E141801E1155003E101018C
:10BD5000786B796B0ED03FEC3BF0AFC1E6FFB9ECEE
:10BD600029F0E5520101786B796B03D0040EDB6A90
:10BD700000D0040EDB5002E02DEF68F0010EF36EF0
:10BD8000040EF3CFDBFFFE0E0101781902E1E86833
:10BD9000791902E123EF68F0760E0101781902E1CA
:10BDA000030E791902E1F8EF67F0610E01017819CD
:10BDB00002E1370E791902E1F8EF67F0770E010121
:10BDC000781902E1030E791902E1F8EF67F0710EBC
:10BDD0000101781902E1370E791902E1F8EF67F0F5
:10BDE000750E0101781902E1030E791902E1E8EFFD
:10BDF00067F0850E0101781902E1030E791902E15D
:10BE00001DEF67F0860E0101781902E1030E791922
:10BE100002E11DEF67F09D0E0101781902E1020EAB
:10BE2000791902E1E8EF66F09C0E0101781902E150
:10BE3000020E791902E1D7EF66F09B0E0101781925
:10BE400002E1020E791902E1CAEF66F09A0E0101D1
:10BE5000781902E1020E791902E196EF66F0990E67
:10BE60000101781902E1020E791902E18BEF66F007
:10BE7000980E0101781902E1020E791902E148EFEA
:10BE800066F0600E0101781902E1020E791902E1F3
:10BE900045EF66F0210E0101781902E1020E7919D1
:10BEA00002E1E7EF65F0220E0101781902E1020ECE
:10BEB000791902E1E7EF65F0290E0101781902E135
:10BEC000020E791902E1E7EF65F0200E0101781901
:10BED00002E1020E791902E1C0EF65F0190E0101CD
:10BEE000781902E1020E791902E19EEF65F0240E45
:10BEF0000101781902E1020E791902E19BEF65F068
:10BF0000230E0101781902E1020E791902E123EFF3
:10BF100065F0710E0101781902E1030E791902E151
:10BF2000C3EF64F0700E0101781902E1030E791974
:10BF300002E161EF64F03A0E0101781902E1010EAD
:10BF4000791902E13FEF64F0390E0101781902E13D
:10BF5000010E791902E118EF64F00101785102E154
:10BF6000010E791902E1FCEF63F0010E010178196D
:10BF700002E1010E791902E1D4EF63F0050E01012F
:10BF8000781902E1010E791902E1C4EF63F0030EA2
:10BF90000101781902E1010E791901E1E5D3040EDE
:10BFA0000101781902E1010E791901E1CDD3020EE8
:10BFB0000101781902E1010E791901E1B5D3450EAD
:10BFC0000101781902E1030E791901E103D3460E4C
:10BFD0000101781902E1030E791901E1FBD2440E47
:10BFE0000101781902E1030E791901E1F3D2500E33
:10BFF0000101781902E1020E791901E1EBD2510E2B
:10C000000101781902E1020E791901E1E3D2530E20
:10C010000101781902E1020E791901E1DBD2410E2A
:10C020000101781902E1030E791901E171D2420E82
:10C030000101781902E1030E791901E169D2400E7C
:10C040000101781902E1030E791901E161D2520E62
:10C050000101781902E1020E791901E159D2540E59
:10C060000101781902E1020E791901E151D2380E6D
:10C070000101781902E1010E791901E142D2370E6E
:10C080000101781902E1010E791901E132D2360E6F
:10C090000101781902E1010E791901E122D2350E70
:10C0A0000101781902E1010E791901E112D2340E71
:10C0B0000101781902E1010E791901E1FCD1060EA6
:10C0C0000101781901E1795101E1E7D1040E010183
:10C0D000781901E1795101E1A2D1170E0101781916
:10C0E00001E1795101E175D1160E0101781901E1E3
:10C0F000795101E154D1150E0101781901E179510D
:10C1000001E11DD1140E0101781901E1795101E11C
:10C11000E1D0130E0101781901E1795101E1CED08E
:10C12000120E0101781901E1795101E1BBD0110E24
:10C130000101781901E1795101E1A8D0100E010146
:10C14000781901E1795101E195D0070E01017819C3
:10C1500001E1795101E182D0050E0101781901E177
:10C16000795170E0020E0101781901E1795162E024
:10C17000340E0101781902E1030E79191DE0350E24
:10C180000101781902E1030E791916E0030E01018D
:10C19000781901E1795110E03C0E0101781902E1B2
:10C1A000030E791909E03D0E0101781902E1030E31
:10C1B000791902E02AEF68F00101AE813D0E01011C
:10C1C000781902E1030E791928E03C0E0101781973
:10C1D00002E1030E79191EE0030E0101781901E155
:10C1E000795115E0350E0101781902E1030E791934
:10C1F0000BE0340E0101781902E1030E791901E018
:10C200000FD03DEC27F00CD062EC27F009D00101F3
:10C210007A6B06D0E7EC35F003D0F2EC35F000D0C5
:10C22000AFC1E6FFB9EC29F0E5520101786B796BFB
:10C230002DEF68F00101786B796B0101010E7A6FC7
:10C240002DEF68F00101AE81AFC1E6FFB3EC28F03D
:10C25000E5520101786B796B2DEF68F00101AE8139
:10C26000AFC1E6FFA8EC29F0E5520101786B796BCC
:10C270002DEF68F00101AE81AFC1E6FF00EC29F0BF
:10C28000E5520101786B796B2DEF68F00101AE8109
:10C29000AFC1E6FF45EC29F0E5520101786B796BFF
:10C2A0002DEF68F00101AE81AFC1E6FF58EC29F037
:10C2B000E5520101786B796B2DEF68F00101AE81D9
:10C2C000AFC1E6FF6BEC29F0E5520101786B796BA9
:10C2D0002DEF68F0010EE66E7DEC2BF0E552E76E77
:10C2E000050EE7CFDBFF050EDB501BE1010100511E
:10C2F000146E156A01011450C05D1550C1590DE24C
:10C30000200EE66EC0C1E6FFD5EC18F0E552E5520E
:10C31000AFC1E6FFB9EC29F0E5520101786B796B0A
:10C320000CD0050EDB50146E156AFF0E141801E1D7
:10C33000155003E10101786B796B2DEF68F0010E68
:10C34000E66E7DEC2BF0E552E76E050EE7CFDBFFE6
:10C35000050EDB5016E101010051146E156A010152
:10C360001450C05D1550C15908E2C0C1E6FFAFC10D
:10C37000E6FF7EEC29F0E552E5520101786B796B1E
:10C380000CD0050EDB50146E156AFF0E141801E177
:10C39000155003E10101786B796B2DEF68F0010115
:10C3A000AE810D0EE66E0F0EE66EFDECB9F0E552B5
:10C3B000E5520D0EE66E0F0EE66EAFC1E6FF5EECC7
:10C3C0002AF0E552E552E5520101786B796B2DEFC9
:10C3D00068F00101AE8192EC86F0E66EE66A7E0EB0
:10C3E000E66E650EE66E010EE66E0D0EE66E0F0E43
:10C3F000E66E31ECBAF0146E070EE15E14500D0ECD
:10C40000E66E0F0EE66EAFC1E6FF5EEC2AF0E55277
:10C41000E552E5520101786B796B2DEF68F001016F
:10C42000AE810101886BE66AE66AE8EC05F0E55248
:10C43000E552E66A010EE66EE8EC05F0E552E552DB
:10C44000E66A020EE66EE8EC05F0E552E552E66AB1
:10C45000030EE66EE8EC05F0E552E552E66A040EDE
:10C46000E66EE8EC05F0E552E552E66A050EE66E8A
:10C47000E8EC05F0E552E552E66A060EE66EE8ECF9
:10C4800005F0E552E552AFC1E6FFD0EC29F0E552E8
:10C490000101786B796B2DEF68F00101AE8101012C
:10C4A000876BAFC1E6FFD0EC29F0E5520101786B54
:10C4B000796B2DEF68F00101AE810101776BAFC19F
:10C4C000E6FFB9EC29F0E5520101786B796B2DEFAD
:10C4D00068F00601030EFF6F0101786B796B2DEF99
:10C4E00068F00601010EFF6F0101786B796B2DEF8B
:10C4F00068F00601020EFF6F0101786B796B2DEF7A
:10C5000068F00601FF690101786B796B2DEF68F027
:10C510000101AE81540E0101781902E1020E791970
:10C5200047E0520E0101781902E1020E79193BE051
:10C53000400E0101781902E1030E791928E0420E3C
:10C540000101781902E1030E791914E0410E01018D
:10C55000781902E1030E791901E02FD0E66AAFC124
:10C56000E6FF5FEC34F0E552E552E76E0B0EE7CFE5
:10C57000DBFF23D0010EE66EAFC1E6FF5FEC34F0C7
:10C58000E552E552E76E0B0EE7CFDBFF16D0AFC1E9
:10C59000E6FFC0EC34F0E552E76E0B0EE7CFDBFFB1
:10C5A0000B0EDB6A0AD035EC37F00B0EDB6A05D0D8
:10C5B0000101AB6B0B0EDB6A00D00B0EDB5005E10B
:10C5C000AFC1E6FFB9EC29F0E5520101786B796B58
:10C5D0002DEF68F0010EE66E7DEC2BF0E552E76E74
:10C5E000050EE7CFDBFF050EDB5001E08FD0010128
:10C5F0000051146E156A01011450C05D1550C159E7
:10C6000001E380D00A0E0101C025E96E090E010187
:10C61000C121EA6EEF500101C06FC16B530E0101E1
:10C62000781902E1020E79195BE0510E01017819C7
:10C6300002E1020E79194AE0500E0101781902E177
:10C64000020E791939E0440E0101781902E1030E56
:10C65000791928E0460E0101781902E1030E7919D3
:10C6600014E0450E0101781902E1030E791901E089
:10C6700041D0E66AC0C1E6FF5FEC34F0E552E55216
:10C68000E76E0B0EE7CFDBFF35D0010EE66EC0C1C3
:10C69000E6FF5FEC34F0E552E552E76E0B0EE7CFB4
:10C6A000DBFF28D0C0C1E6FFC0EC34F0E552E76EF6
:10C6B0000B0EE7CFDBFF1ED0C0C1E6FFFEEC36F06D
:10C6C000E552E76E0B0EE7CFDBFF14D0C0C1E6FFEB
:10C6D00019EC37F0E552E76E0B0EE7CFDBFF0AD01F
:10C6E000C0C1E6FF52EC37F0E552E76E0B0EE7CF24
:10C6F000DBFF00D00B0EDB5005E1AFC1E6FFB9EC6C
:10C7000029F0E5520101786B796B0CD0050EDB50F6
:10C71000146E156AFF0E141801E1155003E10101B2
:10C72000786B796B2DEF68F00101AE8109EC6CF04C
:10C73000000905E1AFC1E6FFD0EC29F0E5520101A7
:10C74000786B796B2DEF68F00101AE8117EC6CF01E
:10C75000000905E1AFC1E6FFD0EC29F0E552010187
:10C76000786B796B2DEF68F00101AE8126EC6CF0EF
:10C77000000905E1AFC1E6FFD0EC29F0E552010167
:10C78000786B796B2DEF68F00101AE8130EC6CF0C5
:10C79000000905E1AFC1E6FFD0EC29F0E552010147
:10C7A000786B796B2DEF68F00101AE8134EC7CF091
:10C7B00000090FE0370EE66E640EE66E010EE66EBF
:10C7C000AFC1E6FF6CEC2AF0E552E552E552E552C6
:10C7D0000ED02D0EE66E640EE66E010EE66EAFC153
:10C7E000E6FF6CEC2AF0E552E552E552E552010114
:10C7F000786B796B2DEF68F00101AE8101018F51EB
:10C8000012E00101746B74C1E6FF550EE66E030E73
:10C81000E66E90EC6BF0E552E552E552AFC1E6FFF3
:10C82000D0EC29F0E5520101786B796B2DEF68F0BF
:10C83000020EE66E7DEC2BF0E552E76E050EE7CFBB
:10C84000DBFF050EDB500EE1C0C1E6FF48EC6EF0E9
:10C85000E552AFC1E6FFD0EC29F0E5520101786B5B
:10C86000796B0CD0050EDB50146E156AFF0E141890
:10C8700001E1155003E10101786B796BEED34F0EA6
:10C88000E66EE66AFD0EE66E630EE66E010EE66E7D
:10C890000D0EE66E0F0EE66E2DECAEF0146E070E6A
:10C8A000E15E14500D0EE66E0F0EE66EAFC1E6FFB0
:10C8B0005EEC2AF0E552E552E5520101786B796BA6
:10C8C000CCD30D0EE66E0F0EE66E040EE66EE1ECB6
:10C8D0002BF0E552E552E552E76E050EE7CFDBFFA0
:10C8E000050EDB5043E1300E0F010D5D146E080E96
:10C8F000145C1EE20E0EE66E0F0EE66E87ECB4F0D0
:10C90000E552E552F350E66E300E0F010D5DEA6A16
:10C910000A0FE96E090EEA22EF50E66EEDEC37F0F1
:10C92000E552E552AFC1E6FFB9EC29F0E5521AD065
:10C93000300E0F010D5D080815E10E0EE66E0F0EAC
:10C94000E66E87ECB4F0E552E552F350E66E080E61
:10C95000E66EEDEC37F0E552E552AFC1E6FFB9EC1B
:10C9600029F0E5520101786B796B0CD0050EDB5094
:10C97000146E156AFF0E141801E1155003E1010150
:10C98000786B796B6AD30D0EE66E0F0EE66E030EB2
:10C99000E66EE1EC2BF0E552E552E552E76E050E4E
:10C9A000E7CFDBFF050EDB5041E1300E0F010D5DDF
:10C9B000146E080E145C1DE2300E0F010F5DE66E62
:10C9C000300E0F010E5DE66E300E0F010D5DEA6A4E
:10C9D0000A0FE96E090EEA22EF50E66E2DEC38F0F0
:10C9E000E552E552E552AFC1E6FFB9EC29F0E55258
:10C9F00019D0300E0F010D5D080814E1300E0F0143
:10CA00000F5DE66E300E0F010E5DE66E080EE66EEF
:10CA10002DEC38F0E552E552E552AFC1E6FFB9EC36
:10CA200029F0E5520101786B796B0CD0050EDB50D3
:10CA3000146E156AFF0E141801E1155003E101018F
:10CA4000786B796B0AD30D0EE66E0F0EE66E050E4F
:10CA5000E66EE1EC2BF0E552E552E552E76E050E8D
:10CA6000E7CFDBFF050EDB5059E10D0EE66E0F0E32
:10CA7000E66E7AECADF0E552E552F3CF14F0F4CF68
:10CA800015F0020ED8801454000E155447E2300EF3
:10CA90000F010D5D146E080E145C1DE20F0EE66EA4
:10CAA0000F0EE66E87ECB4F0E552E552F350E66EF9
:10CAB000300E0F010E5DE66E300E0F010D5DE66E5D
:10CAC00011EC39F0E552E552E552AFC1E6FFD0EC8A
:10CAD00029F0E5521FD0300E0F010D5D08081AE154
:10CAE0000F0EE66E0F0EE66E87ECB4F0E552E552DF
:10CAF000F350E66E300E0F010E5DE66E080EE66E28
:10CB000011EC39F0E552E552E552AFC1E6FFD0EC49
:10CB100029F0E5520101786B796B0CD0050EDB50E2
:10CB2000146E156AFF0E141801E1155003E101019E
:10CB3000786B796B92D23EEC39F08FD2010EE66EB3
:10CB40007DEC2BF0E552E76E050EE7CFDBFF050E1F
:10CB5000DB5009E1C0C1E6FF0BEC24F0E552010116
:10CB6000786B796B0CD0050EDB50146E156AFF0ED6
:10CB7000141801E1155003E10101786B796B6DD256
:10CB8000010EE66E7DEC2BF0E552E76E050EE7CF69
:10CB9000DBFF050EDB500EE1C0C1E6FF49EC24F0DF
:10CBA000E552AFC1E6FFB9EC29F0E5520101786B1F
:10CBB000796B0CD0050EDB50146E156AFF0E14183D
:10CBC00001E1155003E10101786B796B46D2070E44
:10CBD000E66E7DEC2BF0E552E76E050EE7CFDBFF4E
:10CBE000050EDB5045E1290E0101781902E1020E24
:10CBF00079192EE0220E0101781902E1020E79194D
:10CC000018E0210E0101781902E1020E791901E004
:10CC10002BD00101A00EC05D0F0EC15909E2C0C1A9
:10CC20005DF1C1C15EF1AFC1E6FFB9EC29F0E5529B
:10CC30001BD00101FF0ED880C055000EC15507E37F
:10CC4000C0C15FF1AFC1E6FFB9EC29F0E5520CD0ED
:10CC5000C0C1E6FFC1C1E6FFAFC1E6FF50EC2AF05C
:10CC6000E552E552E55200D00101786B796B0CD0AA
:10CC7000050EDB50146E156AFF0E141801E11550F5
:10CC800003E10101786B796BE8D144EC3CF0E5D12C
:10CC9000010EE66E7DEC2BF0E552E76E050EE7CF58
:10CCA000DBFF050EDB502AE10101080EC05D000E1E
:10CCB000C15920E2460EE66E0D0EE66EA3EC00F0C2
:10CCC000E552E55206C09AF107C09BF108C09CF1FD
:10CCD00009C09DF1010EC0C1E7FFE75204E0E8463C
:10CCE000FE0BE706FCE10101996FAFC1E6FFB9EC6D
:10CCF00029F0E5520101786B796B0CD0050EDB5001
:10CD0000146E156AFF0E141801E1155003E10101BC
:10CD1000786B796BA2D10101996BAFC1E6FFB9ECD9
:10CD200029F0E5520101786B796B97D1010EE66E1F
:10CD3000E3EC2CF0E552E76E050EE7CFDBFF050EC6
:10CD4000DB501BE1460EE66E0D0EE66EA3EC00F026
:10CD5000E552E55206C09FF107C0A0F108C0A1F15D
:10CD600009C0A2F1C6C19EF1AFC1E6FFB9EC29F03E
:10CD7000E5520101786B796B0CD0050EDB50146E17
:10CD8000156AFF0E141801E1155003E10101786BDB
:10CD9000796B63D10101AE8101019E6BAFC1E6FFEA
:10CDA000B9EC29F0E5520101786B796B56D101019C
:10CDB000AE810801B46B0801B36B0801B96BAFC158
:10CDC000E6FFB9EC29F0E5520101786B796B45D1AA
:10CDD0000101AE81B40EE66E080EE66E2A0EE66E16
:10CDE000030EE66ECDEC6BF0E552E552E552E552EE
:10CDF000B30EE66E080EE66E290EE66E030EE66EC4
:10CE0000CDEC6BF0E552E552E552E552B90EE66E17
:10CE1000080EE66E2F0EE66E030EE66ECDEC6BF09E
:10CE2000E552E552E552E552AFC1E6FFB9EC29F013
:10CE3000E5520101786B796B10D10101AEB102D0DE
:10CE40000F015E6B0F015E51020A01E1A2D0020ADE
:10CE500001E0BDD0860E0101781902E1030E7919B7
:10CE60001AE0850E0101781902E1030E791901E03B
:10CE700025D0E66A0D0EE66E0F0EE66E110EE66E1A
:10CE800091EC2AF0E552E552E552E552E76E050EC7
:10CE9000E7CFDBFF13D071C1E6FF0D0EE66E0F0E7C
:10CEA000E66E110EE66E14EC2BF0E552E552E552FB
:10CEB000E552E76E050EE7CFDBFF00D0050EDB5035
:10CEC00059E10DCF16F0176A16BE176816C0E6FFB7
:10CED00017C0E6FFC3EC17F0E552E552F3CF14F0AC
:10CEE000F4CF15F01450151006E0300E0F010D5D53
:10CEF0000F015F6F02D00F015F69080E0F015F5DC8
:10CF000009E20F015F51EA6A0A0FE96E090EEA228F
:10CF1000EFCF5FFF010100510F015F5D26E2010EBF
:10CF20005FCFE7FFE75204E0E846FE0BE706FCE1CF
:10CF3000146EB4C1E9FFB5C1EAFF020EEB50141440
:10CF400014E001016D5101016E11156E010E5FCFEC
:10CF5000E7FFE75204E0E846FE0BE706FCE11514A4
:10CF600004E10F01020E5E6F04D00101786B796B52
:10CF70002ED00FD0050EDB50146E156AFF0E14185C
:10CF800001E1155005E10101786B796B20D001D0EA
:10CF90001ED0250EE66E5FCFE6FF20EC19F0E552BD
:10CFA000E552F35013E10E0EE66E0F0EE66E5FCF04
:10CFB000E6FFAAEC7FF0E552E552E552AFC1E6FF8D
:10CFC000B9EC29F0E5520101786B796B00D045D0BE
:10CFD0000101AE81A388A38A0201010EFF6FAFC1D8
:10CFE000E6FFB9EC29F0E5520101786B796B35D099
:10CFF0000D0EE66E0F0EE66E78C1E6FF79C1E6FF14
:10D0000094EC3BF0E552E552E552E552E76E050E31
:10D01000E7CFDBFF050EDB5009E1AFC1E6FFB9EC5E
:10D0200029F0E5520101786B796B0CD0050EDB50CD
:10D03000146E156AFF0E141801E1155003E1010189
:10D04000786B796B0AD00101AE81FF000101786B2A
:10D05000796B03D0040EDB6A00D0040EDB5007E1CD
:10D060000101786B796B0101AE6BF9EC22F00101E3
:10D07000AEA10DD00101785101E1795101E006D056
:10D080000101B35102E10101AE9100D009D00101CB
:10D090007851791105E10701000E646F070E656F85
:10D0A000010E0101AE1508E10101B35105E10701CF
:10D0B000005102E0A2EF3CF0070100510EE1010E29
:10D0C0000101AE150AE10601FE5107E1030E01015F
:10D0D000B31503E10101010E756F130EE15C02E26D
:10D0E000E16AE552E16EE552E7CFD9FF12008FEC1D
:10D0F00087F00B0EE1263BEC88F0070E06C0DBFF45
:10D10000080E07C0DBFF090E08C0DBFF0A0E09C0CE
:10D11000DBFF0101995114E09AEC8DF09A51EE5C1D
:10D12000146E9B51EE58156E9C51EE58166E9D5123
:10D13000EE58176ED8802C0EFCEC8DF001E2996B46
:10D140009E5111E09AEC8DF09F51EE5C146EA0514F
:10D15000EE58156EA151EE58166EA251EE58A8EC7D
:10D160008AF001E29E6B0051DDEC8FF0D7EC8AF083
:10D170008DEC8AF003E09EEC8BF0FDE17EEC89F013
:10D1800000C1DFFFDF5001E18AD151EC91F00101D4
:10D190007A5106E037EC90F0EF9E060EDB6A77D10D
:10D1A0004DEC93F003E1D0EC96F00EE15DEC8DF0E8
:10D1B00002E0000E01D0010E15148B03F31C146E57
:10D1C000D0EC96F0141439E0010EF36E060EF3CF96
:10D1D000DBFFDB5011E02FEC95F0EF1C146E030E1B
:10D1E000DB50B015141408E02FEC95F0EFCF15F0DC
:10D1F000941DB015151421E0E1EC87F040EC8EF0A1
:10D2000011E104511915156E03511815011115106E
:10D21000146ED0EC96F0141405E14DEC8AF036C192
:10D22000EFFF0DD0E1EC87F0090E60EC8FF0E66EB9
:10D230004DEC8AF052EC89F002D0060EDB6A060E45
:10D24000DB5011E15DEC8DF002E0000E01D0010E2B
:10D2500015148B03F3CF14F0D0EC96F0F31403E025
:10D260004DEC8AF0EF6A060EDB5071E1030EDB50E5
:10D2700099156DE1E1EC87F0C8EC95F0DF0B41E129
:10D28000B3511EE0010EDB50765D3BE00A5118E021
:10D29000AC5116E14DEC93F013E1010EDB5003E1CC
:10D2A000080EAF5D2EE02FEC95F034EC8EF076C1D9
:10D2B000E7FFE75203E071EC8AF0FDE1141421E18D
:10D2C0000101A95128E0BDEC96F001510211E5528F
:10D2D000E71421E02FEC95F0EFCF16F0010E76C1A8
:10D2E000E7FFE75203E071EC8AF0FDE1156E080EEE
:10D2F0000101AF5D02E0000E01D0010E1510161401
:10D300000AE00101A5512B11E81C176E030EDB503A
:10D31000031517141CE02FEC95F0EFCF18F01DEC5F
:10D320008FF003E071EC8AF0FDE1181407E0030EC2
:10D330000101AE1503E04DEC93F009E0E1EC87F05C
:10D340001FEC97F0220B0CE04DEC93F009E02CEC75
:10D350008FF006E1E1EC87F00A0E42EC94F01BD06E
:10D36000E1EC87F060EC8FF0010B08E02CEC8FF023
:10D3700005E14DEC8AF0EF500EE107D04DEC8AF05C
:10D38000EF5003E02CEC8FF006E0E1EC87F00A0EA2
:10D39000C0EC87F0EF6A030EDB500801B91505E118
:10D3A000030EDB1C0801F11751D0C8EC8DF004E02E
:10D3B000010E0801BB1503E1060EDB5015E1030E5B
:10D3C000DB1C0801F117B7C8E6FFB8C8E6FF010E7D
:10D3D0003EEC89F0B80E1426000EC8EC87F065EC20
:10D3E00000F0E552E55230D048EC8EF0B80E16262B
:10D3F000000EB6EC96F07DEC95F028E1030EDB50C4
:10D400000801F113030EDB50010103151FE0040EA8
:10D410000801BB151BE0030EDB1C0101A517030E61
:10D42000DB5027159413D0EC88F0CBEC95F05AEC38
:10D4300092F092EC8AF002E1000E151807E0020E5D
:10D440008FEC8FF03BEC80F0E552E552E1EC87F099
:10D450000A0E60EC8FF006E1E1EC87F060EC8FF0F3
:10D46000010B12E0030EDB500801F1150DE1010183
:10D470006D516E11146E030EDB506F15141404E120
:10D4800037EC90F0EF8E03D037EC90F0EF9ED95050
:10D49000040F60EC88F0030EE3EC91F073D60B0EF2
:10D4A000E15C02E2E16AE552E16E94EF87F08AEC1A
:10D4B0008FF000C1DFFFDF501BE051EC91F0010164
:10D4C0001E510DE037EC90F0EF50800B08E018ECA7
:10D4D0008EF048C1EFFF37EC90F0EF8C07D018ECDE
:10D4E0008EF0EF5003E137EC90F0EF9CDF06E3D7CE
:10D4F000020EE15C02E2E16AE552E16E94EF87F030
:10D50000F3EC8BF0300EAFEF8AF0F3EC8BF0310ED2
:10D51000AFEF8AF068EC96F001012E512F1138E040
:10D520000801E05113E046EC96F0DC5DEE50DD5969
:10D53000EE50DE59EE50DF5909E20101AE5107010C
:10D54000001104E10801E06BDBDF22D00801E651A5
:10D550001FE1C8EC8DF002E1A7511AE00801010EAD
:10D56000E06F2EC114F02FC115F01EEC8EF02EC10D
:10D5700006F02FC107F0ABEC90F00801DC6FEE5025
:10D580000320DD6FEE500420DE6FEE500520DF6FCC
:10D5900001012C512D1138E00801E55113E046EC52
:10D5A00096F0E15DEE50E259EE50E359EE50E45949
:10D5B00009E20101AE510701001104E10801E56B28
:10D5C000A4DF22D00801E6511FE1C8EC8DF002E192
:10D5D000A7511AE00801010EE56F2CC114F02DC10E
:10D5E00015F01EEC8EF02CC106F02DC107F0ABEC4F
:10D5F00090F00801E16FEE500320E26FEE5004203E
:10D60000E36FEE500520E46F0801BC51BD1109E045
:10D61000420EE66E0D0EE66E7DEC95F002E1010124
:10D62000AB6BC8EC8DF00801E66F0101A76B040E2F
:10D63000E15C02E2E16AE552E16E94EF87F08AEC88
:10D640008FF0829A8394FE0EDB50020B020802E0F8
:10D65000000E01D0010EE8B08386E8A08396838493
:10D660008394FE0EDB50010BE8B08386E8A083961E
:10D6700083848394DE52800EDD6E080EDF6EDF50F1
:10D6800017E0D0EC88F0FD0EA6EC94F0146E010EBD
:10D69000DB50145C02E0000E01D0010EE8B083867E
:10D6A000E8A0839683848394010EE3EC91F0E7D79E
:10D6B000828A020EE15C02E2E16AE552E16E94EFD9
:10D6C00087F095969594949A1200939693929390DE
:10D6D00093941200F00EC1140709C16E0F0E971437
:10D6E000976E98909690969299961200D4EC05F0C9
:10D6F0003CECA1F0EADFE5DFC7EC00F043EC0EF014
:10D7000068ECB0F06AEF6BF055EC92F007E144EC96
:10D7100088F0FA0EDBCFE6FFDAEC91F094EF87F0B9
:10D7200055EC92F005E1D95090EC93F0DAEC91F0E1
:10D7300094EF87F055EC92F005E1D950D8EC8DF0DC
:10D74000DAEC91F094EF87F055EC92F005E1D950C6
:10D75000DEEC8DF0DAEC91F094EF87F055EC92F07E
:10D760000CE144EC88F044EC88F0DCEC90F004EC44
:10D7700096F0C4EC87F0EEEC8BF094EF87F08FEC32
:10D7800087F032EC91F0FA0EDBCFE6FFC4EC87F0C5
:10D7900065EC89F0F6E094EF87F08FEC87F032ECDF
:10D7A00091F0010EF1EC92F0FAE094EF87F08FEC3B
:10D7B00087F032EC91F0020EF1EC92F0FAE094EF87
:10D7C00087F08FEC87F032EC91F0040EF1EC92F0E0
:10D7D000FAE094EF87F08FEC87F032EC91F044ECB4
:10D7E00088F088EC88F0F3CF15F0F4CF16F0010E36
:10D7F000F324C1EC96F0E66A31ECA3F0176E060E46
:10D80000E15E1750E552E7CF14F0145CE6E094EFC8
:10D8100087F034EC7CF0000909E04FEC8FF09BECD2
:10D820008AF04FEC8FF0F4EC8AF0000C010C010E42
:10D830009EEC8DF00AE04FEC8FF0E66AE66EE66A49
:10D840006C0EE66EF4EC8AF0000C010C010E9EECFE
:10D850008DF005E04FEC8FF0E66A56EF95F0010C85
:10D86000020E9EEC8DF006E04FEC8FF0E66A6C0E37
:10D8700056EF95F0010CD8EC8FF0D950010F8CECDD
:10D8800090F00A0EEE6E090EED6E080EDF6EDF50A0
:10D8900013E045EC8AF001E3DB2AEF50E66E010E5F
:10D8A000DBCFE9FFDB2A020EDBCFEAFF01E3DB2A55
:10D8B00052EC89F0DF06EBD7D5EC8CF030EC88F039
:10D8C000030EE15C02E2E16AE552E16E94EF87F05B
:10D8D0008FEC87F00B0EE126ABEC91F00CE045EC01
:10D8E00091F016BE1768C6EC94F005E0C0EC8BF022
:10D8F000F3E3DB2AF1D7DF6A080EDF5C56E2ABEC1C
:10D9000091F053E0ABEC91F0D00FE66ED950020FDE
:10D91000146EDF500F011424EAEC8AF052EC89F007
:10D920009BEC8CF01424EAEC8AF0EF50070807E235
:10D930009BEC8CF01424EAEC8AF0070EEF6E010EDB
:10D94000DB6ADF500DEC89F01BE2D950020F156E37
:10D95000DACF16F0DF501524EAEC8AF0EFCF14F09E
:10D96000D950020F176EDACF18F0010EDB501724D2
:10D97000EAEC8AF0EF50145C56E0010EDB2AE1D7A6
:10D98000C0EC8BF001E3DB2AABEC91F00CE045EC52
:10D9900091F016BE1768C6EC94F005E0C0EC8BF071
:10D9A000F3E3DB2AF1D7DF2AA7D7080EDF5C48E2D2
:10D9B0000A0EDB68010EDB6ADF500DEC89F020E215
:10D9C000D950020F156EDACF16F0010EDB50152478
:10D9D000EAEC8AF0EF50176E010E175204E0E846A9
:10D9E000FE0B1706FCE1E81C146E0A0EDBCFE7FF06
:10D9F0001450E7160A0EE7CFDBFF010EDB2ADCD757
:10DA0000DE52080EDD6E010EDB5009E00A0EDB501F
:10DA100006E00A0EC7EC89F0010EDB06F4D7010E12
:10DA2000DB50080802E1010E11D09BEC8CF00F01D5
:10DA30001424EAEC8AF0010EDBCFEFFFDF2AB5D722
:10DA400091EC95F018DFE552E552000E146E0B0EC6
:10DA5000E15C02E2E16AE552E16E145094EF87F076
:10DA600001C1E6FF010E5CEC8FF002C1E6FF020E81
:10DA70005CEC8FF003C1E6FF030E5CEC8FF004C199
:10DA8000E6FF040E5CEC8FF005C1E6FF050E5CEFCF
:10DA90008FF015EC95F0DBCF01F1A2EC8CF00317C1
:10DAA00017EF92F015EC95F0DBCF02F1FE0EDB1CC8
:10DAB00001010117FE0EDB1C031717EF92F015ECA6
:10DAC00095F0DBCF03F1A2EC8CF0011717EF92F089
:10DAD00015EC95F0DBCF04F1A2EC8CF00317FE0EF1
:10DAE000DB1C0117BDDF94EF87F08AEC8FF0DF6A53
:10DAF000050EDF5C2EE2A4EC95F0DF5059EC90F0BF
:10DB0000A0EC87F018EC96F0010101510211E552EA
:10DB1000E714A4EC8DF0E712AAEC94F018EC96F060
:10DB200003510411E552E714E81CA4EC8DF0E7164C
:10DB3000AAEC94F0DBCFE6FFDF5059EC90F0A4ECB8
:10DB400087F0FEEC94F0EE52010EDBCFEFFFDF2A00
:10DB5000CFD7020EE15C02E2E16AE552E16E94EF9A
:10DB600087F0CBEC8FF0BAEC8EF0040EDBCF04F133
:10DB70008CEC8CF0E710E66E8CDF4BEC88F003E069
:10DB800071EC8AF0FDE167EC88F0050EDF5C03E2E2
:10DB900053EC8FF0FAD785EC8AF002E2E16AE552A5
:10DBA000E16E94EF87F0CBEC8FF0010EDBCF01F14B
:10DBB000030EDBCF03F1040EDBCF04F1FE0E88EC85
:10DBC0008DF0E710E66E6EDF4BEC88F003E071EC51
:10DBD0008AF0FDE167EC88F0050EDF5C03E253ECB0
:10DBE0008FF0FAD785EC8AF002E2E16AE552E16E45
:10DBF00094EF87F0CBEC8FF0020EDBCF02F1010E39
:10DC0000DBCF01F1040EDBCF04F118EC96F0030E2C
:10DC1000DB50E552E710E66E52DF4BEC88F003E094
:10DC200071EC8AF0FDE167EC88F0050EDF5C03E241
:10DC300053EC8FF0FAD785EC8AF002E2E16AE55204
:10DC4000E16E94EF87F0CBEC8FF0BAEC8EF0010E22
:10DC5000DBCF01F118EC96F0040EDB50E552E71033
:10DC6000E66E36DF4BEC88F003E071EC8AF0FDE104
:10DC700067EC88F0050EDF5C03E253EC8FF0FAD717
:10DC800085EC8AF002E2E16AE552E16E94EF87F0FA
:10DC900015EC95F0DBCFD1F8D1C8E6FFF40E5CECC3
:10DCA0008FF0D1C8E6FFEEEC02F0E55294EF87F07A
:10DCB0001EEC90F00BE2C4EC87F0580EE66E040EFA
:10DCC00039EC89F0F4EC92F0B2EC88F094EF87F044
:10DCD0002CEC91F00BE25CEC88F0580EE66E040E32
:10DCE0002EEC89F0F4EC92F0B2EC88F094EF87F02F
:10DCF0001EEC90F008E2C4EC87F044EC8EF039ECB6
:10DD000089F0DEEC93F094EF87F02CEC91F008E2D0
:10DD10005CEC88F044EC8EF02EEC89F0DEEC93F0B5
:10DD200094EF87F01EEC90F00BE2C4EC87F0800ECD
:10DD3000E66E040E39EC89F0FAEC92F0B2EC88F061
:10DD400094EF87F02CEC91F00BE25CEC88F0800E05
:10DD5000E66E040E2EEC89F0FAEC92F0B2EC88F04C
:10DD600094EF87F01EEC90F00BE2C4EC87F0940E79
:10DD7000E66E040E39EC89F000EC93F0B2EC88F01A
:10DD800094EF87F02CEC91F00BE25CEC88F0940EB1
:10DD9000E66E040E2EEC89F000EC93F0B2EC88F005
:10DDA00094EF87F0B9EC96F0E66EE66AC4EC87F083
:10DDB0003BEC91F029EC93F010EC8BF030EC88F018
:10DDC00094EF87F08FEC87F05CEC88F0A80EE66E9D
:10DDD000040E2EEC89F010EC8BF030EC88F094EF10
:10DDE00087F0A0EC95F00FE2060E50EC8BF0FE0EE3
:10DDF000DB507AEC8FF0FFECADF0166E060EE15EB4
:10DE0000165001EC95F094EF87F02DEC92F0ABEC0E
:10DE100091F00CE045EC91F016BE1768C6EC94F05A
:10DE200005E0C0EC8BF0F3E3DB2AF1D7DEEC8AF0FF
:10DE30001EEC92F0E1EC87F0A2EC8BF016BE1768B6
:10DE4000F5EC94F00AE0E1EC87F0EF5006E0040E08
:10DE5000DB2A050EEFE3DB2AEDD7E1EC87F0EF508C
:10DE600010E0040EDBCFE9FFDB2A050EDBCFEAFF73
:10DE700001E3DB2AEF6AC4EC87F0FFEC95F0B5EC28
:10DE800089F0ABEC91F00CE045EC91F016BE176810
:10DE9000C6EC94F005E0C0EC8BF0F3E3DB2AF1D79D
:10DEA000CBEC88F0080EEE5C000E13EC8AF015E265
:10DEB000DFEC8CF0EFCF14F0080E145C0EE2ABEC4C
:10DEC00091F00BE077EC94F0DFEC8CF0EF50E66E25
:10DED00088DFBAEC8FF0000E01D0010E146E060E32
:10DEE000E15C02E2E16AE552E16E145094EF87F0E2
:10DEF000A0EC95F00DE2060E17EC8CF0FE0EDB5058
:10DF00007AEC8FF02DECAEF084EC94F001EC95F00F
:10DF100094EF87F015EC95F0DB50EA6A4D0FE96E4F
:10DF2000010EE9EC8CF04B0F5CEC8FF094EF87F076
:10DF300015EC95F0DB50EA6A550FE96E010EE9EC3D
:10DF40008CF0530F5CEC8FF094EF87F015EC95F0AC
:10DF5000D5EC8FF0FD0EDBCFEFFFFE0E6FEC95F0F2
:10DF6000C7EC8CF0FEEC96F00E0E04EC96F0A4ECF0
:10DF700087F094EF87F015EC95F0C7EC96F0FD0E66
:10DF8000DBCFEFFFFE0EC7EC96F0EF50C7EC8CF046
:10DF900059EC90F0A4EC87F094EF87F049EC91F005
:10DFA0008FEC92F0DF6A080EDF5C0EE25EEC92F01E
:10DFB000480EE926080EEA22E9C6EEFFEAC6EEFFA1
:10DFC000EBC6EEFFDF2AEFD732EC96F028EF90F0A9
:10DFD00049EC91F0EC0EE66E060EE66E1A0EE0ECE1
:10DFE00090F0080EDF5C0EE25EEC92F0300EE92657
:10DFF000080EEA22ECC6EEFFEDC6EEFFEEC6EEFF1F
:10E00000DF2AEFD7180EE66E300EE66E080EE66ECB
:10E010001D0E28EF90F049EC91F0EF0EE66E060E23
:10E02000E66E350EE0EC90F0080EDF5C0EE25EEC82
:10E0300092F0180EE926080EEA22EFC6EEFFF0C6AF
:10E04000EEFFF1C6EEFFDF2AEFD7180EE66E180ED0
:10E05000E66E080EE66E380E28EF90F049EC91F06F
:10E06000F20EE66E060EE66E500EE0EC90F0080E34
:10E07000DF5C0EE25EEC92F0000EE926080EEA226A
:10E08000F2C6EEFFF3C6EEFFF4C6EEFFDF2AEFD7CF
:10E09000180EE66E000EE66E080EE66E530E28EFC2
:10E0A00090F049EC91F0F50EE66E060EE66E6B0E02
:10E0B000E0EC90F0080EDF5C0EE25EEC92F0A10E58
:10E0C000E926060EEA22F5C6EEFFF6C6EEFFF7C613
:10E0D000EEFFDF2AEFD7180EE66EA10EE66E060EF3
:10E0E000E66E6E0E28EF90F049EC91F0F80EE66EB9
:10E0F000060EE66E860EE0EC90F0080EDF5C0EE297
:10E100005EEC92F0D10EE926060EEA22F8C6EEFF8A
:10E11000F9C6EEFFFAC6EEFFDF2AEFD7180EE66E5D
:10E12000D10EE66E060EE66E890E28EF90F049ECF1
:10E1300091F0FD0EE66E0D0EE66EB60EE0EC90F080
:10E14000080EDF5C0EE25EEC92F0B90EE926060ED8
:10E15000EA22FDCDEEFFFECDEEFFFFCDEEFFDF2A82
:10E16000EFD7180EE66EB90EE66E060EE66EB90E25
:10E1700028EF90F0E66A570E15EC88F09BEC8AF0D9
:10E18000E66A79ECA2F048EF89F0B6EC8FF0010175
:10E19000080E006FE66E9BEC8AF0A4EC87F001019C
:10E1A000056B066B06C1E6FF430E64EC8FF00101C0
:10E1B0000269010EE66E6DDCE552E66A80DCE5522E
:10E1C000E66A86DCE552FE0E01010211E66E6ADCAB
:10E1D000E5520101021D076FE66E4B0E64EC8FF0F5
:10E1E00001016D6B6DC1E6FF18EC8BF0A4EC87F0BC
:10E1F00001016E6B6EC1E6FFB9EC8DF0A4EC87F007
:10E2000001016F6B6FC1E6FF4A0E64EC8FF00101F4
:10E21000706B70C1E6FFBCEC8DF0A4EC87F00101DF
:10E22000440E716FE66E400E64EC8FF00101726B6C
:10E2300072C1E6FF470E64EC8FF00101736B73C18E
:10E24000E6FF480E64EC8FF0E668E66A94EC8BF02B
:10E25000E668E66A99EC8BF0E66A010EE66E94ECED
:10E260008BF0E66A010EE66E99EC8BF0E66A020E20
:10E27000E66E94EC8BF0E66A020EE66E99EC8BF09B
:10E28000040EDF6EDF5002080CE2E66ADFCFE6FF25
:10E2900094EC8BF0E66ADFCFE6FF99EC8BF0DF06BB
:10E2A000F1D7F30EE66E080EE66E3BEC6CF0E5522D
:10E2B000E5520101010E086FE66E270E5CEC8FF04F
:10E2C0000101030E096FE66E280E5CEC8FF0010170
:10E2D000010E0A6FE66E290E5CEC8FF00101010E53
:10E2E0000B6FE66E360E64EC8FF001010C6B0CC107
:10E2F000E6FF370E64EC8FF00101030E0D6FE66E42
:10E30000B80E82EC8FF00101030E0E6FE66E350E33
:10E3100064EC8FF00101020E0F6FE66E2A0E5CECCA
:10E320008FF00101010E106FE66E2B0E5CEC8FF08A
:10E330000101116B11C1E6FFC00E82EC8FF00101EB
:10E34000126B12C1E6FF380E64EC8FF00101136B03
:10E3500013C1E6FFC10E82EC8FF00101146B14C1F2
:10E36000E6FF390E64EC8FF00101156B15C1E6FF75
:10E37000C20E82EC8FF00101166916C1E6FF3A0E5B
:10E3800064EC8FF00101176B17C1E6FF440E64ECDB
:10E390008FF00101186918C1E6FF3B0E64EC8FF0A5
:10E3A0000101196919C1E6FF3C0E64EC8FF001010F
:10E3B0001A6B1AC1E6FFC30E82EC8FF001011B6BD2
:10E3C0001BC1E6FF2C0E5CEC8FF00101010E1C6FEF
:10E3D000E66E2D0E5CEC8FF00101010E1D6FE66EF6
:10E3E0002E0E5CEC8FF00101010E1E6FE66E2F0EFB
:10E3F0005CEC8FF001012A6B2AC1E6FFB90E82ECBA
:10E400008FF001012B6B2BC1E6FF420E64EC8FF005
:10E41000DF6A080EDF5C0DE2DF50EA6ABE0FE96ECC
:10E42000080EEA22EF6AC8EC8EF0200EEF6EDF2AAB
:10E43000F0D761EC8CF030EC88F06AEC8CF030ECCA
:10E4400088F001011F691FC1E6FF300E5CEC8FF000
:10E450000101010E206FE66E310E5CEC8FF00101C0
:10E46000130E216FE66EA20E82EC8FF00101100EEA
:10E47000226FE66EA30E82EC8FF00101170E236F60
:10E48000E66EA40E82EC8FF00101130E246FE66E8F
:10E49000A50E82EC8FF00101130E256FE66EA60E1D
:10E4A00082EC8FF00101266926C1E6FF4C0E64EC78
:10E4B0008FF00101276927C1E6FF3E0E64EC8FF063
:10E4C0000101286928C1E6FF490E64EC8FF00101C3
:10E4D000296B29C1E6FF3F0E64EC8FF0DF6A080E5E
:10E4E000DF5C07E2E66A7AEC93F0A4EC87F0DF2ABF
:10E4F000F6D701012C6B2D6B2CC1E6FF2DC1E6FF79
:10E50000BC0EDFEC94F0CBEC87F0780E01012E6F9F
:10E510002F6BE66E2FC1E6FFBE0EDFEC94F0CBEC66
:10E5200087F00101010E306F31EC8FF0A4EC87F021
:10E5300001010C0E316FE66E330E5CEC8FF00101C1
:10E54000010E326FE66E340E5CEC8FF001010C0EA2
:10E55000336FE66E350E5CEC8FF00101140E346FF4
:10E56000E66E3D0E64EC8FF00101280E356FE66E0D
:10E57000360E5CEC8FF00101366B36C1E6FF370ECC
:10E580005CEC8FF001010F0E376FE66E380E5CEC1D
:10E590008FF0780E0801BC6FBD6BE66EBDC8E6FF5C
:10E5A000450E06EC91F00101960E386FE66E390EBD
:10E5B0005CEC8FF00101010E396FE66ED40E82EC37
:10E5C0008FF01E0E01013B6F3C6BE66E3CC1E6FF17
:10E5D0003A0E0AEC91F0780E01013D6F3E6BE66E4B
:10E5E0003EC1E6FF3C0E0AEC91F00101580E3F6F70
:10E5F000020E406F3FC1E6FFE66E3E0E0AEC91F060
:10E60000010E0101416F426BE66E42C1E6FF400E12
:10E610000AEC91F00101140E436FE66E420E5CECC1
:10E620008FF00101020E446FE66E430E5CEC8FF03A
:10E6300001010A0E456FE66E440E5CEC8FF001019D
:10E64000320E466FE66E450E5CEC8FF001010F0E48
:10E65000476FE66E410E64EC8FF00101486948C1D6
:10E66000E6FF460E5CEC8FF00101030E3A6FE66E9A
:10E67000B70E82EC8FF00801580EAE6F020EAF6F2E
:10E68000AEC8E6FFE66E240E06EC91F00801100E0F
:10E69000B06F0E0EB16FB0C8E6FFE66E260E06EC48
:10E6A00091F00801030EB26FE850E66EE66A280E9C
:10E6B00006EC91F00801010EB56FE66E2B0E64ECCE
:10E6C0008FF00801FE0EB66FE66E2C0E64EC8FF034
:10E6D000B40E0801B76FB86BE66EB8C8E6FF2D0E32
:10E6E00006EC91F00801BA6BBAC8E6FF300E64EC94
:10E6F0008FF00801030EBB6FE66E310E64EC8FF0F5
:10E700000801B36BB3C8E6FF290E64EC8FF0080173
:10E71000B46BB4C8E6FF2A0E64EC8FF00801B96B45
:10E72000B9C8E6FF2F0E64EC8FF001010A0E496FA5
:10E73000E66E470E5CEC8FF001011E0E4B6FE66E2D
:10E74000480E5CEC8FF001010A0E4A6FE66E490E2E
:10E750005CEC8FF00101010E4C6FE66E4A0E5CEC32
:10E760008FF00801200ECE6F030ECF6FCEC8E6FFEC
:10E77000E66EF10E0AEC91F00D017F0E1D6F120E88
:10E78000E66E48EC6EF0E5520801D26BD2C8E6FFA7
:10E79000F50E5CEC8FF00801D36BD3C8E6FFF60EE4
:10E7A0005CEC8FF00801280ED46F040ED56FD4C82E
:10E7B000E6FFE66EF70E0AEC91F008013C0ED66F0C
:10E7C000E66EF90E5CEC8FF00801140ED76FE66E62
:10E7D000FA0E5CEC8FF00801280ED86F040ED96F8A
:10E7E000D8C8E6FFE66EFB0E0AEC91F008011E0E9B
:10E7F000DA6FE66EFD0E5CEC8FF00801180EDB6F31
:10E80000E66EFE0E5CEC8FF0CFEC8EF068EC6EF0F6
:10E81000BAEC8FF0CFEC8EF085EC6EF0F2EC8CF071
:10E82000A2EC6EF0F2EC8CF0C2EC6EF0BAEC8FF071
:10E83000E90EE66E630EE66E010EE66EE2EC6EF039
:10E84000BAEC8FF0DF6A080EDF5C0DE2E80EE66ED0
:10E85000630EE66E010E4EEC8CF078EC6FF0FBEC84
:10E8600096F0DF2AF0D70101020E696FE66E9C0E6A
:10E8700082EC8FF001016A6B6AC1E6FF230E64EC43
:10E880008FF001016B6B6BC1E6FF9D0E82EC8FF088
:10E8900001016C69E4EC93F0060EE66EE66AE10EA7
:10E8A000E66E630EE66E010E9AEC96F0DAEC8BF0F3
:10E8B0000D01686B010EDF6E140EDF5C05E266EC85
:10E8C0008DF0EF6ADF2AF8D78C0E7FEC90F030ECF9
:10E8D00088F00D01010E616FE66EF00E5CEC8FF0BA
:10E8E0000601E96BEA6B9BEC8AF0FF0E0AEC91F0F3
:10E8F0000601640EEB6F0AEC88F0E66EA4EC87F07C
:10E90000120E0601EC6FED6BE66EE66A1A0EC3ECB2
:10E910008FF00601640EEE6FE66E1C0EC7EC8FF0F2
:10E92000110E0601EF6FF06BE66EE66A350EC3EC72
:10E930008FF00601640EF16FE66E370EC7EC8FF0B4
:10E94000130E0601F26FF36BE66EE66A500EC3EC2F
:10E950008FF00601640EF46FE66E520EC7EC8FF076
:10E960001C0E0601F56FF66BE66EE66A6B0EC3ECE5
:10E970008FF00601640EF76FE66E6D0EC7EC8FF038
:10E98000180E0601F86FF96BE66EE66A860EC3ECA8
:10E990008FF00601500EFA6FE66E880EC7EC8FF00E
:10E9A000160E0101FA6FFB6BE66EE66AA10EC3EC70
:10E9B0008FF00101400EFC6FE66EA30EC7EC8FF0E6
:10E9C0000101FD6BFE6B9BEC8AF0A40EC3EC8FF093
:10E9D00001017F0EFF6FE66EA60EC7EC8FF01A0ED8
:10E9E0000D01EE6FEF6BE66EE66AA70EC3EC8FF0DB
:10E9F0000D01A00EF06FE66EA90EC7EC8FF01B0E96
:10EA00000D01F16FF26BE66EE66AAA0EC3EC8FF0B1
:10EA10000D01960EF36FE66EAC0EC7EC8FF0300E64
:10EA20000D01F46FF56BE66EE66AAD0EC3EC8FF088
:10EA30000D01780EF66FE66EAF0EC7EC8FF0270E65
:10EA40000D01F76FF86BE66EE66AB00EC3EC8FF05F
:10EA50000D01780EF96FE66EB20EC7EC8FF0310E35
:10EA60000D01FA6FFB6BE66EE66AB30EC3EC8FF036
:10EA70000D01790EFC6FE66EB50EC7EC8FF00D013F
:10EA8000010EFD6F100EFE6F010EE66E100EE66EAB
:10EA9000B60EC3EC8FF00D015A0EFF6FE66EB80E86
:10EAA000E3EC94F0240E08016C6F6D6BE66EE66A81
:10EAB000DD0EC3EC8FF00801A00E6E6FE66EDF0E68
:10EAC000C7EC8FF0210E08016F6F706BE66EE66A7F
:10EAD000E00EC3EC8FF00801A00E716FE66EE20E3F
:10EAE000C7EC8FF0230E0801666F676BE66EE66A6F
:10EAF000D70EC3EC8FF008017F0E686FE66ED90E5B
:10EB0000C7EC8FF00801696B6A6B9BEC8AF0DA0E38
:10EB1000C3EC8FF00801640E6B6FE66EDC0EE3EC65
:10EB200094F00801900E636F410E646F900EE66ED4
:10EB3000410EE66ED40EC3EC8FF008017F0E656FB8
:10EB4000E66ED60EC7EC8FF0230E0801726F736B62
:10EB5000E66EE66A1D0E06EC91F008017F0E746FFA
:10EB6000E66E1F0E64EC8FF00801756B766B9BEC04
:10EB70008AF0200E06EC91F008017F0E776FE66EAA
:10EB8000220E64EC8FF0250E0601FB6FFC6BE66E27
:10EB9000E66A320E06EC91F006017F0EFD6FE66E1E
:10EBA000340E64EC8FF001015A0E606FE66EBB0EFE
:10EBB00082EC8FF0CEEC6FF0E8EC6FF00BEC70F0C5
:10EBC0002EEC70F051EC70F074EC70F097EC70F08B
:10EBD00000010A0EE06FE16BE26BE36BE66E4BEC5B
:10EBE0008FF0C40ED6EC90F00001640EE46FE56B7C
:10EBF000E66BE76BE66E4BEC8FF0C80ED6EC90F050
:10EC00000001E80EE86F030EE96FEA6BEB6BE80EAC
:10EC100015EC88F0E66AE66ACC0ED6EC90F00001BE
:10EC2000880EEC6F130EED6FEE6BEF6B880EE66ED9
:10EC3000130EE66EE66AE66AD00ED6EC90F001019D
:10EC4000070E746FE66E550E64EC8FF0080EDF6EE3
:10EC5000DF5017E07F0EE66EE66ADF045CEC89F0B9
:10EC60007F0E0AEC88F0DF04EAEC93F0DF045CEC42
:10EC700089F0760E15EC88F0DF045CEC89F0DF0695
:10EC8000E7D77F0EE66EE66A080E5CEC89F07F0E31
:10EC90000AEC88F0080EEAEC93F0080E5CEC89F0C0
:10ECA000760E15EC88F0080E5CEC89F06DECABF09C
:10ECB000E55294EF87F08FEC87F0080EBDEC8CF0F6
:10ECC000040F6AEC95F0E66AB0EC87F0800EFBEC7E
:10ECD0008BF0080EDF6EDF504CE051EC91F011EC40
:10ECE00089F0040EA6EC94F002E0010E17D011ECAE
:10ECF00089F0050EA6EC94F002E0020E0FD011ECA4
:10ED000089F0060EA6EC94F002E0040E07D011EC98
:10ED100089F0070EA6EC94F005E0080EF36E030EE2
:10ED2000F3CFDBFF33EC90F0EE52030EDBCFEFFFBF
:10ED3000DB50040A13E00C0A11E0090A07E0030A99
:10ED400014E1020EDB500101061508E133EC90F0EE
:10ED5000090EC0EC87F035C1EFFF07D033EC90F01F
:10ED6000090EC0EC87F036C1EFFF020EE3EC91F024
:10ED7000B2D7080EE15C02E2E16AE552E16E94EF7F
:10ED800087F08FEC87F0FD0EDB500801B51504E02D
:10ED9000FE0EDB50B31303D0FE0EDB1CB317FD0ECB
:10EDA000DB50B61504E0FE0EDB50B41303D0FE0EAC
:10EDB000DB1CB417FD0EDB50BA1504E0FE0EDB5071
:10EDC000B91303D0FE0EDB1CB91794EF87F0B3C85C
:10EDD000E6FF290E64EC8FF0B4C8E6FF2A0E64EC5F
:10EDE0008FF0B9C8E6FF2F0E64EF8FF0D8EC8FF0EC
:10EDF00062DF800EFBEC8BF0080EDF6EDF5065E00B
:10EE0000FE0E88EC8DF0E7145CE051EC91F0DB50E5
:10EE1000A8EC87F0EE52EF50080A48E00A0A12E028
:10EE2000060A09E0050A4DE1AFEC91F0600E5DECD9
:10EE30008BF0010E40D0AFEC91F0400E5DEC8BF00A
:10EE4000040E39D0020EDB50010105150AE0020E56
:10EE5000DB1C6C17F0EC91F0EF6E100EE66E020EFC
:10EE60001BD054EC8AF04AC1EFFF5BEC8AF04CC136
:10EE7000EFFF205102E1000E01D0010E200DF350F2
:10EE80004009E66E010E7AEC88F052EC89F0020E31
:10EE9000DB506C13020EE66EDBCFE6FF72DFE5524D
:10EEA000E552020EDB1C010107170BD0F0EC91F0CC
:10EEB0005DEC8BF0080EE66E11EC89F062DFE55236
:10EEC000E552020EE3EC91F099D7FAEC8CF030ECBD
:10EED00088F004EC8DF030EC88F09FEC8AF030EC98
:10EEE00088F0E4EC93F007C1E6FF4B0E64EC8FF082
:10EEF0006EDF030EE15C02E2E16AE552E16E94EF3F
:10EF000087F02FEC90F0000EE66E010EE66E9BECA3
:10EF10008AF0A0EC87F0010E0101005D02E2010E13
:10EF2000006F060EE66E010EE66E430E71EC8FF07A
:10EF3000070EE66E010EE66E4B0E71EC8FF0010EC1
:10EF4000E66E010E0AEC88F0E66AA0EC87F0020E8D
:10EF5000E66E010EE66E020E68EC8FF0030EE66EB2
:10EF6000010E15EC88F0E66AA0EC87F0040EE66E60
:10EF7000010EE66E040E68EC8FF0050EE66E010ED3
:10EF8000E66E050E68EC8FF06D0EE66E010EE66E15
:10EF90009CEC95F06E0EE66E010EE66EB9EC8DF00F
:10EFA000A0EC87F06F0EE66E010EE66E4A0E71EC75
:10EFB0008FF0700EE66E010EE66EBCEC8DF0A0ECEC
:10EFC00087F0710EE66E010EE66E400E71EC8FF06A
:10EFD000720EE66E010EE66E470E71EC8FF0730E48
:10EFE000E66E010EE66E480E71EC8FF0DE6ADD6AA9
:10EFF000C1EC88F0050E56EC93F01DE2C2EC8CF0EB
:10F00000F4EC89F0DAEC89F0C6EC88F0A0EC87F03B
:10F01000C2EC8CF0F4EC89F0EE52DAEC89F0010EDF
:10F020001626000EB6EC96F0A0EC87F0DF2A010E53
:10F03000DFE3DB2ADDD7D5EC8CF0B0EC87F0080EEF
:10F04000E66E010EE66E270E68EC8FF0090EE66E96
:10F05000010EE66E280E68EC8FF00A0EE66E010EC9
:10F06000E66E290E68EC8FF00B0EE66E010EE66E72
:10F07000360E71EC8FF00C0EE66E010EE66E370E5A
:10F0800071EC8FF00D0EE66E010EE66EB80E86EC9A
:10F090008FF00E0EE66E010EE66E350E71EC8FF0FF
:10F0A0000F0EE66E010EE66E2A0E68EC8FF0100E63
:10F0B000E66E010EE66E2B0E68EC8FF0110EE66E1A
:10F0C000010EE66EC00E86EC8FF0120EE66E010E9B
:10F0D000E66E380E71EC8FF0130EE66E010EE66EE2
:10F0E000C10E86EC8FF0140EE66E010EE66E390E40
:10F0F00071EC8FF0150EE66E010EE66EC20E86EC18
:10F100008FF0160EE66E010EE66E3A0E71EC8FF081
:10F11000170EE66E010EE66E440E71EC8FF0180EBF
:10F12000E66E010EE66E3B0E71EC8FF0190EE66E88
:10F13000010EE66E3C0E71EC8FF01A0EE66E010EBB
:10F14000E66EC30E86EC8FF01B0EE66E010EE66EC9
:10F150002C0E68EC8FF01C0EE66E010EE66E2D0E86
:10F1600068EC8FF01D0EE66E010EE66E2E0E68EC5A
:10F170008FF01E0EE66E010EE66E2F0E68EC8FF01D
:10F180002A0EE66E010EE66EB90E86EC8FF02B0E9F
:10F19000E66E010EE66E420E71EC8FF061EC8CF0C3
:10F1A000B0EC87F06AEC8CF0B0EC87F0DE6ADD6AD8
:10F1B000C1EC88F0080E56EC93F016E2E00E146EE7
:10F1C000C2EC8CF0BE0EE926080EEA221450EF16AF
:10F1D000C2EC8CF0C60EE926080EEA22EF8ADF2A7E
:10F1E000010EE6E3DB2AE4D71F0EE66E010EE66EA3
:10F1F000300E68EC8FF0200EE66E010EE66E310EDA
:10F2000068EC8FF0210EE66E010EE66EA20E86EC23
:10F210008FF0220EE66E010EE66EA30E86EC8FF0E6
:10F22000230EE66E010EE66EA40E86EC8FF0240E21
:10F23000E66E010EE66EA50E86EC8FF0250EE66EEC
:10F24000010EE66EA60E86EC8FF0260EE66E010E1F
:10F25000E66E4C0E71EC8FF023EC96F0280EE66E05
:10F26000010EE66E490E71EC8FF0290EE66E010E6E
:10F27000E66E3F0E71EC8FF02E0EE66E010EE66E1E
:10F28000BE0EDFEC94F084EC88F02C0EE66E010EDE
:10F29000E66EBC0EDFEC94F084EC88F0300EE66E87
:10F2A000010E31EC8FF0A0EC87F0310EE66E010E0E
:10F2B000E66E330E68EC8FF0320EE66E010EE66EEF
:10F2C000340E68EC8FF0330EE66E010EE66E350EEE
:10F2D00068EC8FF0340EE66E010EE66E3D0E71ECBA
:10F2E0008FF0350EE66E010EE66E360E68EC8FF08E
:10F2F000360EE66E010EE66E370E68EC8FF0370EB6
:10F30000E66E010EE66E380E68EC8FF0BC0EE66E0F
:10F31000080EE66E450E52EC93F03A0EE66E010EC4
:10F32000E66EB70E86EC8FF0AE0EE66E080EE66E59
:10F33000240E52EC93F0B00EE66E080EE66E260E2A
:10F3400052EC93F0B20EE66E080EE66E280E71ECEB
:10F350008FF0B50EE66E080EE66E2B0E71EC8FF098
:10F36000B60EE66E080EE66E2C0E71EC8FF0B70E40
:10F37000E66E080EE66E2D0E52EC93F0BA0EE66EB7
:10F38000080EE66E300E71EC8FF0BB0EE66E080EC6
:10F39000E66E310E71EC8FF0B30EE66E080EE66E7F
:10F3A000290E71EC8FF0B40EE66E080EE66E2A0E92
:10F3B00071EC8FF0B90EE66E080EE66E2F0E71EC52
:10F3C0008FF0380EE66E010EE66E390E68EC8FF0A7
:10F3D000390EE66E010EE66ED40E86EC8FF03B0E13
:10F3E000E66E010EE66E3A0E4DEC91F03D0EE66EC5
:10F3F000010EE66E3C0E4DEC91F03F0EE66E010EF6
:10F40000E66E3E0E4DEC91F0410EE66E010EE66E9C
:10F41000400E4DEC91F0430EE66E010EE66E420E8C
:10F4200068EC8FF0440EE66E010EE66E430E68EC5B
:10F430008FF0450EE66E010EE66E440E68EC8FF01E
:10F44000460EE66E010EE66E450E68EC8FF0470E36
:10F45000E66E010EE66E410E71EC8FF0480EE66E20
:10F46000010EE66E460E68EC8FF0490EE66E010E58
:10F47000E66E470E68EC8FF04A0EE66E010EE66E01
:10F48000490E68EC8FF04B0EE66E010EE66E480EEC
:10F4900068EC8FF04C0EE66E010EE66E4A0E68ECDC
:10F4A0008FF0CE0EE66E080EE66EF10E4DEC91F08A
:10F4B000D20EE66E080EE66EF50E68EC8FF0D30EF7
:10F4C000E66E080EE66EF60E68EC8FF0D40EE66E71
:10F4D000080EE66EF70E4DEC91F0D80EE66E080EB3
:10F4E000E66EFB0E4DEC91F0D60EE66E080EE66E63
:10F4F000F90E68EC8FF0DA0EE66E080EE66EFD0E81
:10F5000068EC8FF0D10EE66E080EE66EF40E68EC35
:10F510008FF0D70EE66E080EE66EFA0E68EC8FF0EE
:10F52000DB0EE66E080EE66EFE0E68EC8FF0140E33
:10F53000E66EF4EC92F025EC92F044EC8EF0E66E80
:10F54000740E25EC92F0FAEC92F025EC92F000ECBF
:10F5500093F0A8EC95F010EC8BF0B0EC87F0380E3F
:10F56000E66EC70EE66E020EE66EB00EA8EC95F0E3
:10F57000030EE66E8FEC92F0030EE66EEC0EE66E76
:10F58000060EE66E1A0E6CEC8FF0EF0EE66E060EAF
:10F59000E66E350E6CEC8FF0F20EE66E060EE66E41
:10F5A000500E6CEC8FF0F50EE66E060EE66E6B0EEE
:10F5B0006CEC8FF0F80EE66E060EE66E860E6CECC6
:10F5C0008FF0FA0EE66E010EE66EA10E6CEC8FF077
:10F5D000FD0EE66E010EE66EA40E6CEC8FF0EE0EE4
:10F5E000E66E0D0EE66EA70E6CEC8FF0F10EE66E79
:10F5F0000D0EE66EAA0E6CEC8FF0F40EE66E0D0E9C
:10F60000E66EAD0E6CEC8FF0F70EE66E0D0EE66E4C
:10F61000B00E6CEC8FF0FA0EE66E0D0EE66EB30EC9
:10F620006CEC8FF0FD0EE66E0D0EE66EB60E6CEC19
:10F630008FF0600EE66E080EE66ED10E6CEC8FF069
:10F640006C0EE66E080EE66EDD0E6CEC8FF06F0E43
:10F65000E66E080EE66EE00E6CEC8FF0660EE66E5F
:10F66000080EE66ED70E6CEC8FF0690EE66E080E93
:10F67000E66EDA0E6CEC8FF0630EE66E080EE66E48
:10F68000D40E6CEC8FF0720EE66E080EE66E1D0E58
:10F69000EFEC93F0750EE66E080EE66E200EEFECC2
:10F6A00093F0FB0EE66E060EE66E320E15EC88F059
:10F6B000B0EC87F0600EE66E010EE66EBB0E86ECD7
:10F6C0008FF032EC96F062EC90F0300EE66E080EA1
:10F6D000E66E1D0E62EC90F0180EE66E080EE66EF9
:10F6E000380E62EC90F0000EE66E080EE66E530ED9
:10F6F00062EC90F0A10EE66E060EE66E6E0E62EC07
:10F7000090F0D10EE66E060EE66E890E62EC90F079
:10F71000B90EE66E060EE66EB90E0CEC96F0040E0F
:10F72000E66EE00EE66E000EE66EC40E9FEC96F0FE
:10F73000E40EE66E000EE66EC80E9FEC96F0E80E44
:10F74000E66E000EE66ECC0E9FEC96F0EC0EE66ECA
:10F75000000EE66ED00E85EC90F0610EE66E0D0E9A
:10F76000E66EF00E68EC8FF0690EE66E010EE66E46
:10F770009C0E86EC8FF06A0EE66E010EE66E230E8E
:10F7800071EC8FF06B0EE66E010EE66E9D0E86EC50
:10F790008FF06C0EE66E010EE66E36EC8FF0A0EC8C
:10F7A00087F05BEC76F08C0E7FEC90F0B0EC87F09D
:10F7B000FAEC8CF0B0EC87F004EC8DF0B0EC87F054
:10F7C0009FEC8AF0B0EC87F0240EE66E640EE66ED5
:10F7D000060EE66E700E85EC90F0040EE15C02E21F
:10F7E000E16AE552E16E94EF87F099928782640EA8
:10F7F000D6EC8EF087921200D8EC8FF0F6EC93F0F6
:10F800000AE00A0ED6EC8EF0F6EC93F002E0000E61
:10F8100003D0010E01D0010E0FEC8CF002E2E16A80
:10F82000E552E16E145094EF87F08AEC8FF0DE6AB7
:10F83000DD6AC1EC88F0080E56EC93F00BE2DFCFE6
:10F84000E6FFDADFE552000905E0DF2A010EF1E309
:10F85000DB2AEFD7DF50C4EC8DF002E2E16AE5521B
:10F86000E16E145094EF87F08AEC8FF00101746B15
:10F87000DF6A740EE66E010EE66E550E71EC8FF0C7
:10F88000070E0101745D02E1010EDF6EDF50C4EC72
:10F890008DF002E2E16AE552E16E145094EF87F0D8
:10F8A000B6EC8FF0DF6AFE0EDB0406E179EC89F03E
:10F8B000550EE66E390E09D0FE0EDB5002080FE140
:10F8C00079EC89F0550EE66E6F0EE66EA0EC87F0CF
:10F8D000070E146EDF50145C04E1010E03D0000E1D
:10F8E00001D0000EE55294EF87F0E668E6684BEC35
:10F8F0008FF057ECB3F0050EE15E1200AB0E0AEC90
:10F9000088F09BEC8AF026EF8EF0E66A190EE66E20
:10F91000E66A040EE66E26EF8EF046EC92F00101E8
:10F92000876B140E4DEC89F00101A46FE66ADEECE2
:10F9300005F0E5520101886FE850146E156AD89001
:10F94000155004E6C80E145C000E155802E2A4051A
:10F950000BE0885192EC8AF001E1155002E0A40519
:10F960001FE0010E876F1CD0882B88C1E6FFE66A76
:10F9700089EC94F0D0B205D0030E06EC93F0030EA0
:10F980000DD0D0B805D0040E06EC93F0040E06D0CE
:10F99000D0B606D0050E06EC93F0050EB8EC88F054
:10F9A0000101A46BD082D088D086875106E15CDF4C
:10F9B000000903E081EC77F078D0E66A140EB8EC29
:10F9C00088F00101876B885192EC8AF01BE1155099
:10F9D00019E1886B876BE66AE66A89EC94F0E66A5F
:10F9E000010EAEEC94F0020EAEEC94F0030EAEEC11
:10F9F00094F0040EAEEC94F0050EAEEC94F0060E0E
:10FA0000B8EC88F0BAEC70F0C5EC70F0E668F6EC93
:10FA100076F0E55268EC16F0FDC8E6FFFEC8E6FF9A
:10FA2000900EE66E2E0EE66E010E31EC8FF08DEC30
:10FA300016F040EC91F0FBC8E6FFFCC8E6FF500E64
:10FA4000E66E2E0EE66E010EE66EFBC814F0FCC8E4
:10FA500015F0320EB4EC8DF04BEC92F08DEC16F00C
:10FA600084EC94F042DFEEEC88F00A0E8EEC94F019
:10FA70000B0EB8EC88F042DFEEEC88F00C0E8EEC4A
:10FA800094F00D0EB8EC88F040DFEEEC88F00E0E2E
:10FA90008EEC94F00F0EB8EC88F0010EE66E140EAA
:10FAA000B8EC88F00101010EA46FBFDEDF6ECCEC74
:10FAB0008DF002E2DFCF00F1AD6BDF6ACCEC8DF0B0
:10FAC00057E2BEEC8FF00C0E4EEC8CF097EC8EF003
:10FAD00000094CE1BEEC8FF0A6ECAEF0E552E55229
:10FAE000D950080F8CEC90F0970EEE6E050EED6E6F
:10FAF000DDEC8EF0EF500FE0DDEC8EF0A2EC8BF041
:10FB000016BE1768C6EC94F006E0080EDB2A090E54
:10FB1000EFE3DB2AEDD7146A14C0E6FF080EE66EA9
:10FB2000E66AD80EE66E630EE66E010EE66E080E0D
:10FB3000DBCFE6FF090EDBCFE6FFDEECADF0156EA6
:10FB4000070E0CEC93F0E76E1418E8AE02D0E73421
:10FB500002D0E750145C0AE2010EDF5205E0DFCF6D
:10FB6000F3FF38EC8BF0FDE10101AD13DF2AA6D7DE
:10FB700092EC94F003E071EC8AF0FDE1A7EC88F0E0
:10FB8000DB1C5AEC92F001010117020EDB50021748
:10FB9000020EDB500317020EDB500417020EDB507F
:10FBA0001F17A56BA66B5BEC76F0DF6A010EDB6AB4
:10FBB000050EDF5C06E2FEEC94F06FEC8DF0DF2AC0
:10FBC000F7D7010EDB1C12E0010EDB1C06019C11B5
:10FBD000E66E040EE66E94EC8BF0010EDB5006012F
:10FBE0009C15E66E040EE66E99EC8BF026C195F13D
:10FBF000DF6A050EDF5C0CE2FEEC94F0020EDB50D7
:10FC0000EF1625EC97F002E094EC8FF0DF2AF1D7A5
:10FC100034EC95F0D7EC8AF08DEC8AF003E09EECA2
:10FC20008BF0FDE17EEC89F000C1DFFFDF5071E079
:10FC3000E1EC87F0EF6AE1EC87F0070E12EC93F04D
:10FC4000030E12EC93F0040E12EC93F0C0EC87F06C
:10FC5000020EEF6ED4EC88F0EF6ADF042AEC8CF031
:10FC6000600EEF6E9BEC8AF0156ADF34FE0B1536E2
:10FC7000146E900E1426000E1522020E145E000E55
:10FC8000155A4BEC92F044EC89F0E552DF04EA6A35
:10FC90001A0FE96E090EEA22EF6AE1EC87F0020E14
:10FCA000DDEC96F0030EDB500801B31505E0AEC89D
:10FCB000E6FFAFC8E6FF08D0030EDB50B41508E03E
:10FCC000B0C8E6FFB1C8E6FFE4EC8EF096EC92F027
:10FCD000DF0476EC8DF0B2C8EFFF030EDB500801B5
:10FCE000B9150EE0B7C8E6FFB8C8E6FFE4EC8EF041
:10FCF000B80E1426000EC8EC87F044EC89F0E552EB
:10FD0000030E7DEC88F0D950040F60EC88F0DF061C
:10FD10008DD7E66A080EE66EEDEC37F0E552E55257
:10FD2000CEC8E6FFCFC8E6FF2DEC03F0E552E55262
:10FD3000D1C8E6FFEEEC02F0E552E66A080EE66E88
:10FD40001BEC8BF0010E15EC93F0020E15EC93F00A
:10FD5000030E15EC93F00101880EB46F060EB56F1B
:10FD6000B66BB36BE66A4BEC8FF0460EE66E0D0E8B
:10FD7000E66E8DEC00F048EC89F03BEC88F006C0B4
:10FD8000B7F107C0B8F108C0B9F109C0BAF1010173
:10FD9000AE6B080EAF6F916F70EC8EF001017A6B55
:10FDA000B16BB06BB26B0501506B0F01006B0101C1
:10FDB000896B8D6B8E6B8F6B3BEC88F006C07BF193
:10FDC00007C07CF108C07DF109C07EF154EC8DF0D4
:10FDD0001EEC8DF001018A6B8B6B8C6B926B936BBD
:10FDE000946B0601FE6B0601FF6B0101010E776F3C
:10FDF000E80E5D6F030E5E6F7F0E5F6F996B9A6BFF
:10FE00009B6B9C6B9D6B9E6B9F6BA06BA16BA26BA6
:10FE1000A36BAAECABF00101A86BA96BAA6BAB6B4F
:10FE20000D01780E446FDF6A080EDF5C06E2DF50DA
:10FE300084EC8BF0EF6ADF2AF7D7DF6A050EDF5C10
:10FE400003E253EC8FF0FAD70101A45107E0080E4A
:10FE5000AF6FAE81E66ED0EC29F0E552F3EC8BF09B
:10FE60002F0EAFEC8AF00A0EE15C02E2E16AE55285
:10FE7000E16E94EF87F0B6EC8FF099EC91F067E2C9
:10FE80008DEC88F003E003EC89F0FDE1F350DF6EC8
:10FE9000DF500801D21503E044EC8EF003D0580E79
:10FEA000E66E040EE66E8CEC93F039EC89F0DF50D0
:10FEB0000801D31508E0940EE66E040EE66E8CEC95
:10FEC00093F0DFEC8BF08CEC93F0E66E8CEC93F01F
:10FED000E66EA4EC96F0090EB8EC8AF03BEC91F0DB
:10FEE0008CEC93F039EC89F03BEC91F03BEC91F029
:10FEF000A4EC96F0170EB8EC8AF0F4EC8FF0EE520A
:10FF0000EF040FE1D7C8E6FF0A0E0DEC8AF0D6C861
:10FF1000E6FF190E0DEC8AF0D4C8E6FFD5C8E6FF5F
:10FF20000ED0DBC8E6FF0A0E0DEC8AF0DAC8E6FF59
:10FF3000190E0DEC8AF0D8C8E6FFD9C8E6FF0B0E03
:10FF4000B1EC95F014EC19F0BAEC8FF0E552E552F3
:10FF500094EF87F0D8EC8FF027EC91F038EC95F027
:10FF6000100ED880F354000EF45408E2100EE76E21
:10FF7000A0EC88F0E750C0EC87F0EF6A310E50EC4F
:10FF80008BF039EC8FF029EC93F039EC8FF039ECF1
:10FF90008FF0A4EC96F0160EB8EC8AF0DE6A200E14
:10FFA000DD6E020E60C1DBFFDECFE6FFFEEC88F007
:10FFB000DD5207EC8AF0030EE15C02E2E16AE552F1
:10FFC000E16E94EF87F0D8EC8FF0DF6ADE52010E1D
:10FFD000DD6ECCEC8DF047E28CEC8CF0E7143EE06B
:10FFE000E66ADFCFE6FF1BEC8BF0010E97EC94F096
:10FFF000020E97EC94F0030E97EC94F0DFCFE6FF3F
:020000040001F9
:100000003ADFE55261CDE6FF220E4EEC8CF00EECAD
:1000100019F0BAEC8FF0010EDB50010129151EE03A
:10002000230EFDEC93F0C8EC8EF0EF50800B03E054
:10003000240EFDEC93F091EC95F07AEC93F0A0ECAB
:1000400087F0020EDB500AE011EC89F0260E4EEC30
:100050008CF00EEC19F0E552E552E552DF2A010E64
:10006000C7EC89F0B6D7030EE15C02E2E16AE55223
:10007000E16E94EF87F032EC92F001019BEC94F08A
:100080001FEC97F014141514E5EC8AF09BEC94F037
:10009000030E60EC8FF01414151494EC91F09BECAB
:1000A00094F0C8EC95F01414151422EC8FF08DEC3C
:1000B0008AF003E09EEC8BF0FDE1DF6E34EC95F00E
:1000C00004EC94F0030E00C1DBFFDB5001E188D0AB
:1000D000ABEC91F0DF1401E17DD0040EDB50DF14B6
:1000E00025E00101921D146E97EC8AF047EC8FF029
:1000F0001414E66E06EC90F052EC89F0DF50011516
:10010000931503E1931DF4EC95F0A51D146EDF50DB
:100110000315141403E006EC90F0EF6A0351A515E3
:10012000E81C146EDF509415141403E006EC90F0F4
:10013000EF6A050EDB50DF1404E006EC90F0DF50B0
:10014000EF128CEC8EF0880E145E060E155A050E1A
:100150000D6E0E6A14C008F015C009F08AECB6F0F6
:1001600008C014F009C015F0010E08C0E7FFE752FF
:1001700003E071EC8AF0FDE10101951513E10EEC4D
:1001800088F0C8EC95F0DF140DE1DF50071504E0AE
:1001900006EC90F0075105D0071D146E06EC90F0A8
:1001A0001450EF16060EDB50DF1405E006EC90F05D
:1001B000060EDB50EF16060EDB1CDF1404E0060E05
:1001C000DB1CF4EC95F0030EDB0484EC8BF0EF1CED
:1001D000F4EC95F0DF90DF42DAEC92F0DB0675D7B5
:1001E000070EE15C02E2E16AE552E16E94EF87F00E
:1001F000CAEC94F003E003EC89F0FDE13CEC90F0F4
:1002000011E09FEC94F0DF50EF12DF500101031575
:1002100005E0DF1CA517DF5027159413E8EC87F0E5
:10022000010E01D0000EE55294EF87F0CAEC94F075
:1002300003E003EC89F0FDE13CEC90F010E0DF1C02
:10024000146E9FEC94F01450EF16DF50010103156B
:1002500002E0DF1CA517E8EC87F0010E01D0000ECC
:10026000E55294EF87F09FEC94F0EF6AA6EC91F0E2
:10027000FBEC94F0CFEC95F00101A517E8EF87F0C7
:1002800015EC95F0C4EC90F0146E50EC92F0EF1277
:10029000A6EC91F0040EC0EC87F0FE0EDBCFEFFF72
:1002A000E8EC87F094EF87F06EEC94F0A3EC94F018
:1002B000DF5205E0DFCFF3FF38EC8BF0FDE1E552D4
:1002C000E710156EFAEC87F01514146E50EC92F0EE
:1002D000EF120101011D0715156EA3EC94F0DF521A
:1002E00005E0DFCFF3FF38EC8BF0FDE1E552E710DE
:1002F0001510146EFAEC87F01414E66E040ED8ECA8
:1003000094F0E8EC87F0E55294EF87F0CAEC94F0B3
:1003100003E003EC89F0FDE1F350DF6E02EC8BF0BB
:10032000EB50DF1401010315A61507E0DF50A513FC
:10033000DF502815BDEC92F001D0010EE55294EF8C
:1003400087F0CAEC94F003E003EC89F0FDE1A9EC3E
:1003500096F007E0DF1CA517DF502715BDEC92F0E3
:1003600001D0010EE55294EF87F0CAEC94F003E05F
:1003700003EC89F0FDE1A9EC96F005E0DF502713CE
:100380002AEC8EF001D0010EE55294EF87F0CAEC12
:1003900094F003E003EC89F0FDE1A9EC96F005E0B0
:1003A000DF1C27172AEC8EF001D0010EE55294EFE6
:1003B00087F0B6EC8FF00101031DA5170351271537
:1003C0009413DF6A050EDF5C11E2FEEC94F0EE524E
:1003D000EFCF15F00101031D1510146EFEEC94F023
:1003E00050EC92F0EF1653EC8FF0ECD7E55294EF0F
:1003F00087F08FEC87F0EBEC8EF003E071EC8AF085
:10040000FDE1E81CDF6E010EDB6A050E0DEC89F0E4
:1004100021E201EC97F0DF50EF16010EC7EC96F0E9
:1004200034EC8EF06FEC95F01414E66E01EC97F05E
:10043000020ED8EC94F0010E17EC97F0E66E01EC8A
:1004400097F022EC97F001EC97F0FBEC94F0010EA2
:10045000DB2ADBD726C195F1020EE15C02E2E16AFC
:10046000E552E16E94EF87F08FEC87F0EBEC8EF0C5
:1004700003E071EC8AF0FDE1E81CDF6E050EF6EC9E
:1004800087F039E2FE0ED5EC8FF0DF50EF16FE0E4E
:10049000C7EC96F0EFCF14F0FE0E6FEC95F014144D
:1004A000C7EC8CF098EC87F0020ED8EC94F0FE0EBE
:1004B00017EC97F0C7EC8CF098EC87F022EC97F0F3
:1004C000FE0ED5EC8FF0FBEC94F08DEC88F003E0A1
:1004D00003EC89F0FDE1F35001012615146E8DEC5B
:1004E00088F003E003EC89F0FDE1F350F31C010117
:1004F00095151410956F010EDB6A050E0DEC89F051
:1005000018E273EC8CF012E001EC97F0DF501DEC78
:1005100095F050EC92F01DEC95F048EC93F01DEC4A
:1005200095F0040EC0EC87F01450EF16010EDB2A94
:10053000E4D7020EE15C02E2E16AE552E16E94EF7B
:1005400087F02DEC92F095EC95F09C0EEE6E060E79
:10055000ED6ECFEC87F0020EDDEC96F0CFEC87F07D
:10056000DDEC96F00BEC94F045EC8AF001E3DB2A2D
:10057000EFCFDFFFDF501BE099EC95F013E0300E7A
:10058000DF5C146E080E145CEFE2BAEC91F0ECE262
:10059000010EF36EDB5003E003EC89F0FDE142EC69
:1005A00090F0E2D76EEC96F0DFE1010E2AD0C5ECB8
:1005B00091F0040EF36E050ED1EC90F00AE2BEEC61
:1005C00095F0050ED5EC8FF0FBEC94F0050EDB2AD0
:1005D000F0D7040EE66E48DFE552100E0101261535
:1005E000146EEF0E95151410956F050EDB6A7EECF8
:1005F0008BF006E2050E8FEC8FF0EFEC8EF0F7D764
:10060000000E146E060EE15C02E2E16AE552E16E54
:10061000145094EF87F032EC92F00EEC88F0EFCFAC
:10062000DFFFDF500CE045EC91F016BE1768C6EC1A
:1006300094F005E0C0EC8BF0F0E3DB2AEED7A2ECFF
:1006400091F0F350F41037E0300EDF5C22EC8FF0C5
:10065000050EF36E060ED1EC90F02DE2C0EC8BF09F
:1006600001E3DB2A060EDB50FEEC96F0BBEC88F0D3
:100670000BEC94F045EC8AF001E3DB2AEFCFDFFFCF
:10068000DF501BE099EC95F013E0300EDF5C146E48
:10069000080E145CEFE2BAEC91F0ECE2010EF36E9E
:1006A000DB5003E003EC89F0FDE142EC90F0E2D78F
:1006B0006EEC96F0DFE1010E22D0C5EC91F07EECFD
:1006C0008BF00CE2060EDB50F36E050EDB50F35C94
:1006D00002E0BEEC95F0050EDB2AF1D7060EDBCF6B
:1006E000E6FFC2DEE552050EDB6A7EEC8BF006E229
:1006F000050E8FEC8FF0EFEC8EF0F7D7000E146E36
:10070000070EE15C02E2E16AE552E16E145094EFFB
:1007100087F0B6EC8FF0FDEC8FF06BDEDF6A050E34
:10072000DF5C03E253EC8FF0FAD7E55294EF87F0E9
:100730008AEC8FF0DF6A45EC8AF001E3DB2AB8EC43
:100740008CF01CE0D0EC88F0E66A1BEC97F0F3E14B
:100750001AEC93F0F4CF15F0F350F4100FE0380ECC
:100760000DEC89F00BE2010EDB50D00FACEC93F0F6
:1007700003E09EEC8BF0FDE1DF12DDD7DF50C4EC2F
:100780008DF002E2E16AE552E16E1450CDD3D8EC6F
:100790008FF00EEC88F0B8EC8CF00CE045EC91F0AA
:1007A00016BE1768C6EC94F005E0C0EC8BF0F1E3E0
:1007B000DB2AEFD71AEC93F075EC8FF003E0F4EC42
:1007C0008EF002E3010E3BD0C0EC8BF001E3DB2A9C
:1007D00073EC95F0FEEC94F06FEC8DF0DBCFE6FF60
:1007E000DFCFE6FF94EC8BF0020EDB6A29EC89F098
:1007F0001DE2DF50F36E020EDB50F35C14E0D0EC30
:1008000088F0020E6FEC95F0E552E7140CE0010E53
:10081000DB1C146E020E6FEC95F01414E66E11ECF6
:1008200089F094EC8BF0020EDB2AE0D73EEC8FF0DF
:1008300029EC89F003E2FAEC95F0FAD7000E0FEC00
:100840008CF002E2E16AE552E16E14506DD3D8EC0F
:100850008FF0E4DBB8EC8CF00CE045EC91F016BEC8
:100860001768C6EC94F005E0C0EC8BF0F2E3DB2AED
:10087000F0D71AEC93F075EC8FF003E0F4EC8EF007
:1008800002E3010E15D0C0EC8BF001E3DB2A73EC20
:1008900095F09FEC92F04EEC8CF099EC8BF03EECE6
:1008A0008FF029EC89F003E2FAEC95F0FAD7000E0C
:1008B0000FEC8CF002E2E16AE552E16E145034D3A1
:1008C000D8EC8FF089EC90F006E2FDEC90F0FE0E93
:1008D000EFCFDBFF02D0010E3DD0020EDB6A29EC28
:1008E00089F02FE2FDEC8FF0020EC7EC96F0010EBE
:1008F000EFCFDBFFFD0EDB500EE08DEC88F003E068
:1009000003EC89F0FDE1F350146E010EDBCFE7FF3D
:10091000F350E7120BD08DEC88F003E003EC89F084
:10092000FDE1F350F31CA4EC8DF0E716AAEC94F073
:10093000DBCFE6FF11EC89F099EC8BF0020EDB2A9D
:10094000CED73EEC8FF029EC89F003E2FAEC95F07B
:10095000FAD7000E0FEC8CF002E2E16AE552E16E8C
:100960001450E2D246EC92F0F80EDBCFE6FFF90E1F
:10097000DBCFE6FFCDDB020EF3CFDBFF080EDB6A39
:10098000DE6ADD6AC1EC88F0FA0EDBCF16F0FB0EF2
:10099000DBCF17F01650145C1750155862E2080EA2
:1009A000DB505FE10EEC8DF0060EF626000EF7220E
:1009B000F8220900F5CF18F00800F5CF19F018500B
:1009C00019104FE0F80EDBCF08F0F90EDBCF09F07D
:1009D000030E08C0DBFF040E09C0DBFF0EEC8DF038
:1009E000F6CF14F0F7CF15F0F8CF16F07EEC8EF0BE
:1009F000070E16C0DBFFB8DAEFCF14F01EEC8CF058
:100A0000145C11E1B1DAEF500EE0030EDB2A040EA4
:100A100001E3DB2AD950050F8CEC90F0EE2A000E92
:100A2000EE22EE22E8D7A0DAEF5003E0080EDB6AF0
:100A30000AD01EEC8CF002E0010E01D0020EF36E23
:100A4000080EF3CFDBFFD950FC0F7FEC94F0090EBA
:100A5000EE26000EEE22EE22DF2A010E93E3DB2AC1
:100A600091D7080EDB5002080AE18BDB1406000E5A
:100A7000155AF60EDBCFE9FFF70EFBEC8EF0080EF1
:100A8000DB50146E0A0EE15C02E2E16AE552E16EAF
:100A900014504AD244DA090EE126DEEC8AF0070E41
:100AA00008C0DBFF080E09C0DBFF060EDB6ADE6A4A
:100AB000DD6A67DBFC0EDB50176AE850145C1750E8
:100AC000155849E2060EDB50020845E0F90EDBCF6F
:100AD00008F0FA0EDBCF09F0020E08C0DBFF030EB0
:100AE00009C0DBFF070EDBCF08F0080EDBCF09F0F3
:100AF0001EEC92F054DAEFCF14F063DAEF50145C8E
:100B00000EE14DDAEF500BE0020EDB2A030E01E39B
:100B1000DB2A040EDB2A050EEDE3DB2AEBD73FDAF6
:100B2000EF500AE14EDAEF5002E0010E01D0020E62
:100B3000F36E060EF3CFDBFFFB0EDB50146E156A6F
:100B40009AEC8DF01450EE261550ED22DF2A010E9E
:100B5000B0E3DB2AAED7060EDB5002080AE111DB58
:100B60001406000E155AF70EDBCFE9FFF80EFBEC6A
:100B70008EF0060EDB50146E090EE15C02E2E16AB3
:100B8000E552E16E1450D0D1D8EC8FF0A4EC95F082
:100B9000FBD9DEDB000902E0FF0E2FD0DF6A140E66
:100BA000DF5C06E266EC8DF0EF5002E0DF2AF7D75B
:100BB000140EDF5C21E213EC97F0070EF35C000EDD
:100BC000F4581AE20FEC94F0620F146E0D0EE0D997
:100BD00040ECADF0FBEC96F0070EE66E0FEC94F0F7
:100BE000E40F146E010ED4D984EC6BF0166E050E72
:100BF000E15E1650DF5001D0FF0E0FEC8CF002E2E8
:100C0000E16AE552E16E14508FD18AEC8FF00FEC5F
:100C100097F075EC8FF00DE00FEC97F08AEC8BF00D
:100C2000070EF35C000EF45804E216EC94F0000991
:100C300002E0FF0E0CD0A8D9620EE66E0D0E19DB95
:100C4000070EC1EC96F0E40EE5D90ADA000EC4EC0A
:100C50008DF002E2E16AE552E16E145065D1D8EC04
:100C60008FF0020E146EE66EA4EC95F08DD9FBECBD
:100C700091F0156E080E0CEC93F0145C02E0FF0E80
:100C800002D0010EDB500FEC8CF002E2E16AE5527B
:100C9000E16E145049D1D8EC8FF016EC94F05AEC78
:100CA00092F0020817E16DDA153414E214500008CE
:100CB000000E15540FE2C2EC8CF0070EC6EC92F059
:100CC00002EC8FF05EDA070EDBEC95F081EC93F02E
:100CD000DF5001D0FF0E0FEC8CF002E2E16AE5522A
:100CE000E16E145021D115EC95F0DB50000818E2AC
:100CF000140E7CD915E2F9EC8AF0620EE9260D0E8D
:100D0000EA22EF500DE0F9EC8AF002EC8FF0FE0ED3
:100D1000DB50070D30D981EC93F0FE0EDB5001D093
:100D2000FF0E02D1B6EC8FF0DF68DF500AE0DF5033
:100D3000EA6A000FE96E0E0EEA22EF5002E1DF06CA
:100D4000F4D7DF50146E156AFF0EB4EC8DF014501A
:100D5000E552EAD0D9CFE6FFE1CFD9FF020EE12676
:100D6000010E0101AE151BE101017851791117E166
:100D70000601FE5114E17BEC04F0000910E1460E7F
:100D8000E66E0D0EE66EA3EC00F0E552E55206C0ED
:100D9000B7F107C0B8F108C0B9F109C0BAF1460E01
:100DA000E66E0D0EE66EA3EC00F0E552E552010191
:100DB000B751065C146E0101B8510758156E010158
:100DC000B9510858166E0101BA510958176ED880EA
:100DD000780E1454000E1554000E1654000E1754BD
:100DE00010E2010EE66EDEEC05F0E552DF6EDF2A62
:100DF000DFCFE6FF010EE66EE8EC05F0E552E552C6
:100E0000FF009D50020B09E09D50010B06E0F250DF
:100E1000800B03E0F250400B10E1020EE66EDEECB8
:100E200005F0E552DF6EDF2ADFCFE6FF020EE66E49
:100E3000E8EC05F0E552E552FF00010E0101AE15A8
:100E400060E10101785179115CE10601FE5159E13F
:100E50007BEC04F0000955E10D01445152E1010E13
:100E6000DB6A01010051F36E010EDBCFF4FFF3509A
:100E7000F45C44E2010EDBCFE6FFFCEC7BF0E552D4
:100E8000000911E1060EE66EDEEC05F0E552DF6EBC
:100E9000DF2ADFCFE6FF060EE66EE8EC05F0E5524E
:100EA000E552FF0028D0010EF36E010EDB5004E086
:100EB000D890F336E806FCE1F3500101AD151BE0D4
:100EC000270EE66E010EDBCFE6FF20EC19F0E552AF
:100ED000E552F350DF6EDF500EE1010EF36E010EAE
:100EE000DB5004E0D890F336E806FCE1F350E66E00
:100EF000E3EC7FF0E552010EDB2AB3D70D01780E4B
:100F0000446F0501505101E10400020EE15C02E270
:100F1000E16AE552E16EE552E7CFD9FF1200D9CF81
:100F2000E6FFE1CFD9FF1200E552E7CFD9FF12006B
:100F3000050D41EC92F0880EE926060EEA22120019
:100F4000CDEC6BF0D6EF94F090EC6BF0BAEF8FF045
:100F50000B0D41EC92F0000EE926040EEA2212007D
:100F6000BFEC6BF0EFEF8FF0030EDBCFE9FF040E69
:100F7000DBCFEAFF1200F3CF14F0F4CF15F012002C
:100F8000E926000EEA22120014EC96F00BEF90F026
:100F900015224BEF92F09AEC6BF0D6EF94F0020E24
:100FA000DBCFE9FF030EDBCFEAFF1200050EDBCF3C
:100FB000E9FF060EDBCFEAFF1200EA6ADB345DEFE1
:100FC00093F0040EDBCFE9FF050EDBCFEAFF120042
:100FD000B4C1E6FFB5C1E6FFACEF95F0640E142690
:100FE000060E1522F1510F01EEEF95F0F36EFE0E95
:100FF000D1EF90F0A6EC91F0EF5012001FECB8F09A
:10100000EFEC8FF01CEC94F0060EDBCFE6FF070E42
:1010100088EF93F0E66E010EE66E1200FD0EDBCF58
:10102000E9FFFE0EDBCFEAFF1200E66E030EE66E6E
:10103000120010EC95F040EC91F0BEEF8FF0DFEC79
:1010400091F01A0FE96E090EEA221200E76EAAEF7C
:1010500094F0010EDBCFE9FF020EDBCFEAFF1200B6
:1010600084EC6BF0EFEF8FF02DEC93F00B0E145E31
:10107000000E155A1200460EE66E0D0EE66EA3EC3B
:1010800000F0E552E5521200FB0EDBCFE6FFFC0E4E
:10109000DBCFE6FF1200E5520BEC90F0F6EC76F0B9
:1010A000E5520BEC90F075EC6DF0E5520101936B9D
:1010B00093C192F192EF94F023EC94F018EF96F034
:1010C0008CEC90F00B0EEE5E000EEF5A1200E81C56
:1010D00094EC91F0DB5001010117050EDB50021773
:1010E000050EDB500317050EDB500417F9EC81F0F9
:1010F000DF6A1200DB502AEF94F0DBCFF3FFF390AE
:10110000F342F3CFDBFF1200D7EC6BF0D6EF94F095
:101110007AECADF0E552E5521200010EF36EFE0ED0
:10112000DB501200E66EBEEC8FF072EF96F0030D0E
:1011300041EF92F0EA6A0A0FE96E090EEA22120004
:10114000FC0EDBCFE9FFFD0EDBCFEAFF1200E76EFE
:10115000020EE7CFDBFF12000BEC90F05EEC2AF002
:10116000BAEF8FF0E66EE66AAEEC6BF0D6EF94F075
:10117000E66E89EF94F0880E1426060E1522BDEF58
:1011800090F0DECF14F0DDCF15F0120016C0E6FFB0
:1011900017C0E6FF1200D9CFE9FFDACFEAFF12004D
:1011A000010EDBCFE6FF1200DF04E96EEA6AD89099
:1011B000E936EA36C80EE926000EEA22EE5212009F
:1011C00018EC16F064C7E9FF65C7EAFF1200DFEC10
:1011D00091F0700FE96E000EEA2212001CEC94F000
:1011E000FF0EE76E10EC92F0E7501416156A1450DB
:1011F000E66E120018EC96F0E66A1200DECFE6FF0B
:10120000DDCFE6FF1200D890F336E80612001FEC9F
:1012100093F0A4ECA3F0D6EF94F0F36E010ED1EFAF
:1012200090F0020EDBCFE6FF1200FE0EDBCFC2F124
:1012300046C141FDAFC1E6FFA5EC23F0E552010137
:10124000AE811200DFEC91F0680FE96E000EEA2229
:101250001200050EF36E020ED1EF90F0E66E61EC17
:10126000ADF0EFEF8FF0AFC1E6FF5EEC2AF0BAEF22
:101270008FF0E66E40ECADF0D6EF94F0156ADB34FB
:10128000FE0B1536146E120065EC00F0BAEF8FF00D
:10129000146E060EE15E14501200E66EDEEC05F0F0
:1012A000E5521200E552E750EF6E1200E12630ECF5
:1012B00094F0010EDF521200E66EF3EC38F0BAEF54
:1012C0008FF027EC91F081EF96F0E66A31ECA3F015
:1012D000156E060E0CEC93F0145C120088ECADF069
:1012E000BAEC8FF0140E075C000E0858000E095877
:1012F0001200D9CFE6FFDACFE6FF1200E76E030E49
:10130000E7CFDBFF1200C3EC17F0E552E552120005
:10131000E66A1CECA2F040EF91F00C6E0D6A0E6ACA
:101320001AC007F01BC008F01CC009F0E4ECB6F0CE
:1013300004C01AF005C01BF006C01CF017500424AE
:10134000146E18500520156E19500620166E1200E6
:10135000FBEC91F0146E080EE15E14501200B1EC3B
:1013600095F0F3EC18F0EFEF8FF006C0DEFF07C04A
:10137000DEFF08C0DEFF09C0DDFFDD52DD521200D6
:10138000B1EC95F0D5EC18F0E552E5521200DBCF48
:10139000F3FFF39EF346F3CFDBFF1200FE0EDBCF2D
:1013A00076F10101010EB36F1200D5EC17F0E55292
:1013B000E5521200E9CF14F0EACF15F0E9CFE6FFCD
:1013C000EACFE6FFDECF16F0DDCF17F0050E1702ED
:1013D000F3CF17F01602F3CF16F0F45017260E0EC7
:1013E0001626000E17221200050EC6EC92F0880E8B
:1013F000E926060EEA221200CBEC95F0E66E95EC9B
:1014000095F072EC94F03AEC96F056EF93F00BEC0A
:1014100090F09EEC19F0D6EF94F0B1EC95F00EEC54
:1014200019F0BAEF8FF0EE58000EEE58000EEE589D
:101430001200A3EC90F015220101B451141812000F
:101440001FECB8F0EFEC8FF00A0EF3CFDBFF0B0EC2
:10145000F4CFDBFF12001C50185C146E1D5019589D
:10146000156E1E501A58166E1F501B58176E12001C
:10147000EE50185C146EEE501958156EEE501A5856
:10148000166EEE501B58176E1200FD0EDBCFE9FFF3
:10149000DB2AFE0EDBCFEAFF1200DFEC91F0800FBB
:1014A000E96E000EEA221200DFEC91F04D0FE96EBA
:1014B000010EEA221200DFEC91F0550FE96E010EE9
:1014C000EA221200790EE66E650EE66E010EE66EF9
:1014D0001200C5EC93F01EEC92F095EC95F089EFBC
:1014E00096F0E846FE0BE706120010EC92F015C0ED
:1014F00014F0156A1450E66E1200F350DF6EA4EF7C
:1015000095F0BDEC96F0EEEF92F00BEC90F0E3EC82
:101510007FF0E552060EE15C12000005146E010E2C
:1015200014521200146E156AFF0E14181200040EE5
:10153000DBCFE6FF1200000EE66EE66A1200080E30
:10154000E66E610EE66E010EE66E940EDFEF94F02D
:10155000176ED8801E0E1454000E37EF94F0E66E0E
:10156000E66AB5EC15F0FBEC96F00F01086B120083
:10157000B1EC95F0F3EC18F0166E050EE15E165026
:101580001200030E14C0DBFF040E15C0DBFF1200B7
:10159000F36EFD0ED1EF90F0D950FD0F7FEF94F078
:1015A000040EDBCF14F0050EDBCF15F01200040E95
:1015B00014C0DBFF050E15C0DBFF1200FD0EDBCFF4
:1015C00008F0FE0EDBCF09F01200E76E040EE7CF45
:1015D000DBFF1200E96E000EDA20EA6E1200146ED4
:1015E000EF501414E66E1200E66A68ECA3F040EFC8
:1015F00091F0FE0EDB50070D41EF92F0A6EC91F05A
:10160000030E1200A6EC91F0020E1200146E050EED
:10161000DBCFE7FF1450E716050EE7CFDBFF120024
:10162000050EE66E3BEC91F05B0EE66EE66A12008C
:101630009E0EDFEF94F028EC39F0E552E5521200EF
:1016400010EC95F0146E0B0EE15E1450BEEF8FF0AF
:10165000020EDBCF07F0030EDBCF08F0040EDBCF6A
:1016600009F0050EDBCF0AF00A34000E0A1812004A
:10167000E846FE0BF30612001A24186E000E1B201B
:10168000196E18C0E6FFE66E84EC6BF01C6E050E5A
:10169000E15E1C50120004EC94F000C1DFFF120068
:1016A000E66EE66A27EF91F0A517EF50E81C941755
:1016B000EF500315271594131200EF6E020EDB5046
:1016C00001016C13020EDB5007131200E552E552C4
:1016D000F3CFDEFFF4CFDDFF120031ECBAF0146E71
:1016E000090EE15E14501200BAEC8FF0DF6EDF508D
:1016F00012008CEC90F0EE50ED101200F36EDBCF88
:10170000F4FFE850F45C1200EA6A120FE96E090E69
:10171000EA221200F3CF16F0F4CF17F01200010EF8
:10172000B6C1E7FFE7521200A6EC6FF0E552E552B2
:101730001200BBEC6FF0E552E5521200E846FE0BDA
:1017400014061200EFCF16F0176A12004BEC92F05D
:10175000EAEC17F0E552E552F350E66E82EC24F025
:10176000E5521200DECF07F0DECF08F0DECF09F041
:10177000DDCF0AF0DD52DD520A34000E0A181200E5
:10178000FD0EDB2AFE0E1200E66ED950080FF8ECB3
:101790008FF081EF96F0DFEC91F0600FE96E000EB4
:1017A000EA221200EA22EECFE6FFEECFE6FFEFCF0D
:1017B000E6FF1200E66E2DECAEF040EF91F0E66E23
:1017C000EAECACF0D6EF94F0E65230EF94F00BEC8C
:1017D00090F014EC34F0E552DF6E1200E66A1CEC77
:1017E000A2F084EF94F00101080EAF6FF20EE66EE6
:1017F000080EE66E1200F36E020EF3CFDBFF12004E
:10180000010EDB500101AF5D12009217EF50E81C92
:1018100093171200E66AC1EC33F0E5521200146E21
:10182000030EE15C1200FE0EDB5008081200E66EAB
:10183000E66AFB0EDBCFE6FF23EF94F0050EDBCF6D
:10184000F6FF060EDBCFF7FF070EDBCFF8FF080031
:10185000F5501200EA6AD80FE96E000EEA22120073
:10186000D5EC23F0080E0101AF5D120038EC2DF02D
:10187000E552E552000912000854000E0954000E0A
:101880000A541200DFCFE6FFE66A1200146E040E5F
:10189000E15C12000101F051040D1200E66EDFCF91
:1018A000E6FF12000A0EDBCFE6FF0B0E88EF93F087
:1018B000030EDBCF14F0040EDBCF15F0080E56EF4D
:1018C00093F0080EE66EBE0EE66E080EE66EA70EEC
:1018D000DFEF94F0080EE66EC60EE66E080EE66EBA
:1018E000AF0EDFEF94F0FE0EDB50F36E010EDB5017
:1018F000F35C120024EC93F061EF0FF0DF04EA6A6E
:10190000780FE96E000EEA221200DF2A020EDBCF0A
:10191000F3FFF39EF3461200A3EC94F0DB50E55284
:101920001200DF502AEF94F0640E1426060E1522E2
:10193000FD0EDB501200D950020F146EDACF15F0F5
:10194000DF501200FE0EDB1C01010217FE0EDB1C35
:101950001200ACEC95F0020EDB2A1200E66E4CECA5
:101960000FF0E552120006C0DEFF07C0DDFF1200D7
:10197000010EEFCFDBFFEF501200E126040EE66E02
:10198000D9501200DECFE9FFDDCFEAFF1200E66E8C
:10199000FE0EDB501200EF50E66EF1C1E6FFF0C123
:1019A000E6FFDCEC38F0E5521200080EE66E0A0E97
:1019B000E66E090EE66E060EE66EE66A1200DFCFF0
:1019C000E9FF010EDBCFEAFF0A0EE926090EEA2243
:1019D0001200EA22FD0EDBCFEFFF14EC96F0FE0EB4
:1019E000DB501200C7DAEC0EE66E630EE66E010EF7
:1019F000E66E1200080EE66E4D0EE66E010EE66E05
:101A00004B0EE66EE66A1200080EE66E550EE66EA6
:101A1000010EE66E530EE66EE66A1200FC0EDBCF98
:101A2000F6FFFD0EDBCFF7FFFE0EDBCFF8FF120057
:101A3000DFCFE6FF9EEC19F0D6EF94F006C07FF101
:101A400007C080F108C081F109C082F11200145072
:101A5000185C1550195816501A5817501B58120078
:101A60000101AF51EA6A700FE96E000EEA22EF50F1
:101A7000120091EC95F0020EE66E120010EC95F05B
:101A8000166E1200030EDBCFE7FFF350E712030ED2
:101A9000E7CFDBFF1200AFC1E6FFB9EC29F0E5525A
:101AA0000101786B796B120006C083F107C084F1E5
:101AB00008C085F109C086F112001A1D156E030ECB
:101AC000DB50F36E030EDB50F35C1200070EDF02F7
:101AD000F350EA6A620FE96E0D0EEA221200010E5F
:101AE000DBCFE7FFEF50E712AAEF94F0EA6AB00FFE
:101AF000E96E000EEA221200EA6A000FE96E070E94
:101B0000EA221200F3CF18F0F4CF19F0F3501200CC
:101B1000DBCFE6FF020EDB50E5521200186A196AAD
:101B2000010E1A6E1B6A1200141401010115E81C43
:101B30006D171200D950070F8CEF90F0E66E50EC45
:101B40007CF0E55200091200146E010EDBCFE7FFB6
:101B500014501200010EF36EFD0EDB5012006E1DCC
:101B6000156E6D1D146E1200D8801456000E155699
:101B70001200A00EDFEF94F0A10EDFEF94F0140E30
:101B8000F35C000EF4581200146E020EE15C1200B9
:101B9000020E0101AE15120001010051DF5C1200BE
:101BA000DB50010101151200E652030EE66E120031
:101BB000FB0FE66EFF0EDA20DFEF94F0F90FE66E12
:101BC000FF0EDA20E66E040EE66E1200070E7615A2
:101BD000E66E59EC1DF0E55200091200020EE126F6
:101BE000DE52010EDD6E00C1DFFF120095DA1450E7
:101BF000EE121550ED1212001454010E37EF94F04E
:101C0000080EDB50EA6AE00FE96E010EEA221200CC
:101C1000010EF36E090EF3CFDBFF080EDB6A120034
:101C2000166E020EEB501614156E010EEB501200DC
:101C3000C6DB880FE96E000EEA221200166A176AE8
:101C40003C0E0B6E0C6A0D6A0E6A1200FEECB3F0CD
:101C5000D6EF94F0E0D9A1EC81F0E552000E12002D
:101C6000020EDB500F0B1200EFCF14F0010E12002A
:101C7000050EDBCFE6FF1200E12601010051120044
:101C8000EE52EF50020812006C0EE66E040E1200C7
:101C9000010E176ADB34FE0B1736166E1200390E72
:101CA000E66E660EE66E010EE66E1200DF04E66E6C
:101CB000FAEC1BF0E55200091200E552E7CF17F0ED
:101CC000E552E7CF16F01200E552E7CF15F0E552E6
:101CD000E7CF14F012009FD944EC22F0E552120035
:101CE0000701006B000E646F070E656F1200FB0E9C
:101CF000DBCFE9FFFC0EDBCFEAFF1200050E14C0BC
:101D0000DBFF060E15C0DBFF12000101020EB36FF0
:101D1000FE0EDBCF76F11200FD0EDBCF14F0FE0ECF
:101D2000DBCF15F01200F36E080ED1EF90F06CECE3
:101D300019F0D6EF94F0DFCFE6FF49EC24F0E5523E
:101D4000DF2A120003DB010EEB501200F3501B6A76
:101D5000700F1A6E020E1B221200EF50E66EF1C1D8
:101D6000E6FF1FEF6BF0050DF3CFB4F1F4CFB5F143
:101D7000880E1200020EDBCF02F1030EDBCF03F15F
:101D8000120084EC6BF0186E050EE15E1850120024
:101D9000DF50EA6AC60FE96E080EEA221200F40E5E
:101DA000E66E630EE66E010EE66E1200E66EE66A01
:101DB00015EC00F0E552E5521200080EDBCFE9FF0A
:101DC000090EDBCFEAFF1200DF04146E156AD8900B
:101DD000143615361200020EE12692EF94F0ACECA8
:101DE00095F0050EDB2A1200010EDB50D00FDF6EDE
:101DF000050EDF5C1200DBCFEAFF14C0EEFF15C05A
:101E0000EDFF1200620EE9260D0EEA22EF6AE66A85
:101E10001200DF6A010EF36E020E12009CEC1FF03E
:101E2000E552000912003FC1E6FF40C1E6FF120083
:101E300018EC21F0E552E5521200010EAFC1E7FFA8
:101E4000E7521200E76E060EE7CFDBFF1200EFCF7E
:101E5000DFFF010EDF521200030EDB5001019E1561
:101E60001200E66E320EE66EE66A1200BA0EDFEF80
:101E700094F0C60EE66E030EE66E1200F9EC81F0E9
:101E8000020EDB6A1200020EDB5002151200DF1C8C
:101E9000E552E7141200E66AE66AE66A1200E66AAC
:101EA000360EE66E1200DF508CEC95F0C8EC87F031
:101EB000ACEC95F0DF2A1200E66EE66AA4EF87F03C
:101EC000C0EC87F0EF50120015EC88F0A4EF87F01B
:101ED000E66EE66AA0EF87F00CEC96F0030EE66E75
:101EE000120015EC88F0A0EF87F0BBEC87F0F35000
:101EF000F4101200070DBBEC87F0C70E1426020E7B
:101F0000C8EF87F0DFEC94F0A4EF87F0DFEC94F0FB
:101F1000A0EF87F08FEC87F0020EE1261200DB5075
:101F20008CEC95F0C8EF87F0FEEC94F0EE52EFCF1A
:101F300014F025EC97F01414E66EFEEC94F0020E0B
:101F4000D8EC94F025EC97F001010115E66EFEEC5B
:101F500094F022EC97F0FEEC94F0FBEF94F03EEC62
:101F600089F0900E1426000EC8EF87F08FEC87F0F2
:101F7000E6521200E552E552E5521200970EE66E67
:101F8000050EE66E12000AEC88F0CBEF87F00AEC43
:101F900088F0A4EF87F08FEC87F0060EEEDC010FDF
